:100000000C944B100C9473100C9473100C9473108C
:100010000C9473100C9473100C9473100C94731054
:100020000C9473100C9473100C9477160C94DD6A76
:100030000C941D6F0C942C6B0C9473100C94001783
:100040000C9465160C9473100C9473100C9473102C
:100050000C9473100C9473100C9473100C94731014
:100060000C94A06F0C9446170C94916B0C94EA6F4F
:100070000C9473100C9473100C94B4690C9473105A
:100080000C9473100C9473100C947310DC18E0181B
:10009000A518AB18B118B118B118D418D818DC18B5
:1000A000E018ED18ED18E4184823482348234823A6
:1000B00075236C236C236C236C236C236C236C23BF
:1000C00058235D235D23ED2EF72E0D2F5A2F992FE8
:1000D000F72F023005305F306330A333B833543428
:1000E000DD356636E4349F39E437E736EF36773767
:1000F000E638DE42B142B442B842BE42C242C742D2
:10010000634B724B7D4B934B9A4BA14BB04BC74B00
:10011000DF4B4B4C764C7E4C864C924CB74CC74CCC
:10012000F14C3E4D4A4D854D9D4DAE4DBA4DC64D9F
:10013000D24DF850C45BCB53F8584B54C45BC45BEE
:10014000C8575E5AC45BC45B0E5308514F552E68A6
:100150001D6817681F68236827681A682B6831684C
:10016000076E0A6E216E3C6E3C6E216E216E1A7116
:100170001C711F7124713571447152715C716C7105
:100180007C71817197719A719E71A071A271A77132
:10019000AB71B671BA71C271C971CD71CF71D371C2
:1001A000D571D771D971DD71E171E671EB71F071C3
:1001B000F571FA71204F6C642056657273696F6E29
:1001C00020454550524F4D202020434845434B2069
:1001D00053455454494E47532F43414C49420041E3
:1001E0006C61726D732044697361626C6564004573
:1001F0004550524F4D206C6F77206D656D004C4F10
:100200004144494E47000553746F70706564006D3A
:10021000537461636B206F666C6F770053776974FA
:100220006368205761726E696E671F506C656173F9
:1002300065205265736574205377697463686573CC
:10024000005468726F74746C65206E6F74206964FA
:100250006C651F5265736574207468726F74746C7A
:1002600065004D45535341474500707265737320D7
:10027000616E79204B657900507265737320616EF1
:1002800079206B657920746F20736B6970004F461D
:10029000464F4E20544873544825002D2D2D002DD7
:1002A0002D2D2D0000006428100703010000000020
:1002B000010101020202020101030020414C4552EA
:1002C00054000001020300020103030102000302C3
:1002D00001000452756420456C6520546872204109
:1002E000696C20004F4E20004F4646000354485290
:1002F000525544454C4549443049443149443241C2
:10030000494C47454154524E4C31204C32204C33DD
:10031000204C34204C35204C36204C37204C382093
:100320004C39204C41204C42204C4320454C8045C8
:100330004C2D454C8152558052552D525581414985
:100340008041492D41498147458047452D47458199
:10035000504231504232001B1E272D36394B4E631E
:100360006C7278878D939CB1B4C6C9D2D8E1E4533E
:10037000706C6173680080400000000000000000A5
:10038000000000000000000000000000000000006D
:10039000000000000000000000000000000000005D
:1003A000000000000000000000000000000000004D
:1003B000000000000000000000000000000000003D
:1003C00000000080C0E0E0F0F8F8FCFCFCF8F8F871
:1003D000F04000000000008080800000000000006D
:1003E0000000000000000000000000000080C0C00D
:1003F000E0E0E0F0F0F0E0C00000000000C0F8FF36
:10040000FF9F878383838383838383838383838320
:10041000838383838383838383038380838383832F
:10042000838383838383838383838383838383839C
:10043000838383C3E3733F1F0000000080E0F0F874
:10044000FCFEFFFFFFFF7F3F1F1F0F0783C3E1E19C
:10045000E0E0C0000E1F3F7F7FFFF3E0E080000080
:10046000000000000000000080F0FCFEFFFFFFFF26
:100470007F3F0F0301010100000080F0FEFFFFC776
:10048000C1C1C1C1C1C1C1C1C1C1C1C1C1C1C1C15C
:10049000C1C1C1C1C1C101C1F0FEFF3F0F070F0DB6
:1004A0000D0D1D191919193131313171616161E178
:1004B000C1C1C18100000080E0F8FCFFFFFFFF2FF9
:1004C000170F038180C0E0F0F8FCFEFFFFFFFFFF85
:1004D000FF7F010000000000000001010307070E7C
:1004E0001E1C3870E0F0F8FEFFFF7F1F0F030001B5
:1004F00000000000000000000000000000000000FC
:1005000000000000000000000000000000000000EB
:1005100000000000000000000000000000000000DB
:1005200000000000000000000000000000000000CB
:100530000000000000007EFFFFFFFFFFFFFBF8FC54
:10054000FCFEFF7F3F1F0F07C3FFFFFFFFFFFF7F83
:10055000070000000000000000000000000000C0D4
:10056000E0F8FEFFFF7F1F0F1F3D7CF8F8F0E080F2
:10057000000000000000000000000000000000007B
:10058000000000000000000000000000000000006B
:10059000000000000000000000000000000000005B
:1005A000000000000000000000000000000000004B
:1005B0000000000000000000010101010103070725
:1005C000070301000000E0FCFFFFFFFFFF1F030027
:1005D00000000000000000000000C0F078DE2713DB
:1005E000090E0703000000000000000001030F7F58
:1005F000FFFC7878F8000000000000000000000018
:10060000808080808080808080008080008080006A
:1006100000000000000080808080808080808080DA
:1006200080808080808080800000000000000000CA
:1006300000000000000000000000000000000000BA
:1006400000000080F0FEFFFFFFFF3F0F01000000F1
:100650000000000000C0E0381E0F03000100000091
:10066000000000000000000000000000000000008A
:100670000000000303010000000000000000000073
:100680000E0E02020202020303000F0F000F0F08FA
:100690000808080808080F0F08080808080F0F00C6
:1006A0000000000F0F00000000000000000000002C
:1006B000000000000000000000000000000000003A
:1006C00000C0F8BFFFFFFF1F7F0100000000000017
:1006D0000000F0FCFF7F7830000000000000000008
:1006E000000000000000000000000000000000000A
:1006F00000000000000000000000000000000000FA
:1007000000000000000000000000000000000000E9
:1007100000000000000000000000000000000000D9
:1007200000000000000000000000000000000000C9
:100730000000000000000000000000000000003089
:100740001C070E0F07010000000000000000000061
:100750000000000000000000000000000000000099
:100760000000000000000000000000000000000089
:10077000000000000000000000564552533A205689
:10078000312E312D1F444154453A2033302E313221
:100790002E323031351F54494D453A2031303A35EB
:1007A000313A34301F2053564E3A20657239782D35
:1007B000723831391F204D4F443A20204E542020AA
:1007C0002020003C06064F4E202020204F46462089
:1007D0002020424F54482020313553656373333015
:1007E0005365637336305365637356617269626C27
:1007F000005653000720382053656373313220536D
:1008000065637331362053656373001E03015341E2
:100810005658004E756D62657220566F696365208B
:100820005377005361666574792053776974636800
:10083000657300434F5059205452494D205B4D453C
:100840004E555D000D4F6E004C4F474943414C20C3
:100850005357495443484553003C010A436F756E52
:100860007420446F776E436F756E7420557020202E
:100870000054696D65721F54726967676572411F24
:1008800054726967676572421F54696D65721F52C1
:1008900065736574205377697463680020547970B8
:1008A000651F20436F756E7472791F42696E641FF5
:1008B00052616E6765003C02094C50342F4C503534
:1008C000202044534D326F6E6C792044534D322FAB
:1008D00044534D580044534D205479706500014EE7
:1008E00059000B4F7074696F6E0004486967684C5B
:1008F0006F7720003C00044E6F6E65003C0105439D
:10090000473032335944383239003C0205475245AA
:10091000454E424C554520444D303037003C02078F
:1009200053594D4158202053594D41583543003CAF
:10093000040759443731372020534B59574C4B52F9
:1009400053594D4158322058494E58554E204E4922
:100950004855492020003C010444534D3244534D36
:1009600058003C01054869736B79484B33313000BE
:100970003C0306466C79736B7956397839202056DA
:100980003678362020563931322020003C0D06467C
:100990006C79736B7948756273616E4672736B79AB
:1009A000204869736B792056327832202044534DA9
:1009B0003220204465766F20205944373137204B50
:1009C0004E2020202053796D615820534C54202014
:1009D0002043583130202043473032332042617960
:1009E000616E670050726F746F636F6C1F54797023
:1009F000651F506F7765721F42696E64202020204A
:100A0000204175746F62696E641F52616E67650084
:100A1000660103504F534E454700506F6C61726939
:100A200074790050504D2046724C656E0D6D5365C3
:100A300063000C52784E756D0004344348203643F1
:100A4000482038434820313043483132434831341C
:100A500043483136434800137553000650504D202B
:100A6000202050585820202044534D3220205050F0
:100A70004D31362050504D53494D4D554C54492021
:100A800053425553202000317374204368616E1F18
:100A900050726F746F000444521F024578706F1FCC
:100AA0001F015765696768741F1F44725377311FB0
:100AB000447253773200034869204D6964204C6FBB
:100AC00077006604042D2D2D2D3132302031323047
:100AD000583134302039302020005377617368203A
:100AE000547970651F436F6C6C6563746976651F1C
:100AF00053776173682052696E671F454C452044E7
:100B00006972656374696F6E1F41494C2044697254
:100B1000656374696F6E1F434F4C2044697265634F
:100B200074696F6E005245544131323300540406EB
:100B3000457870202020457846696E6546696E6567
:100B400020204D656469756D436F61727365005453
:100B500072696D20496E631F5472696D2053771F4F
:100B600048692E52657320536C6F772F44656C6112
:100B7000791F547261696E65721F4265657020430A
:100B80006E74005A01062020456E642043656E7421
:100B9000726500452E204C696D6974731F5468722C
:100BA0002E2044656661756C741F5468726F74748E
:100BB0006C6520726576657273651F5468726F7418
:100BC000746C65204F70656E1F542D5472696D1FD3
:100BD000542D4578706F2D4472006607032D2D2D1E
:100BE0005031205032205033204756344756354735
:100BF00056364756370044656661756C74205377E6
:100C00001F437573746F6D53746B4E616D65731F05
:100C10004175746F204C696D6974731F566F6C75E4
:100C20006D6520436F6E74726F6C00566F696365FB
:100C300020496E646578114D454E550083133C156F
:100C4000471534152E15271578131C151115721319
:100C5000BB16CC130815564100566F696365004DED
:100C6000454E55204C4F4E470044656C65746500F9
:100C7000566F6963652046696C65005402062D2D28
:100C80002D2D2D2D4E756D62657220417564696F35
:100C900000660104506C61794D757465005402065C
:100CA0004E6F202020204265666F72654166746534
:100CB0007220004E03072D2D2D2D2D2D2D486170F6
:100CC0007469633148617074696332486170746932
:100CD0006333000776603D76616C20763D76616C0B
:100CE00020200007280D2900506C617920536F7572
:100CF0007263651F4F6E206E6F2054656C656D6565
:100D00007472791F46696C655479706500536F750C
:100D10007263651F46756E6374696F6E1F56616CF2
:100D200075651F5377697463681F526174651F4846
:100D3000617074696300566F69636520416C61720C
:100D40006D00034D4F564520535449434B532F508C
:100D50004F54530005534554204D4944504F494E7C
:100D60005400035B4D454E555D20544F2053544174
:100D70005254006607044E4F4E454558543145586D
:100D80005432504330205047322050423720504791
:100D900035204C2D575200454C45207377697463BC
:100DA000681F41494C207377697463681F50423152
:100DB000207377697463681F5042322073776974B7
:100DC00063681F50473220496E7075741F50423758
:100DD00020496E7075741F4C2D575220496E7075E6
:100DE000740042616E644761700043616C004D7530
:100DF0006C7469706C696572001802036F66662016
:100E00002B3D203A3D00036D6F64650A2520737207
:100E100063202073770007536C61766500124247A8
:100E200000414E41000F504232000F5042310054F9
:100E300072696D2D202B00204C6566741F52696706
:100E400068741F0355701F20446F776E1F2045780C
:100E500069741F204D656E75004449414700537405
:100E600069636B5363726F6C6C00506F7453637281
:100E70006F6C6C0053706C617368204E616D65001F
:100E800053706C6173682073637265656E00416CAA
:100E900061726D205761726E696E67004D656D6F8E
:100EA0007279205761726E696E67005468726F7450
:100EB000746C65205761726E696E6700426174746C
:100EC000657279207761726E696E671F496E616322
:100ED00074697669747920616C61726D136D004379
:100EE000726F73735472696D1F5468726F74746C8F
:100EF0006520726576657273651F456E61626C650B
:100F00002050504D53494D1F4368616E6E656C20F3
:100F10004F726465721F4D6F646500204861707484
:100F2000696320537472656E6774680042040A42F4
:100F3000656570657220202020506953706B7220A7
:100F40002020204265657072566F69636550695351
:100F5000706B566F6963654D656761536F756E643D
:100F600020005406065175696574204E6F4B6579F3
:100F7000207853686F727453686F7274204E6F726A
:100F80006D20204C6F6E672020784C6F6E672000BC
:100F9000566F6C756D651F4265657065721F536F86
:100FA000756E64204D6F64651F20537065616B65BD
:100FB00072205069746368004C69676874207377A5
:100FC000697463681F4261636B6C69676874206948
:100FD0006E766572741F4C69676874206F66662050
:100FE00061667465721F4C69676874206F6E205368
:100FF000746B204D761F466C617368206F6E2062A3
:1010000065657000436F6E747261737400E4139BC6
:1010100013BC13CC13B313A713DC13D4139113898C
:1010200013C31322047C5E54546D0003457870454D
:101030007846466E654D65644372730011544F5493
:101040001F01544D45115453571F0153544B115315
:10105000542500035B4D454E555D20746F2072652D
:10106000667265736800746D72314C6174206D61D5
:10107000781275731F746D72314C6174206D696ED6
:101080001275731F746D7231204A6974746572121F
:1010900075731F746D61696E126D73005354415402
:1010A000000966726565004D4F44454C53454C0040
:1010B00020464D300A52455441004241434B555061
:1010C00020444F4E45004241434B5550005245533A
:1010D000544F52454400534156494E4700524553E0
:1010E000544F52494E47004C4F4144494E470052DD
:1010F0006573746F7265004261636B7570002046A2
:101100004D005377697463681F5472696D731F468D
:1011100061646520496E1F46616465204F757400E7
:10112000464C204D4F44450052414E4745204348D0
:1011300045434B20525353493A000642494E4449D5
:101140004E47004475706C69636174696E67206D09
:101150006F64656C0044454C455445204D4F4445F3
:101160004C004455504C4943415445204D4F444553
:101170004C00012B2A52004D495845520020202096
:1011800020202020202020202020200044454C45E5
:101190005445204D49583F00436C65617220414CD5
:1011A0004C206D697865733F00035945530B4E4FD2
:1011B0001F035B4D454E555D0B5B455849545D0023
:1011C0004D6178206D69786572732072656163681E
:1011D0003A2033321F1F5072657373205B455849A4
:1011E000545D20746F2061626F7274006601034F5A
:1011F00046464F4E20004E020841646420202020C5
:10120000204D756C7469706C795265706C616365A2
:1012100020004375727665000844696666001145D2
:1012200078706F0001557365204F75747075742068
:1012300020200001536F757263651F015765696750
:1012400068741F014F66667365741F0146697820D4
:101250004F66667365741F01456E61626C65457803
:10126000706F44521F015472696D1F1F1F01537725
:10127000697463681F014D4F4445531F01576172E4
:101280006E696E671F014D756C7470781F0144653F
:101290006C617920446F776E1F0144656C61792021
:1012A00055701F01536C6F772020446F776E1F01BC
:1012B000536C6F77202055700045444954204D49A8
:1012C0005820004F50005343092B0D2A122F0004C1
:1012D0004C314C324C334C344C354C364C374C380A
:1012E0004C394C414C424C430048010546697273ED
:1012F000744C6173742000536F757263651F1F4FC8
:1013000066667365741F4D756C7469706C6965727F
:101310001F44697669736F721F556E69741F536934
:10132000676E1F446563696D616C731F4F666673FA
:101330006574204174005B2D3E5D004356005052A1
:1013400045534554004355525645006A01032D2D1F
:101350002D494E560053575220003C02034431366B
:101360004438204C52503C0203416D654A6170453F
:101370007572566F696365004C2E537769746368A4
:101380006573004D697865720044696167416E61FB
:101390000044696167537774636800417564696FDD
:1013A0004861707469630043616C69627261746959
:1013B0006F6E00436F6E74726F6C7300416C61727C
:1013C0006D730048617264776172650047656E6590
:1013D00072616C0056657273696F6E005472616958
:1013E0006E657200446973706C6179005B4D454EA7
:1013F000555D205748454E20444F4E4500454449D1
:10140000540053454C4543540053454C2F454449E3
:101410005400434F5059004D4F56450044454C45EC
:101420005445004241434B555000524553544F528E
:1014300045004544495400494E5345525400434FDA
:101440005059004D4F56450044454C4554450043C6
:101450004C45415220414C4C00047349447873542C
:1014600048527352554473454C457341494C734738
:1014700045417354524E0012081200081C08080817
:101480001C0800000822004900220800000000009B
:10149000227F2200000008220049002208000008E4
:1014A000220049002208000000227F2200000000E4
:1014B00000082200490022080000081C0808081C37
:1014C0000800534300475600054665657420566F73
:1014D0006C74734465675F434465675F466D41683C
:1014E0002020416D7073204D65747265576174746E
:1014F0007300465643466D416D5718242F2F003315
:10150000383B01524554410050726F746F636F6CE9
:1015100000476C6F62616C5661727300536166655F
:1015200074792053777300437572766573004D6F3D
:10153000646573004578706F2F44720048656C696C
:10154000205365747570004C696D697473004D6F3C
:1015500064656C2053656C656374004D6F64656CE5
:10156000205365747570004C617374204D656E7501
:1015700000526164696F2053657475700053746123
:1015800074697374696373004265657020636F7575
:101590006E74646F776E004D696E75746520626558
:1015A000657000032D2D2D52746D45746D54746D4E
:1015B00041746D52454E527564456C655468724174
:1015C000696C503120503220503320000420204FCD
:1015D0004E204F4646424F544820414C4C4F4E43BC
:1015E0004500072D2D2D2D202020763E76616C2084
:1015F00020763C76616C20207C767C3E76616C7C2B
:10160000767C3C76616C414E44202020204F522055
:1016100020202020584F522020202076313D3D763A
:1016200032207631213D76322076313E76322020CE
:1016300076313C763220204C617463682020462D40
:10164000466C6F702054696D654F666676603D76B6
:10165000616C20004E616D6500065761726E31202D
:101660005761726E322043686565702052696E67FB
:101670002020536369466920526F626F742043686B
:1016800069727020546164612020437269636B74D5
:10169000536972656E20416C6D436C6B526174616D
:1016A00074615469636B20204861707463314861D0
:1016B000707463324861707463330054696D65728D
:1016C00000545245303132414747000354783D536E
:1016D000777200204142434445464748494A4B4CB3
:1016E0004D4E4F505152535455565758595A6162A6
:1016F000636465666768696A6B6C6D6E6F70717242
:10170000737475767778797A303132333435363789
:1017100038395F2D2E00FEFFFDF6F7F8F9FAFBFCD5
:10172000042D2D2D2D54494D3154494D32424154F3
:101730005447767231477672324776723347767203
:101740003447767235477672364776723700032D06
:101750002D2D783E30783C307C787C663E30663C7F
:10176000307C667C63312063322063332063342015
:101770006335206336206337206338206339206364
:10178000313063313163313263313363313463314A
:101790003563313600045031202050322020503340
:1017A000202048414C4646554C4C435943314359FF
:1017B00043324359433350504D3150504D325050C5
:1017C0004D3350504D3450504D3550504D36505093
:1017D0004D3750504D38434831204348322043481C
:1017E000332043483420434835204348362043487B
:1017F0003720434838204348392043483130434854
:10180000313143483132434831334348313443481E
:1018100031354348313653574348475631204756B0
:1018200032204756332047563420475635204756F6
:10183000362047563720544849530053776974631C
:1018400068205761726E696E670067656E777269AE
:101850007465206572726F7200454550524F4D207D
:10186000466F726D617474696E67004261642045F1
:101870004570726F6D204461746100434845434B6D
:10188000204D4F44454C2054494D45525300434848
:1018900045434B204D49582F445220534F555243F6
:1018A0004553004D4F44454C2020202020004D45FD
:1018B000202020202020202000454550524F4D2040
:1018C0006F766572666C6F7700E2AEA1A6A4A2C0C7
:1018D0002F25AF0000000000000000000000000005
:1018E000000000000000000000000B07000000C026
:1018F000C0C0C0C0C0C00000000000000000000068
:101900000000000000000006060000000080E078F3
:101910001E06181E0701000000F8FC8EC66EFCF8BB
:10192000070F1D181C0F07080CFEFE0000001818FA
:101930001F1F1818000C0E86C6EE7C381E1F1B19C0
:1019400018181806C6C6C6EEFC38181818181D0F49
:1019500007C0E0B0988CFEFE01010101011F1F7E4F
:101960007E6666E6C686060C18181C0F07F8FCE6AD
:1019700066E6CC88070F1C181C0F07060606C6E68D
:101980007E1E001C1F0300000038FCEEC6EEFC3873
:10199000070F1D181D0F0778FCCE86CEFCF8040C2F
:1019A0001D191D0F0700000030300000000000036B
:1019B000030000E0F89C869CF8E01F1F0101011F56
:1019C0001FFEFEC6C6EEFC381F1F18181D0F07F8B5
:1019D000FC0E060E0C08070F1C181C0C04FEFE065D
:1019E0000E1CF8F01F1F181C0E0703FEFEC6C6C60D
:1019F00006061F1F1818181818FEFEC6C6C60606CB
:101A00001F1F0000000000F8FC0E06CECCC8070F18
:101A10001C18181F0FFEFEC0C0C0FEFE1F1F0000D6
:101A2000001F1F0606FEFE06060018181F1F1818C6
:101A30000000060606FEFE060E1E18181F0F00FE0A
:101A4000FEF0381C0E061F1F03070E1C18FEFE00BA
:101A5000000000001F1F1818181818FEFC18701836
:101A6000FCFE1F1F0000001F1FFEFC70C080FEFE5A
:101A70001F1F0000030F1FF8FC0E060EFCF8070FD7
:101A80001C181C0F07FEFEC6C6EE7C381F1F000088
:101A9000000000F8FC0E060EFCF8070F1C1B1E0FC2
:101AA0001BFEFE86C6EE7C381F1F03070E1C18386F
:101AB0007CEEC6C68E0C0C1C18181D0F070606FE01
:101AC000FE06060000001F1F000000FEFE000000D2
:101AD000FEFE070F1C181C0F07FEFE000000FEFE96
:101AE00001070E180E0701FEFE008000FEFE1F0F0C
:101AF0000603060F1F1E3EF0E0F03E1E1E1F0301F0
:101B0000031F1E7EFEC0C0FE7E0000001F1F0000DF
:101B1000000686C6E6F67E3E1F1F1B191818180021
:101B2000000000000000181818181818180060604D
:101B30006060E0C0060F1F1B1B1F1FFEFEE060E081
:101B4000C0801F1F1C181C0F07C0E0E06060E0C0D1
:101B50000F1F1C18181C0C80C0E060E0FEFE070F71
:101B60001C181C1F1FC0E0606060E0C00F1F1B1B23
:101B70001B1B01C0F8FCCEC60E0C001F1F0000008E
:101B800000C0E0703070E0C003C7CECCEE7F3FFEF7
:101B9000FEC0E0E0C0801F1F0100001F1F000060AA
:101BA000E6E600000000181F1F180000000000E318
:101BB000E300307060607F3F00FEFEC0E0703818C8
:101BC0001F1F03070E1C18000006FEFE0000000089
:101BD000181F1F1800E0E060C060E0C01F1F000178
:101BE000001F1FE0E0C0E0E0C0801F1F0100001FD9
:101BF0001F80C0E060E0C080070F1C181C0F07E0CA
:101C0000F0703070F0E0FFFF0E0C0E0F07E0F07088
:101C10003070F0E0070F0E0C0EFFFFE0E0C06060D8
:101C2000E0E01F1F0000000000C0E0606060606036
:101C3000191B1B1B1B1F0E6060FEFE606000000076
:101C40000F1F181C0CE0E0000000E0E0070F1C1C58
:101C50000E1F1FE0E0000000E0E001070E180E0775
:101C600001E0E0000000E0E00F1F180E181F0F60F9
:101C7000E0800080E060181C0703071C18E0E0000B
:101C80000000E0E007CFCECCEC7F3F60606060609A
:101C9000E0E01C1E1E1B1B191900000000000000C4
:101CA000006F000007000700147F147F14242A7FB0
:101CB0002A12231308646236495522500005030096
:101CC00000001C2241000041221C0014083E0814A0
:101CD00008083E08080050300000080808080800FE
:101CE000606000002010080402003E49453E0000EC
:101CF000427F40006251494600414949360018146C
:101D0000127F0027454539003E49493200017905D7
:101D1000030036494936000649291E0000363600C0
:101D20000000563600000814224114141414144103
:101D300022140800020151090600060909067E095D
:101D400009097E7F494949363E414141227F41414F
:101D5000221C7F494949417F090909013E414949FE
:101D60007A7F0808087F00417F41002040413F0101
:101D70007F081422417F404040407F020C027F7F59
:101D80000408107F3E4141413E7F090909063E415A
:101D900051215E7F09192946264949493201017FAF
:101DA00001013F4040403F1F2040201F3F40304046
:101DB0003F631408146307087008076151494543DD
:101DC000007F41410002040810200041417F0004CF
:101DD000020102044040404040080408100820541A
:101DE0005454787F48444438384444442038444468
:101DF000487F3854545418087E0901020C5252523C
:101E00003E7F0804047800447D40002040443D00AB
:101E10007F1028440000417F40007C041804787C37
:101E20000804047838444444387C14141408081412
:101E300014187C7C080404084854545420043F447B
:101E400040203C4040207C1C2040201C3C40204046
:101E50003C44281028440C5050503C4464544C449A
:101E6000000836410000007F0000004136080008ED
:101E700008221C08081C22080804027F0204102003
:101E80007F201001020408102040804080080420B8
:101E90001002010000891112239B322446AD5736EF
:101EA00065BF74488CC19D5AAFD3BE6CCAE5DB7E5A
:101EB000E9F7F88110080193331A22A5562C47B789
:101EC000753E64C99C408DDBBF52AEEDDA64CBFF3A
:101ED000F976E802218B30100299132667AF763429
:101EE00044BD554AADC3BC588ED19F6EEBE7FA7C1A
:101EF000C8F5D983310A2091121803A7772E66B549
:101F0000543C45CBBD42ACD99E508FEFFB66EAFDF9
:101F1000D874C904428D5316619F702004A91532EC
:101F200027BB364CCEC5DF5EEDD7FC6888E1997AD9
:101F3000ABF3BA85520C4397711E60A1142805B308
:101F4000373A26CDDE44CFDFFD56ECE9986089FBB9
:101F5000BB72AA06638F7214409D512225AB3430A8
:101F600006B9174EEFC7FE5CCCD5DD6AA9E3B87899
:101F70008AF19B87730E6295501C41A3352A24B1C8
:101F8000163807CFFF46EEDDDC54CDEBB962A8F979
:101F90009A708B088481951AA793B62CC2A5D33E5C
:101FA000E1B7F04008C919522BDB3A644EED5F7679
:101FB0006DFF7C899400859BB712A6ADD224C3BF68
:101FC000F136E0C1184809D33B5A2AE55E6C4FF759
:101FD0007D7E6C0AA583B4188691972EE3A7F23C08
:101FE000C0B5D14229CB38500AD91B666FEF7E7439
:101FF0004CFD5D8BB502A499961087AFF326E2BD28
:10200000D034C1C3394A28D11A580BE77F6E6EF518
:102010005C7C4D0CC685D71EE597F42880A1913ACB
:10202000A3B3B2444ACD5B5669DF78600CE91D72F8
:102030002FFB3E8DD604C79FF516E4A9902081BBE7
:10204000B332A2C55A4C4BD7795E68E11C680DF3D8
:102050003F7A2E0EE787F61CC495D52AA1A3B03887
:1020600082B193466BCF7A5448DD59622DEB3C70B8
:102070000EF91F8FF706E69DD414C5ABB122A0B9A7
:10208000923083C77B4E6AD5585C49E33D6A2CF198
:102090001E780F00F67311241FBECFEFD0E1DEBF14
:1020A000CDBF11E0A0E0B1E0E4EDF9EE02C0059093
:1020B0000D92A231B107D9F71EE0A2E1B1E001C053
:1020C0001D92A536B107E1F710E2C6E9D0E204C0DF
:1020D0002297FE010E94B374C439D107C9F70E9448
:1020E000A6720C94E8740C940000E091510694E000
:1020F000E99FF0011124E80FF11DEE53FD4F84918B
:102100008F5F0895F8948091590D90915A0D7894AD
:102110000895E82FF0E0E555FD4F849108952AE0F9
:10212000829FC00111248B599D4F089590915306B1
:1021300091708091BC0586FB882780F989270895D6
:102140000F93022F24FF03C00F7E9DE201C094E293
:10215000411104C024E04FE952E00EC04530A0F424
:102160009091BC0594FF0BC0006194E0499FA001D1
:1021700011244559594F24E00E949D630DC02FEF53
:10218000240F42ED52E006C0941730F02BEF240FDD
:1021900045E957E10E94C1630F910895442311F06E
:1021A0004C5E01C040E0CCCFCF93DF93E5E8F1E097
:1021B00080917F06108291E0918381FF09C092E2B5
:1021C000928393E29383EF01259694E2948304C073
:1021D000EF01239692E0928382FF09C09FE19883EA
:1021E00090E29983FE01339691E29A8304C0FE0146
:1021F000319693E0988394E0908395E0918396E004
:10220000928384FF09C095E2938396E29483EF0161
:10221000269697E2958304C0EF01249697E0938376
:1022200085FF09C098E2988399E29983DE011396AD
:102230009AE29A8304C0DE01119698E0988399E0AF
:102240009C93FD0186FD02C0319604C032969BE24C
:10225000ED01998387FF03C08CE280833196DF0113
:102260008AE08D938F5F8631E1F78487CF018957AC
:1022700091408093570127E1258740E099270196F7
:10228000242F30E08217930754F0F901EB57FE4FEB
:10229000E081F0E0E85AFE4F40834F5FF1CF90912C
:1022A000830690FF0AC0809164008B7F8093640056
:1022B0008091650084608093650091FF02C0BF98A3
:1022C000C79ADF91CF91089587FF03C0819591E070
:1022D00001C090E0E82FFF27E7FDF095E85AFE4F98
:1022E000808191118195089587FF03C0819591E0C8
:1022F00001C090E0E82FFF27E7FDF095EB57FE4F78
:1023000080819111819508950F931F93CF93DF934F
:10231000D62FC42F022F16E0180F442339F0463170
:1023200041F04A3E81F448EE52E005C04BE952E0EC
:1023300002C044EE52E06D2F812FDF91CF911F91AB
:102340000F910C94D36347FF04C041E20E941063D5
:10235000C1952FEF2C0F273114F026EF2C0F4CEEE8
:1023600052E06D2F812F0E94C163DF91CF911F91A9
:102370000F9108950F931F93CF93DF93D82F162FAC
:10238000C42F022F4D3234F04DE682E18D0F0E94B2
:102390001063CC52202F4C2F612F8AEF8D0FDF91CD
:1023A000CF911F910F91B0CFDF92EF92FF920F93D9
:1023B0001F93CF93DF93D82F162FF42E27FF03C040
:1023C000E5E0F2E002C0E0E0F2E0C281D3802370F9
:1023D000E22E81E0821718F1C4306CF483E0C80269
:1023E000A001112442575D4F0F2D23E0612F8D2F47
:1023F0000E949D6318C0CD5F0F2D2C2F4EE457E136
:10240000612F8D2F0E94C163C0310CF4D6502F2D47
:1024100045E2612F82E18D0F0E94106304C082E0CB
:1024200028130AC004C0E11007C0C13029F42F2DC1
:102430004D2D612F8D2F9EDFDF91CF911F910F9139
:10244000FF90EF90DF900895873038F4E82FF0E0A8
:10245000EE0FFF1FEC5DF74F24C08C3050F184313C
:10246000C0F4482F50E0DA01AA0FBB1FA45FBE4F93
:102470002D913C91803148F4FA01EE0FFF1FE95D88
:10248000F94F80819181281B390BC901880F991F51
:102490000895843248F4E82FF0E0EE0FFF1FE45275
:1024A000F84F8081918108958E3218F484520C94F3
:1024B000F72280E090E008950E94A272882311F034
:1024C000A895FACF1092890D08951F93CF93DF93AB
:1024D000EC01162F0E94C462BE0188E10E94F863DD
:1024E00012FF04C067E182E10E940F7210FD11C06B
:1024F00011FF06C068E772E080E30E94F86306C03F
:102500004AE652E068E38CE10E940E644BEB52E035
:1025100002C042E652E024E060E086E1DF91CF9124
:102520001F910C94D36361E0D0DF0C9412670F937A
:10253000262F00E04CEE52E060E10E94C1630F9153
:1025400008951F93CF93DF93C6E110E08C2F0E9474
:10255000F867110F182BC150CE30C1F780917F065C
:1025600082FF12C08FE10E94A26824E0829FE001F6
:102570001124137CC12B84E00E94A26820E1829F79
:10258000C00111241C2F182B812FDF91CF911F9197
:10259000089570E0882399F090E0019725E0289F46
:1025A000F001299FF00D1124E60FF71FEE0FFF1F1A
:1025B000E05FFA4F808191818B509E4F0895FB011F
:1025C000E35DFB4F8081992787FD909508951F93C8
:1025D000CF93DF93D82F162FC4E0DD2391F0612F26
:1025E0008D2FD7DF9C01253F81E0380764F08BE019
:1025F000820F8D1710F08CE0820FC15029F0D82F78
:10260000ECCFC0E001C0CD2F8C2FDF91CF911F9177
:102610000895CF93C62FDBDF6C2FCF91BACF8E37C3
:1026200091053CF483382FEF920734F483E89FEF51
:1026300003C08DE790E008950895FF920F931F93D4
:10264000CF93DF938A01C62FD0E08823D9F0BFDF74
:10265000F82E8823B9F0C801E2DF2F2D30E0215099
:10266000310945E0429FF001439FF00D1124EC0F2A
:10267000FD1FEE0FFF1FE05FFA4F855F91409183D2
:10268000808305C0C801CBDFC35DDB4F888386E054
:10269000DF91CF911F910F91FF900C94315DAF921C
:1026A000BF92CF92DF92EF92FF920F931F93CF933F
:1026B000DF938C017B016A01A22EB0900B029B2D4F
:1026C0009F7D943439F080910208882309F498C0E2
:1026D000933479F4B19906C080913E01E801C80FA6
:1026E000D11D02C0E801219683E10E94057285E0B8
:1026F00010C0953419F0923409F088C0B19983C0A4
:1027000080913E01E801C81BD10984E10E94057255
:1027100084E00E94F867811168C0E114F104F9F4C3
:1027200081E0C816D104D9F480E6B81619F08EE21B
:10273000B81211C010920208C1E00115110509F08C
:10274000C0E0D0E08B2D0E94C3688EE2B81206C0B4
:102750001092380803C0C170DD2701C0B12C409130
:10276000410150914201C41BD50B80913808813042
:1027700071F440911402B19905C084E14802A001AE
:10278000112403C0552747FD5095C40FD51FCC1603
:10279000DD0644F48B2D0E94C36883E10E9405721C
:1027A000E6010AC0CE15DF053CF48B2D0E94C368FC
:1027B00084E10E940572E701C017D10749F1B19980
:1027C00003C08FEF80939A06209751F48B2D0E94BF
:1027D000B36817FF02C083E101C084E10E94057263
:1027E0008A2D83700E94315D13C0CC27DD27C01B6A
:1027F000D10B85E00E94C36884E00E94C3688DCF3E
:10280000953421F47BCFE80121977FCFE80185CF74
:10281000CE01DF91CF911F910F91FF90EF90DF904C
:10282000CF90BF90AF900895552747FD50957727DB
:1028300067FD7095992787FD909531CF2091FB0713
:10284000F3CF462F2091FB0760E0EECF462F50E0FC
:102850002091FB0760E070E022CF90914A01911136
:1028600003C0811106C00895811103C08FEF890F45
:1028700001C080E080934A018EEB80934901089566
:10288000E0914A01F0E0EE0FFF1FE55BFE4F918300
:1028900080838FEB809349010895809155062AEF3C
:1028A000829FC0011124880F991F20913A01309115
:1028B0003B012817390720F490933B0180933A019C
:1028C0000895EEE2FEE037A1303180F420A541E02A
:1028D000420F40A7DF01A20FB11DA20FB11D8D93C2
:1028E0009C93403108F010A63F5F37A3089590E015
:1028F0008C5F9E4FE6CF90E0E4CF8093160290E08D
:102900004097DFCF0F931F93CF93DF93EC0180911C
:102910005C0681FF07C180916D0686FF89C012E0C9
:1029200001E00E94A2698F3F2FEF920781F029A951
:10293000211104C08F31A9F709ABF3CF213011F475
:1029400019ABEFCF223069F78AAB19AAEACF8EA173
:10295000813041F53FA1332309F452C029A5FE017E
:10296000E20FF11DE20FF11D808191812F5F203177
:1029700008F020E029A731503FA32091C60121FD96
:10298000E0C097FD02C021E101C028E22BA32FE1A6
:102990002AA722E02BA78CA79DA718AA84E08FA7BF
:1029A0002EA32EC0811106C08091580D8D3340F1A9
:1029B00086E025C0823021F19AA99078833049F4CD
:1029C000992329F08BA181508BA3811119C084E038
:1029D00016C0843021F4992399F083E00EC085302D
:1029E00039F48BA181508BA381110AC081E007C00B
:1029F000863031F4992321F084E18BA385E08EA306
:102A00008EA1823009F49DC08BA98F5F8BAB8A3079
:102A100008F497C01BAA8DE18AA781E08BA798A133
:102A2000911101C080E08CA718AA83E08FA789C00C
:102A300098A189A1992311F0846001C08B7F89A39B
:102A40008EA1813081F5C79A2FA1222349F189A552
:102A500031E0380F39A7FE01E80FF11DE80FF11D35
:102A6000808191819DA38CA3303108F019A621505B
:102A70002FA32091C60121FD64C097FD02C021E172
:102A800001C028E22BA329A12C7F97FD226029A356
:102A900089A18BBBC7988FE18AA382E08EA351C026
:102AA00089A18BBB4DC081110CC0C79A89A18360DD
:102AB00089A38BBB8091580D8D3308F441C086E00B
:102AC0002FC0823009F43DC089A18BBBC79ABF9843
:102AD00000C0000000C086B38078BF9A9EA19330EA
:102AE00049F4882329F08BA181508BA3811128C040
:102AF00084E016C0943021F4882311F183E00EC0E5
:102B0000953039F48BA181508BA3811119C081E0DC
:102B100007C09630A9F4882399F084E18BA385E05F
:102B20008EA30EC08091830681FD0BC08091590653
:102B300086FB882780F998A1981711F0C79A01C0E1
:102B4000C798DF91CF911F910F91089590915106F1
:102B500090FD02C093E08927E82FF0E0EE5CF74F8C
:102B6000E081E7FDE95FE595E595E5951E1624F022
:102B7000EE2321F0E19502C080E801C080E0E8305A
:102B800008F0E7E0F0E0EC55FD4FE491EE2319F09A
:102B900099E0909355018E2B0895853030F46FEFB6
:102BA000680F8091EA0635DD24C08D3080F4E82F6F
:102BB000F0E0EE0FFF1FE85EF74F8081918197FDF7
:102BC000079653E0959587955A95E1F712C08D3198
:102BD00070F4E82FF0E0EE0FFF1FE651F84F808110
:102BE00091816AE070E00E946074CB0102C080E0D5
:102BF00090E015CD482F833021F0882321F0E82F75
:102C000003C0E0E001C0E3E0F0E0EE0FFF1FED5E87
:102C1000FE4F80819181443080F420916E0630E037
:102C200002C0359527954A95E2F720FF06C020E0BF
:102C300038E0A901481B590BCA0108951F93CF938F
:102C4000DF9310E0C0E0D0E0812FD4DFC80FD91FA0
:102C50001F5F1430C9F7C058DF4F8D2F90E0DF9110
:102C6000CF911F910895CF93809151068170C2E05A
:102C7000C81B8C2FBFDF6C2F0E94E73C2091BC0546
:102C800025FF05C00F964F9728F080E004C08131E2
:102C90009C4FDCF781E0CF910895E3E1F1E040E063
:102CA000842F806487B9369A3699FECF24B135B126
:102CB000369A3699FECF84B195B1820F931F8193D6
:102CC00091934F5F483061F7089578941F920F9267
:102CD0000FB60F9211248F93809112018F5F809312
:102CE00012018F910F900FBE0F901F90189578943E
:102CF0001F920F920FB60F9211242F938F939F93D1
:102D0000CF93DF93EF93FF93F89487B78F7B87BFC1
:102D100078942091CA018091CC0190915C0688231F
:102D200059F090FF07C08091640E820F8093640E6B
:102D300087FF02C01B9A01C01B9891FF50C0809171
:102D40006D0686FF22C0EEE2FEE087A5882309F427
:102D500046C080910A02811142C080919B0085FF8C
:102D60000DC080A991E0980F90ABEF01C80FD11D65
:102D70008AA580939C0087A5815087A787A581118C
:102D80002EC086A1823059F526C08091420981115A
:102D900026C0EEE2FEE086A1823009F583A18823F9
:102DA00011F081501BC021A1C79A82A180FD09C0EA
:102DB0002D7F84A195A196FD2260880F991F95A370
:102DC00084A381E082278BBB81A3C79882A1815015
:102DD00082A3811104C083E086A385E083A3F894D5
:102DE00087B7806487BF7894FF91EF91DF91CF918F
:102DF0009F918F912F910F900FBE0F901F9018955C
:102E000078941F920F920FB60F9211242F933F9335
:102E10004F935F936F937F938F939F93AF93BF93E2
:102E2000EF93FF9381B7845681BF88EC91E00E94B5
:102E30004E700E94D2688091910D82608093910DB6
:102E4000E2E0F1E08081815011F0808304C084E6EB
:102E5000808381E081838281815011F0828305C06B
:102E60008AE08283838181608383FF91EF91BF91A8
:102E7000AF919F918F917F916F915F914F913F9112
:102E80002F910F900FBE0F901F90189578941F925E
:102E90000F920FB60F9211242F933F934F935F938E
:102EA0006F937F938F939F93AF93BF93EF93FF9312
:102EB0002091800030918100F89480917D008F7D79
:102EC00080937D0078948091970690919806A9014F
:102ED000481B590BCA019695879530939806209305
:102EE0009706409123019C01215A3F402F3D3E42CD
:102EF00030F12FEF240F283028F59C012152334068
:102F000027373540F0F424E620931502E42FF0E053
:102F1000EE0FFF1FEE5DFE4F9C012C5D3540509182
:102F20005706565F529FC001539F900D11246AE0CF
:102F300070E00E946074718360834F5F03C041E062
:102F400001C040E040932301F89480917D008062AD
:102F500080937D007894FF91EF91BF91AF919F9105
:102F60008F917F916F915F914F913F912F910F9032
:102F70000FBE0F901F90189592EC980F81E097303C
:102F800008F080E00895FC018081882359F08432A4
:102F900018F085520C942623815056DA40E060E008
:102FA0000C94177208959C0155E0359527955A9514
:102FB000E1F7280F391FAC01440F452F441F550B73
:102FC000241B350B892F990F990B8595820F931F21
:102FD00008959DE7980F9B3F88F08E57E82FF0E00B
:102FE000EE0FFF1FEE5FFA4F808186171CF460839F
:102FF000862F0895481714F44083842F089544E6DB
:103000006CE9E7CF982F80915C0284FF03C081E0D8
:10301000923009F080E0089549E284029001112481
:10302000359527953595279587FD815C86FB880F1B
:10303000880B80F9A901481B510987FD5395CA01E6
:1030400008954F925F926F927F928F929F92AF926C
:10305000BF92CF92DF92EF92FF920F931F93CF9385
:10306000DF93782E642E882309F4D6C086E1781683
:1030700021F09AEE791203C0D1C081E0D5C0872D2E
:10308000992787FD909597FF03C0919581959109A8
:10309000873191056CF00E943868982F81E01714F1
:1030A0001CF49111C1C0BAC0992309F4BDC0B6C0C7
:1030B000872D87FD81958A3040F4825F0E94F867F2
:1030C00017140CF4B1C091E0A5C08A50E82EF12C81
:1030D0006701CC0CDD1CE601CE0DDF1DCF55DB4FAB
:1030E0008A818F7009F49AC094E0961530F4F70144
:1030F000EC57F94F908191708AC05880498009D867
:10310000811107C08FEF850D9FD98C01898184DFE4
:103110000EC0823041F48FEF850D96D98C018981E4
:10312000815092D904C080E090E000E010E02A8154
:103130002F70822E912CF4013197EE30F10508F0BA
:1031400071C0EA5BFF4F0C94B17417FF35C0119545
:103150000195110931C017FF33C01195019511096F
:103160002FC001E0060D402F60E0852D6ADF182F8B
:10317000402F60E0842D65DF2A812F70253061F4B7
:10318000112309F44FC0882309F44CC08A81829529
:103190008F7059F591E031C0263019F41111F6CF36
:1031A000F2CF982F91271EC008171907D9F5EECF37
:1031B0000817190759F736C0801791073CF332C03A
:1031C000081719071CF32EC0F601E255FE4F918136
:1031D0009095991F9927991F05C0F701EC57F94F52
:1031E000908191709111D2CF08C089300CF08F5F1F
:1031F00041E0460D60E025DF982F2A812F7030E0F6
:103200002C30310524F4F701EC57F94F9083171453
:103210003CF081E0892708C0862F06C080E004C00A
:10322000892F02C090E0E9CFDF91CF911F910F91DC
:10323000FF90EF90DF90CF90BF90AF909F908F90D6
:103240007F906F905F904F90089540E060E0F9CEDE
:1032500080913E06FADF811113C080913A0190916E
:103260003B01892B69F410924E0E8091580D90917C
:103270009906981749F0809399068EE29EE042CB1A
:1032800081E080934E0EF1CF0895CF93DF93C62F48
:1032900020914802222339F090934A0280934902F8
:1032A000DF91CF91089564E010D90E941267C11197
:1032B00003C080913B0601C089E10E94E066FCD812
:1032C000D1E00E94A272882319F0DF91CF91F4C857
:1032D0008091910D833019F4A8951092910DCC2313
:1032E00019F0D0934E0E02C010924E0EB1DFE9CF0E
:1032F00060E0CBCFE0914A01E43018F08FE092E03B
:10330000F7CF2FEB20934901EF5FE0934A01F0E004
:10331000EE0FFF1FE55BFE4F918380830895809140
:10332000500680FD16C0B9DC9EDC811112C066E03B
:1033300081E492E0CAD80E941267BED8AEDC88DF72
:10334000A89591DC811105C00E94A2728823B1F377
:10335000B3C80895DF92EF92FF920F931F93CF931C
:10336000DF938091500681FD8FC0C091FA04F090E8
:103370000C0680917F0682FD0CC08C2F88738830EC
:1033800041F0803131F0803221F0C77CC860C093B9
:10339000FA04E12CDD24D394D4D8182F85E20E94BE
:1033A000A268082FD12FDC276E2D62608CE192E09D
:1033B0008CD8D0FF03C060E082E0B9D8D1FF03C051
:1033C00061E087E1B4D880917F0682FF1AC08D2F1B
:1033D0008C7051F0612F70E07595679575956795C4
:1033E00063706B5E8CE2A3D88D2F8073F9F0612F30
:1033F00070E044E0759567954A95E1F763706D5FFD
:1034000013C0D2FF03C062E08CE291D88D2F887385
:1034100069F013FF02C063E007C014FF02C064E05C
:1034200003C015FF03C065E081E481D880917F0669
:1034300084FF0AC0802F8F25837061F0602F637036
:10344000655E86E574D806C0D6FF03C066E086E5F3
:103450006ED80F2DD7FF03C067E08BE668D80E94B7
:103460001267DD2021F028D834E0E32E01C0E12CE2
:103470001C1302C00F1541F00E94A272811104C0FA
:10348000E7DEA895D12C88CFDF91CF911F910F91C6
:10349000FF90EF90DF9008958111FFD980913A015C
:1034A00090913B01009709F0019720913901222367
:1034B00061F020915D064AEF249F90011124220FB4
:1034C000331F8217930708F4C90190933B0180933F
:1034D0003A01BECE1F93CF93DF93C8E1D5E090E0D1
:1034E000888111E0190F882329F0AFDE882311F0BD
:1034F000812F05C0912F2A96143091F780E0DF913B
:10350000CF911F9108958F929F92AF92BF92CF92C9
:10351000DF92EF92FF920F931F93CF93DF93EC0113
:10352000A62EB12C6501CC0CDD1CF601E95EFD4F29
:10353000008111818981882309F457C08D809E8084
:10354000888181500E9424127C018981853038F461
:10355000833050F4813079F0823091F039C0853079
:10356000A1F0863071F134C0F7FE03C0F194E1940C
:10357000F108833029F481E08E149F043CF125C0CA
:1035800081E0E814F90414F120C08881F5DC882377
:1035900069F08AE09701829F7001839FF00C1124EB
:1035A000F4018E9F40018F9F900C1124E818F908B8
:1035B000FFE1EF0EF11C81E02FE3E216F10430F0A1
:1035C00004C081E0E814F90409F080E0E82EF12C51
:1035D0008A81811104C0EF2829F081E01BC035DE0B
:1035E0008111F9CF00E010E014C08A81882331F006
:1035F0002CDE81110BC00FEF1FEF0CC08B818330CD
:1036000040F09C81907681E029F403C080E091E055
:1036100002C080E090E0892BF501E95DFD4F5F017C
:10362000F080209105019B8121FD2EC0933059F43B
:103630008A810E94A268F81689F1FF24F394F80E9B
:1036400000E010E02CC0813041F4F11003C0292FBC
:103650002D7FB1F0913089F421C0F1E0FF120CC050
:103660008FEF890F823040F480E000E010E092306C
:10367000B1F4E2E0FE2E13C080E0913219F40CC0E8
:1036800000E010E0F82E0BC0FF24F394913209F013
:10369000F12C0FEF1FEF03C00FEF1FEFF12CF5011F
:1036A00080838C8187FD03C0F1100AC07BC08881B4
:1036B0008530D0F3855283D7882309F473C0F4CFC3
:1036C00017FF04C08B81833028F46CC001151105ED
:1036D00009F055C08C818076803211F4CE0153DC24
:1036E0008C81877059F1813021F52F81822F988547
:1036F0008C3FF1E09F0740F040E050E060E070E078
:1037000084E0820FE2D60DC0853F21E0920748F0A9
:10371000FC01EE0FFF1FE85EFE4F8081992787FDB9
:1037200090952F2D30E021503109820F931FC9D879
:1037300005C060E070E08F810E940A728C81807603
:10374000803411F4CE011FDC8C81282F287181F088
:10375000869586958695837090E0029724F02831AF
:1037600021F48FE003C08DE001C08EE00E9405725D
:103770008B8183508E31A0F00FEF1FEF13C0101616
:10378000110684F40F5F1F4F8B813AE0839FC001C5
:1037900011244397081719072CF000E010E002C02D
:1037A00001E010E0F601E95EFD4F11830083DF9137
:1037B000CF911F910F91FF90EF90DF90CF90BF902E
:1037C000AF909F908F9008951F93CF93DF93C4EC99
:1037D000D5E010E0612FCE0196DE29961F5F1830EC
:1037E000C9F7DF91CF911F9108959F92AF92BF9239
:1037F000CF92DF92EF92FF920F931F93CF93DF93BD
:10380000109237088091120102B79091120189132A
:10381000F9CF10E0182B41DA8EE587B91BBA8FE19A
:103820008ABB00C099B38FEF8ABBECE0F2E08781DE
:10383000882311F080E202C0892F807E8483292FA3
:10384000207C8081281759F08074880F907831810E
:10385000891711F0315001C03F5F3183208382818D
:103860009381891711F0838381838091590D909101
:103870009306282F291B20933C0180939306809167
:103880000A02811106C060E08AED97E00E94AC4711
:1038900001C0A89580913C01882309F4CCC2C4E3FF
:1038A000D1E080910008882319F0815080930008AE
:1038B000C5D92B813C818217930741F09C838B8370
:1038C0001A82198281E0809339012DC060915206DD
:1038D000665F49F180913D01823328F188818F5FD5
:1038E0008883803100F189819A8101969A83898346
:1038F000188247E751E0649F9001659F300D1124C5
:103900002817390780F48F719927019761F4809106
:10391000C6018D7F8093C60186E00E947D146DE212
:1039200080E10E940F720E9466310E948130809176
:103930001502882319F081508093150280E00E94BF
:10394000835D0E94C4620E948C67D82E80910A0217
:103950008111B4C13D2D3F70A32E4AEFA40EC0913A
:103960005D02C43021F0C33019F4C4E001C0C8E0E6
:1039700057E05A1508F495C08D2D807F803209F4E8
:1039800090C08A2D86950E94751090916D0690FDCD
:1039900004C0CC24CA94C80E03C0E4E0CE2EC81ADA
:1039A0006C2D8091EA060E94E712B82E6C2D0E94C1
:1039B00009137C01C1110CC0EC0197FF04C0CC2796
:1039C000DD27C81BD90BD595C795D595C795CF5F72
:1039D00082E0C8120FC080915C0280FD02C0912C71
:1039E00003C099249394C2E00E949610882319F092
:1039F000C19501C0912CDD27C7FDD095A0FE03C065
:103A0000CE0DDF1D04C0F701EC1BFD0BEF0120976D
:103A100021F08D2F8F2587FF11C091100FC0EF2847
:103A200069F040E050E06C2D8B2D0E941D138D2D10
:103A30000E94C36886E10E940572C8C39E01245893
:103A40003F4F293F310548F4AE016C2D8B2D0E946C
:103A50001D136C2FC7FF18C016C01C161D061CF4C2
:103A60004DE750E002C043E85FEF6C2D8B2D0E94C4
:103A70001D13CE0183589F4F8B3F910508F0A6C3BD
:103A80006C2F1C160CF4619567FD6D5F659565954F
:103A9000772767FD7095645C7F4F85E10E940A720D
:103AA00095C38D2D8F7B71F480919A06B1998AC34D
:103AB0008F3F31F08F5F883C19F48FEF6DEBD62E7E
:103AC00080939A06EFE3F1E08091300890913108FD
:103AD00020813181281B390B37FF02C0215E3F4F07
:103AE00055E0359527955A95E1F72115310561F097
:103AF00024813581281B390B37FF02C02F5F3F4FD0
:103B0000359527959183808395838483809153068F
:103B100085FD04C08091FE07882311F020E030E08D
:103B200033832283CCE0D2E02D818981821B8F3FB9
:103B300009F480E087FD8F5F85958887982F990F1E
:103B4000920F9D838D29A8DCF0906906F7E0FF0EA7
:103B5000E0914A01F0E0EE0FFF1FE55BFE4F208190
:103B600031812953354409F040C080915A088111B0
:103B70003CC02885222371F08E81332727FD3095A4
:103B8000F901E80FF11D87FDFA95CF010E940F138F
:103B90008E831886E091C7048E2F807E31F1E295E6
:103BA000E695E770F0E0E430F10554F4EE0FFF1F06
:103BB000E65DF74F208131813C5F60E078E00CC02A
:103BC000EE0FFF1FE650FB4F2081332727FD309576
:103BD00023583F4F6AEF70E047E0429FC001439F88
:103BE000900D11240E944C74F62E80911602F81646
:103BF00019F08F2D0E947D148091590687FF3CC0DB
:103C0000809156018823C1F1809155018823B1F13B
:103C10008091920687FD03C08F5F8093920682E0B9
:103C20000E94A615982F9F7789F0209192069217EF
:103C300028F510929206D11021C0D82ED094DD1C08
:103C4000DD24DD1C83E68D19D82E18C083E00E9488
:103C5000A615982F9F7791F020919206921770F4F5
:103C600010929206D1100AC0D82ED094DD1CDD240B
:103C7000DD1CF4E6DF0E02C01092550181E0809356
:103C80005601E0901202FF24E7FCF094C3E0D5E077
:103C90008881882371F0853031F00E94CD159927F5
:103CA00087FD909501C0C7010E940F13FE01319757
:103CB0008083229625E0C131D20751F780914902D5
:103CC00090914A020097B1F060E00E9465120E9454
:103CD000A27290919106992339F0811128C0109217
:103CE0004A021092490223C0882309F181E080939F
:103CF00091061DC010929106C0914901CC2331F06C
:103D00001092490187E10E940572DC2E84E18093C4
:103D10003E01D0920B02E0914A01F0E0EE0FFF1F4E
:103D2000E55BFE4F0190F081E02D8D2D09950E94FD
:103D30001267C091650088EC91E00E943A70882378
:103D400011F084E105C08091630E882321F0815039
:103D50008093630E06C08091630086958170809386
:103D6000620E8091620E80934702882309F42CC270
:103D70008091590685FD28C2CF7EC0936500809151
:103D8000580D8F71823009F054C0809121019091BB
:103D90002201AC01A4E0440F551FAA95E1F797FD5D
:103DA0000796BC01F3E075956795FA95E1F72091C8
:103DB0003D06332727FD30952A5F3F4F629FC001A4
:103DC000639F900D729F900D1124840F951F209179
:103DD000530626FD05C0609100017091010102C0EB
:103DE00060EF70E00E944C7480913D01680F711D7E
:103DF0006F5F7F4F7595679560933D018091900649
:103E0000805F80939006811114C080913C066817F2
:103E100080F4623370F06EE281E10E940F72809153
:103E2000530683FF06C082E390E090933B018093AA
:103E30003A01109239018EE587B9369A3699FECF4C
:103E400084B195B190930101809300018091910D0F
:103E5000833019F4A8951092910D2091120182B728
:103E6000909112012913F9CF90E0922B801B910BB6
:103E700020910801309109012817390720F4909307
:103E800009018093080180910501882309F419C173
:103E900000919506109196060F5F1F4F109396069E
:103EA000009395068091C7048F7150E1B52EB81A22
:103EB000F7E1FB1508F477C0EB2CF12CE701CC0FF0
:103EC000DD1FC853DB4F3FE03B1528F4E701CC0F63
:103ED000DD1FC45DDA4F8881C82EC294C69427E0E6
:103EE000C222D98045E04C1550F05AEF5D1538F4E8
:103EF000ED2DF0E0EE0FFF1FEE5EFC4FD0808F71D6
:103F000009F44FC0A2D9A82E80910501F701E15D07
:103F1000FD4F7F0181FD43C08C2D857049F4808168
:103F2000811106C0AA2021F08D2D90E00E9461141D
:103F30008FEF8C0D823058F4F7018081813079F554
:103F4000A1102DC0F2E0CF1226C0D39424C025E0EA
:103F50002C1548F4F7018081811121C0AA20F9F0C5
:103F6000898174D31CC0F2E0FC15C8F4AA20B9F012
:103F700024E0C21631F035E0C31631F066E970E096
:103F800005C06CE271E002C068E572E0C8010E9401
:103F90004C74892B21F48D2D90E00E946114F7015F
:103FA000A082B39485CF01EA14E0B4E8AB2EB6E06A
:103FB000BB2ECEEACC2EC1E0DC2EE12CF12CF80198
:103FC0009280892D8F700E9489108330D9F5F60177
:103FD000C081D181209771F4F801C081C7FD06C06E
:103FE000C095FAE0CF02E00111241BC0DD27C7FD18
:103FF000D09517C0D7FF14C0219699F4F701EE555C
:10400000FB4FC081C7FD06C0CF5F2AE0C202E001BE
:10401000112406C0DD27C7FDD095C095D09501C0FD
:104020002197892D807F59F0892D82958F70893055
:104030000CF08F5F0AD9811102C0CFEFDFEFF601DC
:10404000D183C083F501C081F80182818F708C30EB
:1040500071F48081FAD8811109C0F701EE55FB4F48
:104060008081F3D8882319F0C0E001C0C1E0F801D5
:1040700082818F708D3091F48081E7D8882359F048
:10408000C1FD0CC0F701EE55FB4F8081DED88823BF
:1040900021F0C3E003C0CD7F01C0C2E0F501C193B0
:1040A0005F010D5F1F4FF3E0EF0EF11C22E0C20E27
:1040B000D11C34E2E316F10409F081CF85DB1092C4
:1040C000050180910301882309F482C020919406A0
:1040D0002F5E822F8F7090E00C970CF0207F209342
:1040E00094068091C7048F71A0E1FA2EF81ACBE4F0
:1040F000D2E0E12C422F4073D42E522F5F70C52E98
:10410000822F8077B82E207FA22EEF1409F450C0A2
:104110008E0103581D4FF8018081982F907C9034B8
:10412000A9F4D11013C0880F880F859585958DD877
:10413000882361F080915C0680FF05C0FE01E25893
:10414000FD4F808101C081E00E940572F8018081ED
:10415000982F907C903849F5880F880F8595859524
:104160008731B4F08751813039F018F0823039F05E
:104170001CC0B1101AC006C0C11017C003C0F0E2C5
:10418000AF1213C0FE01E258FD4F80815FD20DC017
:10419000D1100BC05AD8882341F0FE01E258FD4FE0
:1041A0008081805890E00E946114E3942296ADCF04
:1041B0001092030180915501882351F08150809322
:1041C000550106C080E07CCCC061D7CDD12C6CCC31
:1041D000DF91CF911F910F91FF90EF90DF90CF90E3
:1041E000BF90AF909F900895282F30E0883058F00E
:1041F0002850310949E0429FC001439F900D11248E
:10420000875A9B4F089545E0429FC001439F900D00
:1042100011248F5C9B4F0895813641F40E94C3683E
:1042200081E00E942D1482EF9DE464D860EC71E17E
:1042300080E10C94F863CF93C82F80918F0D80FF9D
:1042400003C06AE371E102C068E271E188E10E94A3
:10425000F863C13629F410928F0D80E00E942D146E
:104260008091D80881508093D808811103C081E0E3
:104270000E940572CF910895CF93DF93EB01E7E59C
:10428000F8E08F3B19F49091570803C08E3B21F45E
:1042900090819150988310829281992321F091818D
:1042A0009F779083128290819923A1F0813211F03F
:1042B0008E3871F520910208211108C09150988321
:1042C00010820E94C36887E10E9405721092020862
:1042D00080E01EC09881843621F49417C0F4995F61
:1042E00016C0853621F4973090F0975010C0803674
:1042F00011F08E3261F49F5F9083906891830E94E9
:10430000C36810920B021092D90790E080E0988366
:10431000DF91CF9108951F93CF93DF93182FD62F5E
:10432000C42F662329F06FE0842F0E942114C82F28
:1043300080915C024C2F83FF02C0440FD06250E09A
:104340002D2F612F80E60E94FB658C2FDF91CF918E
:104350001F910895FF920F931F93CF93DF93182F10
:10436000F62E0AE08AE0189FE0011124CB59DD4FB8
:104370002FE130E0211B3109029FA001039F500D66
:104380001124BE01CE010A960E94C074FF2049F09C
:10439000BE016A5071094AE050E0CE010E94C0742B
:1043A0000DC0FE0111920A95E9F78091E308888318
:1043B000898384E68A838F8188608F831093E508E0
:1043C00082E0DF91CF911F910F91FF900C94315DAE
:1043D000EF92FF920F931F93CF93DF93E62E142F4C
:1043E000EC0188E0F82E00E0FE01659174918F2DBC
:1043F0000E94F8630E1540F4FE013E9645915491DB
:104400006F2D85E40E940E640F5F229688E0F80EFF
:10441000073051F74FE360E083E40E94AE6411235C
:10442000B1F0612F660F660F660F183028F06853E1
:1044300020E04BE385E403C020E042E480E0DF912C
:10444000CF911F910F91FF90EF900C943464DF9106
:10445000CF911F910F91FF90EF9008950F934430EB
:1044600051F490915A029F70913029F445E553E13F
:104470000F910C94D363022F242F40E257E10E9446
:10448000C1630F9108959C01220F331F280F391F1C
:104490009595879595958795280F391F95958795BB
:1044A0009595879595958795820F931F08954296C8
:1044B00043E7489F9001499F300D1124C901E6E070
:1044C00095958795EA95E1F70895CF92DF92EF925F
:1044D000FF920F931F93CF93DF937B018A01D090BC
:1044E000370895E09D1508F45FC091E09D0D90930D
:1044F0003708EBE08E9FE0011124C257DA4F888124
:10450000882349F081500E9424129C01442737FDE2
:104510004095542F03C020E030E0A901D092370825
:10452000DE80FD2DF870CF2ED3FC0AC089819A81E0
:10453000AA2797FDA095BA2F280F391F4A1F5B1F86
:10454000AB81B0E011960E941E742C8130E02F5F89
:104550003F4F442737FD4095542F0E949574CC203F
:1045600051F089819A81AA2797FDA095BA2F280F2B
:10457000391F4A1F5B1FD0FE07C0509540953095EC
:1045800021953F4F4F4F5F4FE114F10419F08D819A
:10459000F70180830115110529F08E8186958370BE
:1045A000F8018083C90102C080E090E0DF91CF91E3
:1045B0001F910F91FF90EF90DF90CF90089581E0D1
:1045C0000895E82FF0E0EA5EF84EE491862F9927EF
:1045D00087FD909583589F4FEE5FE23038F42AE0D4
:1045E000AC01249FC001259F900D11240895E82F50
:1045F000F0E0EA5EF84EE491E03F29F1ED3F4CF443
:10460000EE0FFF0BEA5EFA4F8081992787FD9095A8
:104610000895ED3FA1F0BCF0EF3F09F0A4F48E2F18
:10462000992787FD909502962FE0289FF001299FFA
:10463000F00D1124E75CF74F8385948508958091F0
:104640003D0190E0089580E090E00895CF92DF92E0
:10465000EF92FF92CF93DF9300D0CDB7DEB7F82E65
:104660001A821982C4DFEF2DF0E0EA5EF84E249141
:10467000422F552747FD5095652F752F415F5F4F9E
:104680004F30510590F54C5A5F4FFA010C94B174BC
:10469000AE014F5F5F4FBE016E5F7F4F8FE0820FB5
:1046A00014DFEA81F0E0E650FB4EE491EA831DC09E
:1046B00024E22A8321E0298318C06CE370E00E9481
:1046C00060746B017C0146E260E0C6010E941772D3
:1046D000C70125E32A8309C0E22FEE0FFF0BEA5E34
:1046E000FA4F8081992787FD90954A8169810E94C0
:1046F00017720F900F90DF91CF91FF90EF90DF90A6
:10470000CF9008950F939FE0499FF0011124E75C3B
:10471000F74F43855485022F0E9439660F91089503
:104720008F929F92AF92BF92CF92DF92EF92FF92C1
:104730000F931F93CF93DF9300D0CDB7DEB7F82E42
:10474000D62EC22EB32E102F80E28A83E42FFF27AD
:10475000E7FDF095EA5EF84EA4908E2D8170982EBC
:10476000E0FE20C0AFE0AA0DA43008F08CC08BE0C2
:10477000A89FD0011124FD01EB56FA4F80818823B8
:1047800009F481C0AF0100E124E08F2D0E949D63F8
:1047900012FD03C008E10F0D06C00CE10F0D88EFFC
:1047A000D80E01C00F2D8E2D8870882EE3FC1F7B44
:1047B00081EFA8160CF43DC084EF8A152CF482E03A
:1047C0008A0D8230F8F035C0AE014F5F5F4FBE01F9
:1047D0006E5F7F4F8FE08A0D78DE2981213011F4E2
:1047E000106203C0223009F41063EA81F0E0EE5059
:1047F000FB4EE491EA83E7FE02C08C2D9B2DC82E70
:10480000B92E17C012FD02C08CEF01C082E0800FEC
:104810009110865F1770012F212F4C2D5B2D6D2D70
:1048200083500E943966E3E3EA0DEA838AEFF80ECB
:104830000AC0882071F18DE38F0D212F4C2D5B2D47
:104840006D2D0E94FB658E2D867069F0E2FE04C01E
:104850008AE08F0D1B7F02C08091450D212F4A8178
:104860006D2D0E9410638A810F900F90DF91CF9180
:104870001F910F91FF90EF90DF90CF90BF90AF907E
:104880009F908F9008954F5F20E06D2D8F2DE6DD76
:104890007FCF802FD2CF0F931F93CF93DF93C82F5B
:1048A000D62F042F122F45EC54E10E94D36340E32E
:1048B000400F212F6D2F8CE08C0FDF91CF911F9136
:1048C0000F910C941063EF920F931F93CF93DF938C
:1048D000C42F122F2E2DDE2DD3709DE7940F9B3FFA
:1048E00080F043E84C0F8251D6DFDD2359F122E0FE
:1048F00042E850E06EE770E08C2F90E00E944F138A
:104900000CC0552747FD50950E94FB65DD23D1F073
:10491000402F612F8C2F0E941E14C82F80910B02F4
:104920008D3B81F48DE78C0F8B3F40F0EC2FF0E056
:10493000EE0FFF1FEA5FFB4FC08101C0CEE782E0B0
:104940000E94315D8C2FDF91CF911F910F91EF90DD
:104950000895EF920F93E22E0DE723E8B4DF0F9155
:10496000EF900895CF93DF939EE0899FE00111249B
:10497000CB50DC4F8C850E942519882339F08D851A
:104980000E942519811104C081E003C080E001C0AC
:1049900082E0DF91CF910895942F9695691B242F83
:1049A000891B0C949F669091140281E0191624F0E3
:1049B000911101C080E0819510921402089521E0C8
:1049C000AC0160E080E00C94D3630F931F93CF930E
:1049D000C62F0E94FB65B8018C2FCF911F910F91BC
:1049E0000C94F863EF92FF920F931F93CF93DF9392
:1049F000E82E142FFB01F490EB012296319644919E
:104A0000222381F08091FA07882321F08091020807
:104A1000882351F02091FB0760E0812F0E9414143D
:104A2000182F02C000E002C00091FC07212FAE0148
:104A30006E2D8F2D0E94C163812FDF91CF911F9129
:104A40000F91FF90EF900895982F862F242F492FD4
:104A50006CEE71E1C7CF0F931F93CF93DF93182FA5
:104A6000D62F022FBA018D2F0E94F863C1E0402F8C
:104A70006D2F8C2F811BE8DFC81B8C2FDF91CF910E
:104A80001F910F910895982F862F242F492F6BE4A3
:104A900073E1A8CF0F9390915A029F7021E091305B
:104AA00009F020E000E04BEC56E10E94C1630F9159
:104AB0000895442321F050E08E5E0C94FB6548EE8F
:104AC00052E00C94D363EF92FF920F931F93CF9316
:104AD000DF93EC01062FF42E1091D907A0912C083A
:104AE000B0912D0820912E0830912F08EFE3F1E0CE
:104AF000868197818A1B9B0B97FDCF9666E09595E3
:104B000087956A95E1F7482F8093FF078085918507
:104B1000821B930B97FDCF9656E0959587955A95F6
:104B2000E1F7982F8093FD07442311F0B783A68304
:104B3000992311F0318720878091FE07811104C0ED
:104B40008091530685FF06C01092FF071092FD0763
:104B50001092FE078091FF07811108C08091FD0728
:104B6000811104C082819381892B11F00E944D1420
:104B7000E090E8088FEFF81609F44DC080913808EE
:104B800081112DC08091E008882319F01092E0086F
:104B90001E2D09DF18166CF41E1510F41F5FC9F4E2
:104BA00088818F1518F48F5F888301C0188210E008
:104BB00010C0882371F011110BC08881882319F06F
:104BC0008150888301C0F88281E08093E00801C0B1
:104BD00011500E3271F481E0809338080AC08130A0
:104BE00041F40E3221F080910208811102C010922E
:104BF00038088091D807B1990BC08F3F19F08F5FAB
:104C00008D3338F091E0909302089093380801C0FA
:104C100080E08093D807E092FA0780910208811122
:104C20002CC08091FD078823A1F04881481B47FDD7
:104C300040E08F2D90E0242F332727FD3095281753
:104C400039070CF04F2D4883E11608F41E2D109201
:104C5000FD078881882389F08091FF07882369F008
:104C6000181B17FD10E08E2D90E0212F332727FD14
:104C70003095281739070CF01E2D003679F190F485
:104C8000023409F46BC028F40132E9F10E3231F13B
:104C900084C0043409F442C008F46EC0053409F439
:104CA0004DC07BC0053609F44BC040F4033609F40F
:104CB00066C0B0F5023609F454C06FC00E3801F179
:104CC0000F3B39F0013809F068C01092020881E00A
:104CD00022C018821092020810E05FC08FEFF81611
:104CE00009F45BC081E090910208911180E080930B
:104CF0000208882309F451C081E0809338084DC030
:104D00008EE80E94C36880910208882319F01092EF
:104D1000020843C080E00E942D143FC01E15E9F137
:104D2000EE20D9F180910208811137C01E1510F4D0
:104D30001F5F01C010E010920B022FC0112369F118
:104D4000EE2059F180910208811127C0112319F03A
:104D5000EE24EA94E10E10920B021EC088818F159A
:104D6000E1F080910208811118C088818F1510F43C
:104D70008F5F0DC018820EC08881882371F08091EA
:104D8000020881110AC08881882319F08150888324
:104D900001C0F882E11608F41E2D209102082111AD
:104DA0000AC031E08091410190914201892B09F4C0
:104DB00030E0832F01C081E0809301081093D90770
:104DC000222311F082E001C081E08093FC07109261
:104DD000E808DF91CF911F910F91FF90EF90089518
:104DE000AF92BF92CF92DF92EF92FF920F931F93F9
:104DF000CF93DF93C82F81E195E1E1DD4AE06C2F8D
:104E00008BED98E060DEC090DB08B090D90786E0BB
:104E1000CE3211F0C03671F48C1578F489EF8C0D18
:104E20008093E9088C2F0E94C3688AE09BE40E946B
:104E30007A1962C08C1508F45FC081E08093E8089D
:104E4000E12CF12C18E065EC74E1812F0E94F863ED
:104E5000AE2C41E34E0D612F8CE00E949B63E70175
:104E6000CC0FDD1FCE5FDA4FD12CCA1005C0BD10AC
:104E700003C00091FC0701C000E080910208882374
:104E800009F486C0D1101BC0002329F062E2898199
:104E90000E942114898329812D3018F443EA55E1B9
:104EA00005C02D3140F42D5F45E957E1612F8CE3BA
:104EB0000E94C16315C02D514FEC52E1F7CF002382
:104EC00031F04DE763E888810E941E148883488191
:104ED000552747FD5095202F612F8CE60E94FB65DA
:104EE000D39482E0D812C1CF185F8FEFE81AF80A86
:104EF000103409F0A8CF41C089EFC80E0EE815E0C4
:104F000071E3E72EE8E0FE2E66EC72E18F2D0E9441
:104F1000F8634E2D6F2D8CE00E949B63E80120E02A
:104F200048816F2D88E10E94A01049815A816F2D20
:104F30008BE40E9429664B8150E04F5F5F4F6F2DDD
:104F400080E60E9429664C8150E04F5F5F4F6F2DD5
:104F50008EE70E94296688E0F80EE394055F1F4FF4
:104F600088E2F812D1CF6C2D660F660F660F685F6E
:104F700020E04EE780E00E943464DF91CF911F91E2
:104F80000F91FF90EF90DF90CF90BF90AF9008957A
:104F9000D1109DCF80CF1F93CF93DF93C82FD62FF3
:104FA000142F47E16BE2F8DC43E06AE28C2F0E94A9
:104FB000AE6443E06BE28FEF8C0F0E94AC64812FF4
:104FC00069EF0E943F74382F375D8D2F67E00E9494
:104FD0003F748C0F25E045E0632F8250DF91CF9125
:104FE0001F910C947F66CF92DF92EF92FF920F9306
:104FF0001F93CF93DF93C2E3D8E0498168818AE2AF
:10500000CADF4A816B8186E5C6DFC4E2D8E0289614
:10501000AAE3FA2E0DE510E0B7E3CB2E8991999122
:105020009C5FB8010E946074DD24D394D60EEC2CF2
:10503000E61A4D2D6E2D8F2D0E94AE644D2D6E2DD6
:1050400081E08F0D0E94AE644D2D6E2D82E08F0D9C
:105050000E94AE6485E0F80E89E4F812DFCFDF919C
:10506000CF911F910F91FF90EF90DF90CF90089517
:1050700046E353E168E388E60C940E640F931F93B4
:10508000CF93DF93D82F162FC42F022F47FF08C0CE
:1050900041E28AEF8D0F0E94106386E08C1BC82FBF
:1050A0002C2F4EE457E1612F8D2F0E94C163DF91B9
:1050B000CF911F910F9108950F931F93CF93DF937B
:1050C000162F042FC62FD0E0AE014F5F5F4F202F69
:1050D000682F86E60E94FB65002329F06FEFCE0162
:1050E0000E942614182F812FDF91CF911F910F91CD
:1050F00008950F93CF93DF93C42FD02FD27001FF69
:1051000003C00E94BA1102C00E94841100FF41C076
:10511000DD23B9F1CD3274F084ED8C0F0E9464115F
:105120002091570130E0280F311D87FD3A9521501D
:10513000310907C08C2F0E946411282F332727FDC7
:10514000309580915701482F440F4250C1E06C2F99
:10515000681B822F0E941E1490915701482F5527DB
:1051600047FD5095292F30E0421753073CF0C91BEB
:105170008C0F0E947411CCE2C80F0BC00E947411F6
:1051800007C040915701642F61958C2F0E941E1417
:10519000C82F8C2FDF91CF910F910895FF920F931D
:1051A0001F93CF93DF93182FF62EEA01022F498128
:1051B000453249F4298522952695277049E554E121
:1051C0000E94C16311C020610E94A0108981855195
:1051D000803150F48F8186FF07C0202F43EC52E1CD
:1051E0006F2D812F0E94D363DF91CF911F910F917B
:1051F000FF90089580919B03882329F08CE091E231
:105200000E947A1981E00895CF93DF93C82F88E038
:105210000E94F86369EA71E188E20E94F863C1368E
:1052200071F028F4CE3269F0C03659F012C0CE3891
:1052300031F0CF3B71F480E00E9405720AC0D2E0E9
:1052400001C0D1E08C2F0E94C36881E00E942D1420
:1052500001C0D0E08D2FDF91CF910895CF93909131
:10526000D6079F3F19F468E971E102C06CE871E16B
:10527000CBDF813019F0823019F127C0C091D607F9
:10528000CF3F19F40E94E5691BC08C2F0E948F103C
:105290002FE130E02C1B3109CAE0C29FA001C39F5F
:1052A000500D1124BC01665F7F4F0E94C074EBE972
:1052B000F3E0DF011D92CA95E9F782E00E94315DBB
:1052C00082EF9DE4CF910C947A19CF9108950F93BA
:1052D000CF93C82F4FE06EE578E08091D3070E940E
:1052E000765C00E12AE04EE558E060E181E00E9452
:1052F0009D634FE360E182E40E949B638091D40749
:10530000882319F062E671E102C065E571E18C2F36
:105310007BDF813019F08230F9F024C08091D4070E
:105320008823A9F083E491E10E9493128091D3072E
:105330000E94BE5C882339F087E10E94057282E0FA
:105340008093D40709C080E00E94057205C0809157
:10535000D3078F5F0E946B608AE49AE2CF910F912E
:105360000C947A19CF910F910895DF92EF92FF92EA
:105370000F931F93CF93DF93EC01062FD42EF62EBD
:1053800018E0E12CFF20B9F0F0FE0EC02D2D4DE706
:1053900051E1612F82E10E94CE63AE01612F88E16D
:1053A0000E940E64E394185FF694FE0184912196A6
:1053B0008111FBCFE7CFCD2DCC0FCD0DCC0F2AEF38
:1053C000210F4C2F67E082E10E949F6644EF4C0F53
:1053D00060915B08660F660F660F685F20E088E1EA
:1053E0000E943464E0DA282FCAE5D8E099818B81E5
:1053F000882351F03091580D36FF08C081508B83BF
:10540000811104C018821CC08FEF8B8380910B0226
:10541000813681F028F4803249F08E3239F012C0A2
:105420008336C9F088F08E3829F00CC018821B82B0
:1054300081E01AC00E94C36810920B0218821B827E
:1054400082E012C012162CF4EA949E1530F49F5F8D
:1054500004C0222339F0911191508B81882311F0DF
:105460008FEF8B83998380E090915B089F5F20E0B2
:1054700000FF02C0915021F006952F5F2830C1F740
:1054800020935C08DF91CF911F910F91FF90EF90D7
:10549000DF900895DF92EF92FF920F931F93CF93C7
:1054A000DF93C82F87EA90E18ADAF090D2088091E2
:1054B0005A08811105C04FE06C2F82ED98E003DBA4
:1054C00061EA70E180E00E94F8630E94915FAC01A4
:1054D00060E086E60E9429661091D2088091D40788
:1054E000823021F41092D1081092D40780910308E1
:1054F00091E0980F191728F4123068F08FEF810FA0
:105500000BC094E0980F911738F48CEF810F8B301B
:1055100018F08AE001C080E080930308082FD0E1F2
:10552000EE24E3941013E12CDD24D394D00E2E2D21
:105530004D2D6D2F82E10E942B6680913A06081353
:1055400005C04AE26D2F81E00E949B634FE06EE54B
:1055500078E0802F0E94765CEE2031F08091D108B7
:10556000882311F001E101C000E12FE04EE558E091
:105570006D2F88E10E949D63D85FD03411F00D2D0E
:10558000CFCF80915A08882309F477C08091D20840
:1055900090913A06981302C0D9E501C0DEE70E9457
:1055A000A75C811101C0D6E980915C0682FFDF73A0
:1055B0004AE06D2F8DEF93E1D8DE813009F09CC079
:1055C000D0915C08D11105C088EA90E50E94401492
:1055D00093C09FEF9D0F923060F50091D208009329
:1055E0003A0680938E0D8C2F0E94C3680E942D5E18
:1055F00000933A06802F0E943C5E809105018260F4
:105600008093050181E00E94315D0E942D5E0E9421
:105610008F190E94AA19809155020E9477140E9446
:105620008C6F80915A08823079F2D23009F055C0DF
:10563000CBCFD53031F48C2F0E94C3681092D407A1
:1056400004C0D33049F48093D4071093D30787E67E
:1056500099E20E947A1950C0D63019F480936208FA
:1056600004C0D73039F4109262081093660889EAB2
:105670009EE2EFCF8093D1083FC0C63638F4C436DF
:1056800088F4C036C1F0C13641F036C0C13829F1C6
:10569000CF3B39F1CE3681F50EC08091D1088823F9
:1056A00059F10FC090913A068091D208981709F4E9
:1056B0008BCF82E00AC0109202088091D108882323
:1056C00019F01092D10818C081E080935A088C2FED
:1056D0000E94C36810925B080FC081E00E942D14E5
:1056E0000BC01092D10810925A0880913A0680930C
:1056F000D20881E00E94835D8091D1088823F9F06F
:10570000CF2DDD27C7FDD095812F90E0C817D90791
:10571000B1F061E0610F81E08F0D0E944A608091DD
:105720003A06181303C0F0923A0606C090E0C81774
:10573000D90729F410933A0681E00E94315DDF9188
:10574000CF911F910F91FF90EF90DF900895CF922E
:10575000DF92EF92FF92CF93DF93FC01EB019C016C
:10576000DC010E94FF739B01AC01DE010E941474F6
:10577000272F382F492F5527DF010E9414746B0102
:105780007C013CE0F694E794D794C7943A95D1F71E
:1057900024E630E02C1B3D0B0E94FF736E5C7F4FB4
:1057A0008F4F9F4F6C0D7D1D8E1D9F1D24E630E099
:1057B00040E050E00E947374C901DF91CF91FF90E7
:1057C000EF90DF90CF9008951F93CF93DF936115F3
:1057D000710519F1192F111F1127111F19F091953A
:1057E0008195910977FF0FC0719561957109C0E0AE
:1057F000D4E09E01281B390BC901A9DF9E01281B9B
:10580000390BC90101C0A3DF112329F02227332757
:10581000281B390B01C09C01C901DF91CF911F9159
:105820000895EF920F93CF93DF93382F862F642F35
:10583000922F332319F02091FC0701C020E0C09182
:10584000E6084EE0C49FE0011124CB50DC4F9336B4
:1058500029F4032F4C854DDC8C8724C0923629F423
:10586000032F4D8546DC8D871DC0E02FF0E0E90F4A
:10587000F11DE90FF11DEE0FFF1FEE0DF11DEC0FF5
:10588000FD1FEF01011106C0E22E04E62CE948815C
:105890001AD807C048814C59E22E04E620E013D8FC
:1058A00084568883DF91CF910F91EF90089590E017
:1058B000E92FF0E0ED52F94EE491E81721F0EE23E4
:1058C00021F09F5FF5CF892F089580E008958234FD
:1058D00030F4E82FF0E0ED52F94E8491089580E223
:1058E0000895DF92EF92FF920F931F93CF93DF9370
:1058F000F82E162FEA01E22ED02E64E576E1812FF4
:105900000E94F86300E12E2DAE01612F82E40E9417
:105910009D63DD2099F18F2D880F8F0D880F2091C9
:10592000020846E0612F8E5B0E9434644E2D440FC6
:105930004E0D440F4C5F6FEF610F29E080E40E9431
:105940009F66809102088823C9F0CF0DD11D888100
:105950008111ADDF2D2D41E460E00E941414B7DF0A
:10596000488150E0282F332727FD309542175307F1
:1059700029F088838091FB070E94315DDF91CF91F0
:105980001F910F91FF90EF90DF900895FF920F937A
:105990001F93CF93DF93C82FD62FF42E122F622F91
:1059A000842F0E94C912FC01E53F81E0F80774F0E2
:1059B0009BE09E0F9F1510F09CE09E0F40E3490F67
:1059C000202F6D2F8C2F0E94106307C0212F42E0E3
:1059D00055E16D2F8C2F0E94C163DF91CF911F91F4
:1059E0000F91FF9008957F928F929F92AF92BF92F6
:1059F000CF92DF92EF92FF920F931F93CF93DF939B
:105A0000182FC091E9082AE0C29FE0011124C05F6D
:105A1000DA4F80E291E10E94DF2443E0612F87EDBD
:105A200098E051D84091E9084F5C60E080E30E9423
:105A30009B63B090D70878E0C72ED12CE3E0AE2E60
:105A4000BD1003C09090FC0701C0912C82E0D816D5
:105A500009F467C0E3E0DE1609F478C0F1E0DF1670
:105A600081F062E071E18C2D0E94F86301E09110F9
:105A700001C000E0292D48856C2D80E33ADB888742
:105A800080C09110A092E8086CE3762E812C809162
:105A9000D907881511F000E001C0092D4091E908EF
:105AA0004F5F282D6C2D872D71DF992099F1809102
:105AB000D90788112FC080910108882359F18E01E0
:105AC000080D111D080D111DF801E080F180FBE0AB
:105AD000EF1AFEEFFF0A24EFE21621E0F20624F4AB
:105AE00054EFE52EFF24F39422E048EF51E064EFF9
:105AF00071E0C7010E944F138E159F0559F0843F36
:105B0000E1E09E0711F480E090E0855F9140F801AC
:105B1000918380838394F6E07F0E24E08212B7CFD6
:105B200030C0992051F089856FE08F700E94211458
:105B30008F709985907F982B998749854F70292D73
:105B4000206285E0489FA001112417C0992061F0D0
:105B500089856FE082958F700E9421148295807FE5
:105B600099859F70982B9987498542954F70292D6B
:105B70002062E5E04E9FA00111246C2D86E60E9474
:105B8000FB65D394F8E0CF0E24E0D21259CFDF9119
:105B9000CF911F910F91FF90EF90DF90CF90BF902A
:105BA000AF909F908F907F9008951F93CF93DF9336
:105BB000C82FD62F142F4FEF50E10E940E6440E300
:105BC000410F6D2F8CE08C0FDF91CF911F910C94C2
:105BD0009B63BF92CF92DF92EF92FF920F931F933E
:105BE000CF93DF93C82F8EE295E10E94DF2443E03C
:105BF0006C2F83ED98E00E946325B090D308C036E7
:105C000011F0CE3649F4B092E9088C2F0E94C36897
:105C100083EF9CE20E947A1960EB70E180E10E94C0
:105C2000F863F0E1EF2EF5E0FF2EA8E1DA2E10E0A8
:105C3000CC24C3941B11C12CE7018985882331F042
:105C40002C2D4AE26D2D89E70E9410631F5F412FC2
:105C50006D2D86E0AADF2C2D48856D2D88E10E94F0
:105C60008411DCE3C0E00C2D2C2F412F6D2D8D2FE6
:105C70008DDECF5FDA5FC430B1F78AE0E80EF11C49
:105C800088E0D80E1430A1F60E946A1A682F660FB9
:105C9000660F660F615F29E04AE180E0DF91CF91F6
:105CA0001F910F91FF90EF90DF90CF90BF900C94D9
:105CB0009F661F93CF93DF93162FEC01112329F0DA
:105CC00089910E949B691150F9CFDF91CF911F916B
:105CD0000895CF93C82F0E94A2698F3F21F08C13A3
:105CE000FACF81E001C080E0CF910895CF93C82F13
:105CF00081E00E949B6980E00E949B698C2FCF917C
:105D00000C949B69EEE5F8E01382128282E08093A6
:105D1000E20884E40C949B690F932091640830910D
:105D2000650842E3429FC001439F900D112461EE3C
:105D300071E00E944C74062F28E044E660E38EE098
:105D40000E94AA660F910895AC0168E184E20C9468
:105D50000E649F92AF92BF92CF92DF92EF92FF922A
:105D60000F931F93CF93DF93B82ECEE5D8E08C81AD
:105D7000882319F087EF90E102C08FEE90E10E9436
:105D8000DF24A89521E6B21659F08FEBB81217C0A0
:105D90000E9489691092E20819821092D6080FC0F9
:105DA0008AE50E949B6980913A060E943C5E89E0E8
:105DB0008093E2081092020881E60E94C368C090B6
:105DC000D6084091E20850E04A30510508F084C1FD
:105DD000FA01ED59FF4F0C94B1748BE10E949B695D
:105DE0008BE10E949B6918821B8281E09FC08B819E
:105DF000853030F48EE36DDF8B818F5F8B836CC1D8
:105E00008C81882341F01D8287E08093E20882E440
:105E10000E949B6961C176DF5FC127E08C2D622FF4
:105E20000E943374829F202D1124298387EE90E1F4
:105E30008BDF1CE00AE00E94A2698F3F09F44CC18D
:105E40002091D4083091D5082F5F3F4F3093D5086B
:105E50002093D408833009F469C08D3009F480E0C0
:105E60002A819881FE01129FE00DF11D1124E90F96
:105E7000F11D8187811116C09B818981981750F08F
:105E800081E0820F8A83883028F088E50E949B6930
:105E900083E04CC08EE40E949B698B818F5F8B8373
:105EA0001882C9CF81E0890F8B3010F48883C3CF6B
:105EB0000883C1CF8A81982E883010F017E0912E88
:105EC0004981480F41506B2D86ED98E00E94632573
:105ED0008981C81A8C2D873008F09DCF7E0199E00A
:105EE000E90EF11C00E010E0B8E0AB2EDD24C7FCA9
:105EF000D094091598F421E0C016D10609F020E0ED
:105F00002061A7016A2D8CE00E94D36328E0A20ED5
:105F10000F5F1F4F8CE0E80EF11CEBCF90E6B9123B
:105F2000DBC082E50E949B691D8284E08093E208C9
:105F3000D3C08DED90E108DF8D81811120C01F82DB
:105F40001E8282E7C6DE882309F44FC08DE0CEDED4
:105F50008C2D90E02981821B91092CE0289FF00173
:105F6000299FF00D11243996EC0FFD1F82EC8387D9
:105F700083E084876DE0CF019CDE188264C08130AD
:105F8000A1F50E94A2698F3F2FEF920771F19881CE
:105F900021E0290F2883FE01E90FF11D8187888107
:105FA0008F3078F38E819F8102EC13E0081B190B70
:105FB0000D30110510F00CE010E0A8016AE678E061
:105FC000855B9D4F0E94B7748E819F81800F911FCA
:105FD0009F838E83823C934008F48AC085E080933F
:105FE000E20885E60E949B69188296DE75C086ED00
:105FF00090E1AADE88850E94365C882309F46CC093
:1060000086E094CF8DEC90E15CC086EC90E19CDE64
:106010008D8181111AC01F821E8282E65ADE88237A
:1060200021F388850E94A95C8DE060DE6AE08BE444
:1060300092E03FDE8BE00E949B6982EC0E949B69AC
:1060400083E00E949B6981E02FC0813049F483E6A0
:1060500040DE882351F282E08D831F821E82C5CFED
:106060008230D1F48E819F81823C934028F083E07E
:106070000E949B6984E018C08CE038DE8E819F818D
:106080006CE0855B9D4F15DE83E08D838E819F8163
:106090000C969F838E83A9CF833041F484E619DE6A
:1060A000882309F4A2CF82E08D839FCF86E011DEA2
:1060B000882309F49ACF88E08093E20896CF8AEB90
:1060C00090E142DE09C08AE704DE882329F00E94BD
:1060D000936980E00E942D14DF91CF911F910F9161
:1060E000FF90EF90DF90CF90BF90AF909F9008957A
:1060F0008EE678CF21E0411101C020E0405D0C9494
:1061000010630E9482102091CF083091D008AC011A
:10611000421B530B9A01283E334088F09093D008DD
:106120008093CF0880915A028F70823041F485E1CC
:106130000E942519882319F087E00C9405720895B0
:106140000F9300E020E00E9439660F9108951F939D
:10615000CF93DF93182F8CE990E10E94DF2416364D
:1061600028F4143630F4113659F00FC01E3841F0BF
:106170000CC08091CE0891E089278093CE0805C09D
:106180001092CE0880E00E942D148091CE088823C2
:1061900009F43FC0C6E0D1E0103641F48FEF8883A8
:1061A00019821B821A8287E10E94057266E670E1FD
:1061B00088E00E94F8634981469550E068E086E6F1
:1061C0000E9429664881469550E060E186E60E947B
:1061D000296649818881481B469550E068E186E63A
:1061E0000E9429668A819B8129E1289FA001299F1D
:1061F000500D1124569547955695479520E360E23A
:1062000086E60E94FB6563E570E188E30E94F8631F
:1062100029C0C9E3D8E06CE370E180E00E94F86334
:106220004091CE075091CF0768E08AE289DF4C8128
:106230005D8168E08EE484DF4F81588560E18AE209
:106240007FDF49855A8584E0569547958A95E1F721
:1062500060E18EE475DF4091CC075091CD0760E09E
:106260008EE46EDFDF91CF911F910895CF93DF937E
:10627000282F30E095E0899FE0011124C050DE4FC7
:106280004C818FE0829FF001839FF00D1124E75C29
:10629000F74F9881898195878687442311F090E094
:1062A00080E0938784871086178215821482128675
:1062B000118611821082DF91CF9108951092CF073D
:1062C0001092CE0780E0D2CF81E0D0CF5F926F9264
:1062D0007F928F929F92AF92BF92CF92DF92EF9276
:1062E000FF920F931F93CF93DF930CEC17E0F8010D
:1062F0008F0186818F5F868379E3A72E78E0B72EA2
:10630000E4E0EE2EE2E0FE2E812C55245394E501CC
:10631000811003C08091BA0502C08091BB0588231B
:1063200009F48FC18D324CF08C520E9425199E8148
:10633000891709F486C18E8302C00E94251988231B
:1063400009F47FC1811002C0B9DF01C0BDDF66243E
:106350006394F70132979080F701319770808EEF48
:10636000890D823028F4C0902808D090290802C0F6
:10637000C12CD12C80913608882319F0C12C6CEFE8
:10638000D62EF3E0F91548F4E92DF0E0EE0FFF1FEB
:10639000EE52F84FC080D18002C0992059F12CE212
:1063A000271504F5F8018481958128813981822B94
:1063B000932B2B81822B2681822B2A81822B892B66
:1063C00009F41A8284ED870D0E942519882341F073
:1063D0009A81911105C091E02B81211190E09B835E
:1063E0008A8308C0772029F0872D0E9425198B8386
:1063F00001C05B828B81882379F061100DC0FCEFB6
:10640000DF1AD7FE03C02FE3C20ED11C46E0D5949D
:10641000C7944A95E1F701C0C12C888199818C0D00
:10642000911D998388830E948210F801C480D580D1
:106430008C199D098436910508F46AC0668170E064
:10644000888199810E946074462F99838883F8011E
:1064500081100DC0208131812F5F3F4F3183208318
:10646000228133812F5F3F4F3383228307C01682FF
:10647000F4E6CF0ED11CF801D582C482442331F05A
:106480002F8138852F5F3F4F38872F83611009C0D8
:106490002B81222331F02C813D812F5F3F4F3D83A3
:1064A0002C8377277595679589859A85680F791F5D
:1064B0007A876987F7013497808191819C878B87E0
:1064C0009920E1F0F1E09F1209C0711004C0F801B9
:1064D000628173810EC06C817D810BC0F2E09F12DE
:1064E00003C06F81788505C024E0769567952A956D
:1064F000E1F79C01261B370B3C872B87F701208196
:10650000222331F02B853C85821B930B9C878B8744
:106510008394FFE0AF0EB11C25E0E20EF11C32E0E7
:106520008312F5CE09E318E0F8018F01F090040220
:106530008091000290910102C385D485258536851E
:106540002C173D0709F47FC0D687C58723812223F6
:1065500009F479C0FF2021F09C012C1B3D0BE901BF
:106560002091530622FF2DC0892B59F1CE31D10540
:1065700019F469E289E10BC0C431D10519F46AE26A
:106580008AE105C0CA30D10529F46BE28BE10E9493
:106590000F720AC0C630D1052CF4D7FD05C06C2F90
:1065A0008CE1F5CF80E001C081E09091530693FF2C
:1065B00008C0882331F082E390E090933B01809300
:1065C0003A01D7FF05C0FF2019F0F801C385D48533
:1065D0006CE370E0CE010E946074DC01CB0140915D
:1065E000530641FF1AC0AB2BC1F440915C0641FF3A
:1065F00007C0009741F046E260E00E94177203C0B6
:1066000080E00E9405728091530683FF06C082E3FA
:1066100090E090933B0180933A01F8018385948543
:106620000A960A9780F48CE10E94057280915306C5
:1066300083FF09C082E390E090933B0180933A018D
:1066400002C0612C86CEDF91CF911F910F91FF90F8
:10665000EF90DF90CF90BF90AF909F908F907F9002
:106660006F905F9008950F9304E12AE04BE452E0AD
:10667000682F88E10E949D630F9108950F931F93E7
:10668000CF93DF93D82F162FC42F423049F4809137
:106690007F0682FF12C08FE10E94A26825E10AC036
:1066A000463059F480917F0684FF07C085E20E943E
:1066B000A2682BE1280F00E006C081E08C0F0E9449
:1066C0002519082F2C2F4CEE52E0612F8D2F0E94A0
:1066D000C163DF91CF911F910F9108956F927F92C7
:1066E0008F929F92AF92BF92CF92DF92EF92FF92E2
:1066F0000F931F93CF93DF9391E09093FB079091BB
:10670000C60190FF02C044E001C043E06AEC78E0BB
:106710000E943C21F82E4091EA084150682F8AECF3
:1067200098E00E946325E090CA08D090FC07009191
:10673000570810E00C30110508F0C6C6F801E359FF
:10674000FF4F0C94B17481E795E10E94DF248091A2
:10675000C60180FF02C06BE001C06AE06093EA08F6
:1067600041E04E0D67508DE090E10E94E821ACC6FB
:1067700084EE93E10E94DF2486E08093EA08EE2015
:1067800011F0C0E001C0CD2D40913B0650E004E087
:1067900010E12C2F68E086E60E94E524CC2351F01E
:1067A0004DE26AE080913B060E941E1480933B06F6
:1067B0000E94ED6668EB7FE080E10E94F86381E073
:1067C000E8120CC040915701642F619580913E06FC
:1067D0000E941E1480933E062D2D01C020E04091A2
:1067E0003E0660E180E60E94841141E092E0E912F9
:1067F00040E08091590668E186FB882780F90E9475
:1068000024259091590680FB96F990935906C091E2
:106810005506E3E0EE1207C068E78C2F0E942114B2
:10682000C82F2D2D01C020E04C2F440F440F4C0FDA
:1068300060E286E60E945925CC2329F043E760E216
:1068400088E70E949B63C0935506C0915D06F4E003
:10685000EF1206C068E78C2F0E942114C82F01C0D8
:10686000D12C4C2F440F440F4C0F2D2D68E286E69F
:106870000E945925CC2329F043E768E288E70E946B
:106880009B63C0935D0641E085E0E81240E08091A3
:10689000530660E383FB882780F90E9424259091AA
:1068A000530680FB93F9ACC48BE993E10E94DF248B
:1068B00086E08093EA0860E97FE088E00E94F86360
:1068C000C0916906C95FE11008C0DD2DD06467E0A2
:1068D0008C2F0E942114C82F01C0D0E44C2F50E00F
:1068E0002D2F68E086E60E94FB65C750C0936906BD
:1068F00021E0E21220E040915006469546954695EB
:10690000477062E67FE080E10E94F2248770880F82
:10691000880F880F90915006977C982B9093500683
:1069200040915C06443008F044E021E092E0E91236
:1069300020E06CE27FE088E10E94F224843008F0DD
:1069400087E080935C06E3E0EE120AC044E661E073
:1069500080915A060E941E1480935A0621E401C0B9
:1069600020E440915A0650E060E286E60E94FB6512
:10697000F4E0EF1209C065E080915B060E942114EB
:1069800080935B0621E401C020E440915B0650E067
:106990000BE11FE068E286E60E94E524C091530601
:1069A000C695C17067E975E180E30E94F86341E034
:1069B00085E0E81240E060E38C2F0E94242590914E
:1069C000530680FB91F91CC483EB93E10E94DF2402
:1069D0008AE08093EA0895E09E1508F4C3C00E94FF
:1069E00038286FED7EE088E00E94F86341E0E11016
:1069F00040E080916D0668E081700E9424259091AE
:106A00006D0680FB90F990936D06C0915306C1709E
:106A100041E0E41240E060E18C2F0E942425817067
:106A20009091530680FB90F9909353068C130E942B
:106A30008F1941E0E2E0EE1240E08091590668E1F2
:106A400085FB882780F90E9424259091590680FBB8
:106A500095F990935906F3E0EF12D12CE091560688
:106A6000F0E0E95AFC4FD491CCE6ED2FE370F0E072
:106A7000ED5FFA4E44912D2D60E28C2F0E94106341
:106A8000D695D695C650C43581F7DD2039F067E13B
:106A9000809156060E9421148093560614E2C0E0AD
:106AA000D0E02C2F47E754E168E2812F0E94CF62AB
:106AB00020916E0630E00C2E02C0359527950A9481
:106AC000E2F720FF06C020E042E168E2812F0E9449
:106AD00034642196185E143821F794E0E9120FC04F
:106AE0008091C60180FFFFC46FE080916E060E9416
:106AF000211480936E068091580D86FFF4C4809116
:106B00005106E5E0EE1213C090910208992389F036
:106B100063E00E94211490915106891761F09091D1
:106B200059069F77909359068093510604C020E040
:106B300003C021E001C022E041E3480F60E382E1AD
:106B40000E941063D4E2C0E08C2F0E94751020E0F8
:106B5000482F60E38D2F0E94A010CF5FD85EC43015
:106B600099F7B2C4F9E0FE1528F489E08093CA08C9
:106B700069E0E62E83E08093E808CFE6D6E010E0F7
:106B800058E0F52E00E0212F42ED52E06F2D8EE10E
:106B90000E94C16301E086E0810FE81200E024E07A
:106BA000AE016F2D8091D9070E94712C88E0F80EFC
:106BB0001F5F2496143031F787C48CEB93E10E9459
:106BC000DF2486E08093EA086CEB7EE088E00E9498
:106BD000F863E1100BC0CD2DC06448E768E28091F6
:106BE0003C060E941E1480933C0601C0C0E42C2F7A
:106BF00040913C0668E086E60E94096691E0E91251
:106C000009C04EE666EF809152060E941E148093E2
:106C1000520601C0D12C80915206482F552747FDBE
:106C20005095465F5F4F2D2D60E180E70E94FB6528
:106C300021E0E2E0EE1220E0809150064BEA5EE0B7
:106C400068E181700E942B259091500680FB90F99D
:106C50009093500621E0F3E0EF1220E0809150067F
:106C60004BE358E160E2869581700E942B2590915C
:106C7000500680FB91F99093500621E084E0E812E1
:106C800020E0809150064CE95EE068E282FB8827B4
:106C900080F90E942B259091500680FB92F99093E9
:106CA000500621E095E0E91220E08091500687FB34
:106CB000882780F94EE85EE060E30E942B259091E2
:106CC000500680FB97F990935006FEC38CEC93E13D
:106CD0000E94DF2486E08093EA08E11003C089E087
:106CE0008093E80801E0E11000E02AE04EE556E07C
:106CF00068E08091D9070E94712CC0915306C2FBB5
:106D0000CC27C0F968E875E180E10E94F86341E0B2
:106D1000E41240E060E18C2F0E94242590915306FC
:106D200080FB92F99093530621E0E2E0EE1220E01E
:106D30008091530640E85EE068E1829581700E9490
:106D40002B259091530680FB94F99093530621E0F4
:106D5000F3E0EF1220E08091590644E75EE060E244
:106D6000829581700E942B259091590680FB94F9A1
:106D70009093590621E084E0E81220E080915306C8
:106D80004AE65EE068E285FB882780F90E942B25B1
:106D90009091530680FB95F990935306C091590644
:106DA000C7FBCC27C0F96EE57EE080E30E94F86364
:106DB00041E095E0E91240E060E38C2F0E94242539
:106DC0009091590680FB97F9909359067DC384ED05
:106DD00093E10E94DF2469E777E080E105C189E55E
:106DE0009EE00E94DF2410E0C0E0C43018F0D8EF2D
:106DF000D10F01C0D12F80917F0601E00C0F82FFDF
:106E000004C0C23011F442E005C084FF07C0C630A0
:106E100029F446E06D2F80E331DC0EC020E0402FE6
:106E20006D2F8AE20E9484118FE08C0F0E94F86718
:106E3000482F6D2F84E45ED9C02F185F0930A9F662
:106E400067E37EE080E10E94F863D8E3C0E08C2F26
:106E50000E94F867482F6D2F80E24CD9CF5FD85041
:106E6000C630A9F74FE25EE068E184E50E940E6457
:106E700016E0C0E2D0E02D2F47E754E16C2F84E507
:106E80000E94CF62812F0E94F867482F6C2F8CE6FA
:106E900031D981E0810F0E94F867482F6C2F88E775
:106EA00029D9DF5FC85F1E5FD43029F780917F0644
:106EB00086FF0CC06AE27EE088E00E94F8638BE205
:106EC0000E942519482F68E088E714D980917F0631
:106ED00087FFFAC265E27EE080E10E94F8638CE2FF
:106EE0000E942519482F60E188E704D9EDC281E2AC
:106EF0009EE00E94DF2481E08093EA081092560110
:106F0000D0E0C0E019E10D2D006241E46D2F88E171
:106F10000E949B6341E34C0F6D2F8EE10E949B63A7
:106F20008C2F0E94FA15AC016D2F8AE20E9410642A
:106F3000C43028F48C2F0E947510815003C0C730D4
:106F4000D9F08C2FE82FF0E0EE0FFF1FEC5DF74F2C
:106F500020813181129FF001139FF00D1124F7FF62
:106F600002C0E150FF4F5F2F550F550B4F2F6D2F74
:106F70008AE50E94296605C0402F6D2F8AE50E9490
:106F80001D66CF5FD85FC83009F0BFCF6DE17EE0EE
:106F900088E20E94F863409100015091010160E392
:106FA00088E70E94296681E08093FE0780910208AD
:106FB000882309F489C24FE761E880913D060E9469
:106FC0001E1480933D0680C28CED93E10E94DF2465
:106FD00086E08093EA088090D9078091630081FF62
:106FE00006C066E17EE088E10E94F8636DC266E05B
:106FF0007EE088E00E94F863C7E4D6E0A12C10E1AF
:1070000033E0732E992493949A0C20E0492D612F3C
:1070100080E00E94A010B12CEA1004C07092E80831
:107020008B1419F020E0C12C02C0CD2C22E0E2E04C
:10703000BE16D1F1F3E0BF1609F44DC081E0B816D9
:1070400089F04981429546954695437069EF7DE008
:10705000812F0E94F2248295880F880F807C99816D
:107060009F731FC00981000F000F059505959DE0D6
:107070000902F0011124F7FD3396AF0155954795AC
:10708000559547952C2D612F82E40E94FB65C1FE2A
:107090003AC04FE161EE802F0E941E148F739981D8
:1070A000907C982B99832FC06880E62DE7706E2E18
:1070B00020E12E0F0C2D45E957E1612F88E40E9455
:1070C000C163C1FE20C063E0862D0E942114877039
:1070D0009881987F16C008810595059505952C2DFA
:1070E000402F612F8AE50E948411C1FE0CC04FE041
:1070F00061EF802F0E941E14880F880F880F9881DF
:107100009770982B9883B394F4E0BF1285CF185FE3
:107110002296103311F0A92C75CF84E0E8120BC031
:10712000CD2DC06248E266EF809157060E941E1482
:107130008093570601C0C0E240915706552747FD8E
:107140005095465F5F4F0EEE1DE02C2F60E38EE4FE
:107150000E94E52404E211E0CFE3D6E090E3D92ECB
:10716000F801419151918F0129913991421B530BA3
:10717000440F551F20E268E38D2D0E94FB65F8E166
:10718000DF0E80E9D812ECCF95E0E91215C0E0E6F9
:10719000FE1214C01092020888E0E4E2F1E0AFE3CE
:1071A000B6E001900D928A95E1F781E00E94315D91
:1071B00087E10E94057202C020E001C021E04AEE92
:1071C0005DE068E380E00E94D3637EC183EC93E1DD
:1071D0000E94DF2488E08093EA08E11014C00E9436
:1071E00038288091530621E042EE5DE068E086FB9E
:1071F000882780F90E942B259091530680FB96F9F1
:107200009093530661C167E97DE088E00E94F863CE
:10721000C0E008E0C0907F06C23051F0C33069F092
:1072200040918006C13079F442954F7010E10DC055
:10723000409182064F7010E408C04091820642954A
:107240004F7010E802C04F7014E0FF24F394FC0E5E
:1072500021E0EF1020E063E77DE0802F0E94F22420
:10726000D82F812F80958C21D11103C080937F0668
:1072700003C0182B10937F0680917F06C8120E94CE
:10728000D410C23051F0C33069F0C130A1F4D295AE
:10729000D07F909180069F7012C0DF70909182061F
:1072A000907F05C0D295D07F909182069F709D2BD4
:1072B0009093820607C0DF7090918006907F9D2B8F
:1072C00090938006085F083211F0CF2DA3CFF5E030
:1072D000EF1611F040E001C04D2D8091830668E269
:1072E00081700E9424259091830680FB90F99093F1
:1072F000830686E0E81611F040E001C04D2D809134
:10730000830660E3869581700E9424259091830610
:1073100080FB91F99093830697E0E912D12C80913C
:1073200083064D2D68E382FB882780F90E9424257F
:107330009091830680FB92F990938306C5C087EAFB
:1073400093E10E94DF2481E08093EA081092CA084A
:10735000CEE5D8E010E0812F0E94FA152E853F85FA
:10736000821793070CF49C013F872E874C8D5D8D0F
:10737000481759070CF4AC015D8F4C8F143060F046
:107380002E853F85240F351F37FF02C02F5F3F4FEB
:1073900035952795398328831F5F22961730D9F6B4
:1073A000809188088093FE07E0E2FE1621F0FFEB53
:1073B000FF120EC00BC08F5F80938808833041F4AA
:1073C00087E10E94057281E00E94315D1092880879
:1073D00080918808813089F050F0823009F072C0C5
:1073E00010925601ECE6F8E0CEE0D6E01FC062E66F
:1073F0007DE088E10E94F86365C0CEE5D8E0D12C3D
:1074000018E9E12E1AE3F12E08E615ECFF86EE8668
:107410001D8F0C8F8D2D0E94FA1589939993D3940B
:1074200087E0D812F3CF64E57DE043C061917191AC
:10743000848595859B01281B390B37FF03C0319547
:1074400021953109233331053CF1DF0150974D91EE
:107450005C91598348839A01261B370BB90137FF8A
:1074600002C0615C7F4FB6E075956795BA95E1F70C
:10747000261B370B3F872E87841B950B9C0197FF9C
:1074800002C0215C3F4FA6E035952795AA95E1F70C
:10749000821B930B9D8F8C8F229698E0EA37F90719
:1074A00029F60E94F85B909339068093380662E4CF
:1074B0007DE080E10E94F8634CEE53E168E182E1F7
:1074C0000E940E640E94F327DF91CF911F910F91CC
:1074D000FF90EF90DF90CF90BF90AF909F908F90F4
:1074E0007F906F90089529E04CE567E283E20E9467
:1074F0009F6605CBCF93DF93C82FD62F462F60E230
:10750000BDD841E04D0F68E28C2FB8D842E04D0F56
:1075100060E38C2FDF91CF91B1C81F93CF93DF939E
:10752000EC01862F11E0683008F410E00E94F4208E
:10753000FC019E013C5F37FD0DC0211588E0380736
:1075400084F0112319F048E050E002C044E050E01C
:10755000E40FF51F8081992787FD9095982F882744
:1075600023C0832F112321F03327220F331F02C0A2
:1075700086953170482F50E0E40FF51F608140E0A0
:1075800052E0421B530B559547956403C001659F1C
:10759000900D11246181359527956203A001639FA9
:1075A000500D1124840F951F69E170E00E946074F2
:1075B000CB01DF91CF911F910895BF92CF92DF92BF
:1075C000EF92FF920F931F93CF93DF93182F7B01BE
:1075D0000E94B224C82E812F0E940218811104C07B
:1075E00001E01E141F040CF400E08EE0189FE0017F
:1075F0001124CB50DC4F84E0C89E60011124F601B9
:10760000E00FF11DEC0FFD1FB080812F0E940218CA
:107610008823A1F08B2D0E94FF17682F772767FD25
:107620007095C7019C5F97FD0196959587950E947F
:10763000E42B7C01EE0CFF1C00E00BC08B2D0E94A4
:10764000FF17682F772767FD7095C7010E94E42B0D
:107650007C01CC0DDD1DC00FD11D8A8144E660E0A8
:107660008C590E94E9179701A82FBB27A7FDB09559
:107670000E94F97324E630E040E050E00E949574E7
:10768000E901812F0E9402188111D450CE01DF91AF
:10769000CF911F910F91FF90EF90DF90CF90BF900F
:1076A0000895DF92EF92FF920F931F93CF93DF9392
:1076B000D62E20EEF22EF80EC0E0DCEF0FE730E21F
:1076C000E32ED11005C06091E708CE0126DF04C08B
:1076D000BE018091E60871DF97FD4F969C0195E011
:1076E000359527959A95E1F7122F0F3709F4022F58
:1076F000412F552747FD5095401B510907FD5395D4
:1077000057FF03C0519541955109423030F46E2D19
:10771000611B8F2D0E9460640CC001171CF09FEF4D
:10772000940F01C090E06E2D611B691B8F2D0E948C
:10773000AE64112321F060E28F2D0E946064F39407
:10774000A096C03284E0D80711F0012FBACFDF91A4
:10775000CF911F910F91FF90EF90DF900895DF92EE
:10776000EF92FF920F931F93CF93DF93D82E8091C8
:10777000E708EE24E394883008F4E12C0E94F4201A
:10778000EC0140E460E08CE50E94AE64F12C0CE971
:107790001FEF2F2D30E0EE2019F049E050E002C03D
:1077A00045E050E0241735075CF5C90145E0880F36
:1077B000991F4A95E1F7EE2019F064E070E002C0ED
:1077C00062E070E00E946074E62FDE01A20FB31F3A
:1077D0002C9130E22302C0011124B8010E94607490
:1077E000DF1005C0625E25E045E08AE304C0615E0B
:1077F00023E043E08BE38E0F0E949F66F394C9CF92
:1078000060E08CE5DF91CF911F910F91FF90EF9099
:10781000DF9047CF5F926F927F928F929F92AF924D
:10782000BF92CF92DF92EF92FF920F931F93CF936D
:10783000DF93882EAA24A3948091E708883008F467
:10784000A12C85E493E10E94DF24AA2011F049E0F5
:1078500001C045E0682D8FED98E00E9463258FEB15
:10786000881202C01092DE084091E70850E04F5F96
:107870005F4F21E060E08AE20E94FB658091E708AB
:107880000E94F420EC01B090DF086090FC07AA2071
:1078900019F0F9E07F2E02C0E5E07E2E5C2E0C2F61
:1078A0001D2F65E0E62EF12C70E1972ECB2CD12C0C
:1078B000802F8519B81611F020E001C0262DF8019F
:1078C00041918F01552747FD5095692D88E10E9410
:1078D000FB65AA20A1F0F9E0EF1689F0CE14DF04D1
:1078E00011F020E001C0262DFE01EE0DFF1D4081AC
:1078F000552747FD5095692D80E30E94FB6588E080
:10790000980EEFEFEE1AFE0AF8E39F12D1CFB714EC
:1079100011F020E001C0262D4EE353E168E38CE036
:107920000E94D363B7103AC0809102088823F1F116
:1079300080920B021091DE0820E044E06CEF812F72
:107940000E941414082F8093DE08811779F1AA2071
:1079500011F024E001C022E0122F119530E059E12E
:10796000F52EE12FFF27E7FDF0952E173F0794F046
:10797000EC0FFD1FE20FF31F1002A0011124F49E73
:10798000C001F59E900D1124B9010E9460746083BE
:107990001F5FE7CF82E00E94315D08C0CB0DD11D93
:1079A00044E66CE988810E941E1488838B2DDF9148
:1079B000CF911F910F91FF90EF90DF90CF90BF90EC
:1079C000AF909F908F907F906F905F90C8CEEF9216
:1079D000FF920F931F93CF93DF93C62FD0E0FE014A
:1079E000EE0FFF1FE35FF94F21813281821B930B62
:1079F0009C01BC01882777FD8095982F0AE0660FCF
:107A0000771F881F991F0A95D1F7121613061CF4C9
:107A1000258D368D02C0278530892436310514F432
:107A200024E630E0442737FD4095542F0E9495749A
:107A3000790121308CEF380744F0211584E03807B4
:107A40003CF0E12CA4E0FA2E03C0E12CBCEFFB2EAD
:107A50000E949610882379F080915106082F0170BA
:107A600010E082E090E0801B910BC817D90719F451
:107A7000F194E194F108C701DF91CF911F910F912B
:107A8000FF90EF9008952F923F924F925F926F92E6
:107A90007F928F929F92AF92BF92CF92DF92EF929E
:107AA000FF920F931F93CF93DF93CDB7DEB7A197CC
:107AB0000FB6F894DEBF0FBECDBF8F879B876D8B4F
:107AC00080915106880F880F9E012F5F3F4F49011B
:107AD000E12CF12C1D8E1C8E1B8E212C682E712CFE
:107AE000A3014E535D4F3A0160726E8B5D895170F8
:107AF0005D876D896270562E3E2C8E2D0E94FA1580
:107B00006E2D65DF8C0173E07E1570F054E0959565
:107B100087955A95E1F7F701EE5CF74F8083F30103
:107B2000EE0DFF1D449001C04E2CC42CD12CC6017B
:107B3000880F991F9A878987FC01EC5DF74F1183A5
:107B40000083C80117FD0F9634E0959587953A9507
:107B5000E1F7282F87FD219522307CF481E090E029
:107B60000C2C01C0880F0A94EAF7211102C0982F4B
:107B700003C09091CB079823292A93E0931508F42A
:107B800073C0AD85A11158C08091570281FF54C0C8
:107B90005601AA0CBB1CF501E95BF94F5F0181811D
:107BA000807C09F449C080818595859585950E94E2
:107BB0002519882309F440C0809115028823E1F13A
:107BC000D501EC91E770F0E0DF01AA0FBB1FAC5DBF
:107BD000BE4FEE0FFF1FE15CF94F8D919C9120810C
:107BE0003181821B930B97FD0196AC01559547950A
:107BF000F5012181322F330F330F3595359534033D
:107C0000C001359F900D11246FE170E00E946074F7
:107C1000660F771F660F771F22952695269523708E
:107C2000213009F09DC6060F171FF2E04F1204C065
:107C30007C8F6B8F21E02D8F3E89332339F0F60145
:107C4000EE0FFF1FED53F84F11830083B801842D11
:107C5000B4DC8C01632D8091EA060E940913880F21
:107C6000991FD4018D939C93BE89BB2339F0F601F3
:107C7000EE0FFF1FE555F84F118300835520E1F00B
:107C8000E3E0E315C8F0F2E04F16B1F0065F1F4FD6
:107C90000531110538F0F601EE0FFF1FE555F84FDD
:107CA00011821082E1E0F0E0EC0FFD1F29853A859A
:107CB000E20FF31F118210823FEFE31AF30A42E052
:107CC000840E911C57E0E516F10409F015CF809160
:107CD0005C0280FF27C062E08091EA060E940913DF
:107CE000182F0E949610012F81110195202F332704
:107CF00027FD3095432F532F23583F4F4F4F5F4F52
:107D0000A0E0B4E08091AF079091B007A81BB90B39
:107D10000E941E7420E034E040E050E00E94957420
:107D20003E832D836E89662309F435C1109160026C
:107D300012218091CB078095812319F088E10E9460
:107D400005721093CB070BEA17E0D8018D0180E094
:107D500094E0FD0197878687918B808B4091630229
:107D6000442309F458C0A281B381E680F7809D01C5
:107D70000E94F9734B015C019701D7010E94F973CE
:107D8000860E971EA81EB91E842F0E940C187C0117
:107D90009C01DC010E94F973681579058A059B0531
:107DA000D0F580E1C82ED12C40E050E8E0E0F0E8CA
:107DB0009A01DA010E94FF7386169706A806B90693
:107DC00010F44E275F27F695E79521E0C21AD108F7
:107DD000C114D104E9F4F801228133814A01A12CB4
:107DE000B12CD7010E94F973A50194010E949574EA
:107DF000F8013383228326813781D7010E94F973EA
:107E0000A50194010E949574F8013783268303C06D
:107E10004E2B5F2BCDCF60916102862F807E09F4BF
:107E2000BAC051100EC0F801228133818B819C8130
:107E3000280F391F868197814F815885840F951FA0
:107E400004C080E090E020E030E0409162024423F2
:107E500079F04150E42FF0E0EE0FFF1F443118F4A9
:107E6000E00FF11F02C0E452F84F4081518102C07F
:107E700040E050E062FF03C031952195310963FF76
:107E800003C091958195910964FF03C05195419577
:107E90005109629566956770633009F463C0643078
:107EA00009F469C0623059F1BC0197FF02C0695FF3
:107EB0007F4FF3E075956795FA95E1F7DC01A61B16
:107EC000B70BBC0197FF02C061587F4F660F672F49
:107ED000661F770BA61BB70B97FF02C081509C4F04
:107EE000892F990F990B85958595A81BB90B7A0158
:107EF000E21AF30A37FF2CC02F5F3F4F29C0B901A8
:107F000037FF02C0695F7F4FF3E075956795FA957B
:107F1000E1F7D901A61BB70BB90137FF02C06158C1
:107F20007F4F660F672F661F770BA61BB70B37FFB8
:107F300002C021503C4F232F330F330B259525953D
:107F4000A21BB30B7A01E81AF90A97FD01969C016E
:107F500035952795240F351FB9016A0F7B1F2A1B02
:107F60003B0B12C07A01E21AF30A240F351FB90144
:107F7000680F791F07C07A01E21AF30ABA01680F85
:107F8000791F9A01281B390BF801F38AE28A758B55
:107F9000648B378B268BFF85FB8B2B852C8B45EADF
:107FA00053E05A8F498F1E861D86B5E62B2EB2E010
:107FB0003B2E1F8A198A5D8559A3B101665F7F4FE9
:107FC000788B6F87C12CD12C7601D1018C9190E0F8
:107FD0000197ED85FE858E179F0709F059C3EF8540
:107FE000F889389780810E94FF178A8B7F89672FD5
:107FF00070E07A8769876551794F5B01FB01E05634
:10800000FF4F908040E061E00F851889075011090B
:10801000D8018C910E942118F8019081992359F080
:10802000EF85F889399790819C50983020F4909191
:108030001502992399F0882391F0F10181858F71C0
:1080400090E00090EA0602C0959587950A94E2F7C1
:1080500081709927F1E08F27817001C080E02F8522
:1080600038892950310938A32F8FD9011C918111EA
:1080700031C0F501E056FF4F10821D32C9F4E98589
:10808000FA85EE0FFF1F29853A85E20FF31FE55DA4
:10809000F84FAFE8B2E0A70196010E941474BB2725
:1080A00097FDBA95A92F982F872F80839183A2835C
:1080B00088EF810F823008F0DEC2F101878186707F
:1080C000843009F4D8C280E0193009F0BCC000E067
:1080D0001CEFBDC081E0911080E0982E2FEF210FA2
:1080E0002C30B0F4822F90E0DC01AA0FBB1FA55505
:1080F000B84F0D911C91243008F091C0F1012781F7
:1081000026FF8DC0FC01EE0FFF1FED53F84F26C078
:108110002431C0F483EF810FE82FF0E0DF01AA0FD4
:10812000BB1FAC5DBE4F0D911C91843040F4EE0F2F
:10813000FF1FE15CF94F80819181081B190B000F33
:10814000111F6DC0243280F4F1018781E22FF0E02D
:10815000EE0FFF1F86FF05C0EE54F84F008111811E
:108160005EC0E452F84FFACF243281F5F1019185D7
:10817000929596959770B1F08EE0890F823128F034
:1081800081E1890F853149F01CC08131D1F4909192
:108190007F0692FF16C01FE106C090917F0694FDF6
:1081A000E4C30FC014E0812F0E943868811135C0EC
:1081B00081E0810F0E943868882361F100E010E0BF
:1081C0002EC00E94F867882341F124C02C3260F44D
:1081D000E22FF0E0EE0FFF1FE854FB4F0081F8E0C4
:1081E0000F02800111241BC02C3251F4C701B601CB
:1081F00024E630E040E050E00E94957489010FC011
:1082000040E050E060E070E082ED810F0E94652266
:108210008C0105C000E014E002C000E01CEFF10199
:108220008781982F907391F082958370815021E01F
:1082300030E002C0220F331F8A95E2F7C901398965
:10824000382B398B03C000E010E001C081E0E985E4
:10825000FA85E557F84F8083F101878183FD0EC0D1
:10826000EF85F88932978081882341F04DE763E8F4
:108270000E94E9170E940C18080F191FF101F681DE
:10828000FE8FF11105C0F1018581882309F421C118
:1082900080915C0283FF03C0F4E1F88F02C024E602
:1082A000288F49855A85440F551FDA01A551B94FCA
:1082B0003C91FD012181E985FA85E40FF51FE55D1B
:1082C000F84F80819181A281AC016A2F772767FDE9
:1082D00070952A013B01BB2777FDBA95A72F962FF2
:1082E000852FB801681B790BCB01AB01465F5F4F4F
:1082F0004531510550F0A32EB22EA114B10439F42A
:10830000F1012581211108C002C0A12CB12C9110CE
:1083100003C09C878B8737C0F101878186708430CA
:10832000D9F4E081F0E0EE0FFF1FEE5FF74FA08180
:10833000B18120E034E60E940E742B013C01FA89E1
:10834000FF2351F02F2F332727FD3095432F532F35
:108350000E94957429013A01BB2777FCBA95A72D95
:10836000962D852D9801281B390B3C872B872115CD
:10837000310549F0F101858137FF82958F70F88DC5
:10838000F89F500111241A141B04B4F480913C018D
:10839000882331F021E0A21AB108A114B10449F0F8
:1083A000332777FC3A95272D162D052D1C861B8625
:1083B00003C0AA24AA94BA2CE985FA85EE0FFF1F00
:1083C000E551F94FB182A0824B855C85452B09F4BC
:1083D00073C04801AA2497FCA094BA2C5E8D552343
:1083E00009F466C080913C01882309F440C06A8981
:1083F000662379F0262F27FD219530E040E050E0FC
:1084000060E070E080E293E00E949574CA01B901D7
:1084100004C060E070E080E293E0F10126814B85CA
:108420005C851416150644F09095809570956195BD
:108430007F4F8F4F9F4F22952F7030E021153105D0
:1084400091F0A88DA29FA001A39F500D11249A0125
:10845000442737FD4095542F0E949574420E531EB9
:10846000641E751E04C04424582C692C7A2CBB272A
:1084700077FCBA95A72D962D852DEB85FC851E16CC
:108480001F0634F488169906AA06BB0634F009C004
:1084900088159905AA05BB0524F44424582C692C99
:1084A0007A2C332777FC3A95272D162D052D04C0FD
:1084B0004424582C692C7A2CE985FA85EE0FFF1F8D
:1084C00029853A85E20FF31FE55DF84F408251821E
:1084D0006282F1018781EF85F889369787FF26C090
:1084E00080810E94FF17A82FBB27A7FDB0951A1601
:1084F0001B0644F417FF62C024E630E02A1B3B0B46
:10850000D90109C0109709F459C0101611060CF0D2
:1085100055C0AC59BF4F98010E94F97324E630E072
:1085200040E050E00E949574890148C060818BE171
:10853000860F873340F06058772767FD7095C80134
:108540000E94E42B34C0862F992787FD9095A92F90
:10855000B92F87309105F8F4FC01E758FF4F0C94D0
:10856000B17417FF2BC010C0101611066CF026C096
:1085700017FF24C011950195110920C0101611068E
:10858000C4F002C017FD18C000E010E017C01016BC
:1085900011067CF011C067FF06C011950195110905
:1085A00036E0361B632F6750C8010E948D3A8C015C
:1085B00005C000E014E002C000E01CEFF1014781BB
:1085C00040FD12C0AF8DB8A18C919FEF980F9430F1
:1085D00058F4FE013196E80FF11DE80FF11D3297B6
:1085E00080819181080F191F9801EA89AE2FBB275E
:1085F000A7FDB0950E94F9734B015C0143FF15C0C4
:10860000EF85F88932978081882379F04DE763E818
:108610000E94E9170E940C1824E630E0DC010E9459
:108620000E74860E971EA81EB91EF10187818695CD
:108630008370813039F08230E1F0C80CD91CEA1C1B
:10864000FB1C19C0C501B40124E630E040E050E055
:108650000E949574CA01B901A70196010E94247471
:1086600020E034E040E050E00E94957469017A0116
:1086700002C075016401FAE02F0E311C2F892F5FB3
:108680002F8B4F855889465F5F4F588B4F879DCC06
:108690001092360880919B06882309F441C08F010F
:1086A000000F111F000F111FF801E556F94F8784C5
:1086B0009088A188B288FE89FF2319F0812C912C23
:1086C0005401C701B60124E630E040E050E00E94CA
:1086D0009574E091EA06F0E0EE0FFF1FE556F94FC2
:1086E000A581B6810E941474680D791D8A1D9B1D99
:1086F000F801E556F94F6787708B818B928B2D8936
:1087000026FFF9C020919E0630919F0640E050E080
:108710000E949574A4E6B0E00E9414746B017C0181
:108720000D851E85000F111F0C5F174FC701B60185
:1087300024E630E040E050E00E949574D8012D938B
:108740003C93698C7A8CF3013F0183819481809002
:10875000FB04912C881699063CF091948194910821
:10876000881699060CF44C01F30121818401FAE08A
:108770002F02000D111D1124D3012C91F4014AE0A8
:108780002402E00DF11D11249F01285E33400851A1
:108790001C4F033E54E0150714F002EE14E04901AB
:1087A0002E316BEF360724F42EE1822E2BEF922E22
:1087B000302F212F8017910714F4382F292FA32E43
:1087C000B22EA814B9040CF45401C114D104E1046C
:1087D000F104A9F0F7FE04C0D501A819B90903C036
:1087E000D801AA19BB09A70196010E941E7420EAAC
:1087F00036E841E050E00E94957469017A01C501B4
:108800000E94D3175C01AC0CBD1CC8010E94D31799
:108810008A159B050CF45C01C4010E94D317A816AD
:10882000B9060CF45C01F3018281882319F0B1943C
:10883000A194B1089091C7049F7180E1891BF9A1AF
:10884000F81708F052C00D851E85000F111F085340
:108850001B4FD8018D018C91982F9F7309F445C04F
:10886000982F907C903409F440C09038F1F1880F33
:10887000880F859585950E942519F8019081907C37
:10888000903C39F5882319F01092CB081BC09091C9
:10889000BC05209128083091290895FF06C02D5E5F
:1088A0003F4F2732310520F00DC024313C4F54F4A6
:1088B000AD8DAA2309F45BC02B8D3C8D24313C4F38
:1088C0000CF455C09091CB08911101C081E08093C8
:1088D0003608882351F0ED85FE85EE0FFF1FE75324
:1088E000FB4F80810E940C185C01F894AB89BC8915
:1088F000AD92BC927894ED85FE853196FE87ED872A
:108900002B893C892E5F3F4F3C8B2B8B498D5A8D99
:108910004B5F5F4F5A8F498F709709F04CCB109186
:10892000580D798970FF05C0111103C08EE10E94B6
:108930000572898981FF07C0812F877F803419F4F0
:108940008FE10E940572998992FF15C0812F877F60
:10895000803811F0103979F480E20E9405720BC062
:10896000223009F062C98B0160C915E21CCC91E08C
:108970009093CB08A7CFA1960FB6F894DEBF0FBE99
:10898000CDBFDF91CF911F910F91FF90EF90DF90BE
:10899000CF90BF90AF909F908F907F906F905F909F
:1089A0004F903F902F900895FF920F931F93CF9376
:1089B000DF930E946A1A182F8093EA0663E68EE519
:1089C00098E061D861E68EE798E05DD8CEE5D8E022
:1089D000E7EAF3E021813281499159918E8D9F8D93
:1089E000481B590B8081811103C051954195510954
:1089F000240F351F293E83E038073CF428318CEFE3
:108A000038072CF428E13CEF02C028EE33E0328333
:108A10002183359628E0CE37D207E1F600E0023018
:108A200071F40F5F0430D9F786E00E94315D81E078
:108A3000DF91CF911F910F91FF900C940572602FE1
:108A4000812F0E940913EC01F12C602F8F2D0E94C1
:108A5000C912853F21E092073CF4AC014C1B5D0B31
:108A6000602F8F2D0E941D13F39484E0F812EDCF38
:108A7000D8CF8F929F92AF92BF92CF92DF92EF9218
:108A8000FF920F931F93CF93DF9390914F06292F5F
:108A90002F70F22E1092560120915A082111A5C074
:108AA0009077813809F48BC088F4843209F441C08E
:108AB00038F4823209F462C0833209F452C095C09E
:108AC000853209F440C0803809F18FC0843841F103
:108AD00060F4823809F460C0833809F086C087EA00
:108AE00090E30E947A1983E85CC08E3879F08F3B5E
:108AF00009F46DC0853809F078C081E08093FE07E5
:108B00008EE693E30E947A1985E828C092E090935C
:108B10005A0810925B080E94C36810920B0265C04D
:108B200081E08093FE078AE49AE20E947A1984E841
:108B300015C042E0F41259C08091E1088F5F833084
:108B400054F080E008C052E0F5124FC08091E10877
:108B5000815087FD82E08093E10847C00E94C3688E
:108B600044C0F39483E08F1508F4F12C9F2990936F
:108B70004F0681EA0E94315D83E126C0FF2011F09B
:108B8000FA9402C0E3E0FE2E9F2990934F0681EAFB
:108B90000E94315D84E118C087EA90E30E947A194F
:108BA00082E8DF91CF911F910F91FF90EF90DF90BE
:108BB000CF90BF90AF909F908F900C94C3680E940D
:108BC0005E310E94643187E10E9405720EC081E02F
:108BD0000E94C36883E00E94C36882E00E94C36869
:108BE00081E08093CD081092E10880915F020E949D
:108BF0002519C82F882329F08091CD08811101C043
:108C0000D3DEC093CD0890913D0180913C0698172A
:108C100010F4C6E001C0C4E080E00E9433334C2F62
:108C2000406860E185E20E941D6646E568E186E2F3
:108C30000E949B6324E040E060E18FE50E94822374
:108C400020E040E068E183E30E94D4110E946A1AA8
:108C5000882379F0482F60E186E20E94D52D29E033
:108C600046E26FE085E20E949F66D0E07FE1E72E5A
:108C70003EC000E020915D024BE250E160E186E2FF
:108C80000E94C16380915C0280FFEFCF47E250E118
:108C900060E188E30E940E64E8CF559547955595AD
:108CA00047954423B9F1443E0CF444EE142F4D3162
:108CB0000CF01CE18FEF8D0F46E3823008F040C0CE
:108CC00064E08C2F0E94AE64D13069F180915C0227
:108CD00080FF29C06E2D611B635027E047E08DEFB8
:108CE0008C0F0E947F66DF5FD43009F43DC08D2F6A
:108CF0000E947510E82FF0E0EE5DFF4EC4916D2FDD
:108D00008091EA060E940913AC0197FFC6CF4D5F20
:108D10005F4FC3CF1816190614F441E0C4CF492F92
:108D2000440F440BC0CF43E06EE18FEF8C0F0E94E5
:108D3000AE6443E06EE181E08C0F0E94AE64CACF66
:108D40006BE385EE8C0F0E94AC640FEF0C0F43E0D9
:108D50006AE3802F0E94AC6443E06CE3802F0E94A2
:108D6000AC64C10F6BE3B8CF91E09F1508F489C0E4
:108D70000AED17E0E12C29E1D22E3BE1C32EF801E8
:108D8000C191D1918F018E2D8370F1E0FF1639F1E1
:108D90008C9D802D112423E02E1510F068E201C077
:108DA00060E39E01D7FF02C0215E3F4F95E03595FD
:108DB00027959A95E1F7AE01421B530B9A01D7FF15
:108DC00002C0C158DF4FAE01440F452F441F550B61
:108DD000420F531F20E28F5D0E94FB654DC053E0A0
:108DE0005E1518F0A2E2AA2E02C0FEE5AF2EB82E44
:108DF000BB0CBB0CB80EE6E28E2E8B0C8091610290
:108E000081FF03C060E075E002C060E074E0AE0185
:108E1000D7FF04C0442755274C1B5D0BD49EF0019F
:108E2000D59EF00D1124CF019E5F0E946074962E96
:108E300089E1861714F479E1972E25E543E3682D3F
:108E400087EE8A0D0E94716445E064E26B0D8A2D05
:108E50000E94AE641C161D0614F4A39401C0A91848
:108E600067E26B0D492D8A2D0E94AC646B2D6B5D02
:108E7000492D8A2D0E94AC64E39498E0E9127FCFDB
:108E800027C0E2E0FE1218C00E94F3276091E108BB
:108E9000C1E0C60F662329F0862F880F680F660F82
:108EA0006D5F8AE00E947A3A6C2F660F6C0F660F36
:108EB00084E60E947A3A0CC024E041E068E289E34B
:108EC0000E94822320E840E060E38FE00E94D411FA
:108ED00080915A08882399F14EE06FE18EE495E184
:108EE0000E94B52910925908813049F590915C088B
:108EF000911103C08AE49AE220C0913039F4909332
:108F0000FE071092380888EA90E517C0923061F4A5
:108F100080935908E0914A01F0E0EE0FFF1FE35BF8
:108F2000FE4F8081918109C0933019F48EE693E35E
:108F300004C0943021F487EA90E30E947A19DF910B
:108F4000CF911F910F91FF90EF90DF90CF90BF9046
:108F5000AF909F908F900895AF92BF92CF92DF9283
:108F6000EF92FF920F931F93CF93DF936C01162F15
:108F7000CBE9D6E00E946A1AF82E4091CC088417FB
:108F8000E1F1442361F0EFEFE40F8AE0E89FF001A4
:108F90001124E75EFA4F808182958F7001C080E0D6
:108FA000FF2061F0EFEFEF0D9AE0E99FF00111244F
:108FB000E75EFA4F90819F70891718F08823D9F0E7
:108FC00001C0892F682F70E080E092E00E946074F9
:108FD0007A83698381E090E09C01042E01C0220F16
:108FE0000A94EAF73881322B0F2C01C0880F0A94BB
:108FF000EAF7382B3883F092CC081062E12E888192
:10900000882329F11C821B828E01B12CAA24A394EF
:1090100088818A21A1F0BF1491F0B092EA068B8179
:109020009C81F80125813681820F931F9C838B835D
:109030006E2DC6010E94433DFE2DFF7DEF2EAA0C32
:10904000B3940E5F1F4F85E0B812E2CF09C0FE0156
:10905000EF0DF11DEF0DF11D80E094E69683858301
:10906000FE01EF0DF11DEF0DF11D8B819C8125811E
:109070003681820F931F9C838B83F092EA066E2DBC
:109080006064C6010E94433D8881882309F43EC084
:1090900080913C018823D1F1FE01B0E0A1E080E0A5
:1090A00094E62581368118814A2F412331F10091C0
:1090B0003C0169817A81069FA001079F500D112410
:1090C000BF1559F04217530718F4241B350B17C06E
:1090D0002A2F20952123288310C0BC01621B730B0B
:1090E0004617570718F4240F351F09C02A2F20955B
:1090F0002123288320E034E602C020E030E03683DC
:109100002583AA0FBF5F3296B53059F6DF91CF9114
:109110001F910F91FF90EF90DF90CF90BF90AF9095
:1091200008950F939CEF940F9D3138F450E0425016
:1091300051098E5E0F910C94FB65413208F04D5140
:10914000022F242F4CEC55E10E94C1630F9108952A
:10915000CF92DF92EF92FF920F931F93CF93DF9303
:10916000C82E86E39DE00E94DF244091E90850E08C
:109170004F5F5F4F60E08EE40E942966C091E9086E
:1091800089E0C89FE0011124CC53DA4F8C818770AD
:1091900011F04AE001C049E06C2D89EC98E00E9492
:1091A00063251091C90816301CF46DE07DE002C003
:1091B00068EE7CE088E00E94F863F090FC071630CF
:1091C0000CF0ACC00E943828111107C06EE28881F3
:1091D0000E94211488832F2D01C020E0488168E07F
:1091E00080E60E94A01088818823D9F081500E94D7
:1091F00024126C0163EE7CE088E00E94F8634881F1
:10920000453250F0455202E0E02E00E0960168E061
:1092100088E40E94902305C0A60168E088E40E94CB
:109220002966113039F466E089810E94211489830E
:109230000F2D01C000E02981253018F442EE55E1E0
:1092400003C0255043ED5CE060E18EE40E94C16301
:10925000123081F484E680933E0122E040E05DE735
:1092600060E073E88D819E810E944F139E838D8301
:109270002F2D01C020E048818D819E81453250F024
:109280004552B2E8EB2E022F9C0168E188E70E946C
:10929000902305C0AC0168E188E70E94FB651330AC
:1092A00051F440915701642F61958A810E941E14E8
:1092B0008A832F2D01C020E04A8160E280E60E946F
:1092C0008411143031F461E28B810E9421148B836C
:1092D00001C0F12C2F2D4B8168E280E622DF21E0D6
:1092E000153009F020E04C8146954695469543702F
:1092F00063EB7CE080E30E94F2248370880F880F88
:10930000880F9C81977E982B9C83DF91CF911F9132
:109310000F91FF90EF90DF90CF90089521E01630ED
:1093200009F020E04C814295469543706DE97CE060
:1093300088E00E94F22483708295880F807E9C8151
:109340009F79982B9C8321E0173009F020E04C8115
:1093500047FB442740F961E97CE080E10E94F22468
:109360004C8180FB47F94C83042F077021E01830B3
:1093700009F020E0402F6BE77CE088E10E94F224B6
:1093800087709C81987F982B9C83801711F018869A
:109390001F828C81877009F466C060E77CE080E200
:1093A0000E94F8638C818770813009F041C01930C8
:1093B00069F422E04FEF51E060E070E08F81988522
:1093C0000E944F1398878F830F2D01C000E04F81BB
:1093D00058854C3FE1E05E077CF0202F42EC54E1E1
:1093E00060E28CE60E94D3634F814B5C202F60E2E9
:1093F00088E70E94106333C0453FF1E05F073CF00F
:10940000445F202F60E28CE60E944B2428C0202F6E
:1094100060E288E70E94FB65002309F180E8C8123A
:1094200004C08F8198850E9461141092020817C0B1
:109430008230A9F4193059F44FE060E08F810E9426
:109440001E14482F50E058874F830F2D01C000E0B5
:109450002F8149E556E160E28AE50E94C163AAE0F6
:10946000DA2E08E203C0F9E0DF2E00E269E67CE0D4
:10947000802F0E94F8634D2D50E0E12FFF27E7FD7C
:10948000F095E417F50781F4E0E8CE120EC089E00C
:10949000FE0111928A95E9F7109202081A3029F418
:1094A00088E08093C90801C0F12C2F2D4FE55CE0C6
:1094B000602F88E4DF91CF911F910F91FF90EF9083
:1094C000DF90CF900C94D363CF93C62F20E04EE172
:1094D000682F80E00E94346480910B02803831F460
:1094E000C0938F0D8BE191E20E947A1910920208CD
:1094F000CF9108951F93CF93DF93D82F162F23700A
:1095000021F0223021F4C1E803C0C0E801C0CDE25F
:10951000612F8D2F0E949B634C2F612F86E08D0F52
:10952000DF91CF911F910C949B6390910308282F9A
:10953000291B181644F4273014F0865005C027FD67
:1095400003C0892F01C080E0809303080895CF9263
:10955000DF92EF92FF920F931F93CF93DF93C82F69
:1095600087E295E10E94DF244FE06C2F8DED98E0BB
:109570000E946325F090DD088F2DD7DFD82EC036EE
:1095800021F0C43611F0CE3269F4F7FC0BC0F09232
:10959000E7088C2F0E94C36810920B028AE09CE3BC
:1095A0000E947A1988E0E82E0F2D112707FD1095EB
:1095B000CD2DD0E0CC24C3940C171D0709F0C12C8D
:1095C0002C2D4BE353E16E2D80E00E94D363AE015E
:1095D0004F5F5F4F88E08D1510F486E101C081E197
:1095E0002C2D6E2D0E94FB6588E0E80ED39480E45C
:1095F000E812DECFF7FC05C0F092E70884E60E948F
:10960000AF3BDF91CF911F910F91FF90EF90DF90D3
:10961000CF9008956F927F928F929F92AF92BF9258
:10962000EF920F931F93CF93DF9348E0682F8CED59
:1096300098E00E94632562EC74E180E00E94F86388
:10964000C091E90841E34C0F60E08CE00E949B630D
:10965000A090DC088A2D69DF782E45E24C0F92E05D
:10966000E92E00E020E030E060E080E30E949023FB
:109670004091030867EF72E188E00E94FD6318E003
:10968000BB24A7FCB0948BE0C89FE0011124C25713
:10969000DA4F4E01E7E08E0E911C23E0622E472D3B
:1096A00050E0A416B50619F40091FC0701C000E0D3
:1096B000872D90E08930910508F093C080589F4F26
:1096C000FC010C94B174202F4881612F82E40E9428
:1096D000A010002309F485C06EE288810E94211445
:1096E00088837FC001116092E80824E0A401612F03
:1096F0008091D9070E94712C74C049815A81202F12
:10970000612F8EE40E94FB65002309F46AC022E009
:1097100040E05DE760E073E889819A810E944F1321
:109720009A8389835EC0402F6B81812F0E945C28C1
:109730008B8357C0402F6C81812F0E945C288C83C3
:1097400050C0002329F067E08D810E9421148D8391
:109750002D8148EC54E1612F88E40E94C16341C02F
:10976000002349F08E8161E081700E9421149E8166
:1097700080FB90F99E838E8180FF02C04DE201C084
:109780004BE2202F612F88E40E9410632AC000233F
:1097900061F08E81869562E083700E94211483704F
:1097A000880F9E81997F982B9E834E8146954370AA
:1097B00050E0202F612F84E50E94FB6512C021E05C
:1097C000A416B50609F020E04E8143FB442740F97A
:1097D00069EE72E1812F0E94F2249E8180FB93F951
:1097E0009E837394185F103409F059CFDF91CF91A5
:1097F0001F910F91EF90BF90AF909F908F907F90AF
:109800006F9008956F927F928F929F92AF92BF92C6
:10981000CF92DF92EF92FF920F931F93CF93DF933C
:10982000C82E8091E5080E948F10EC014FE06C2D4E
:109830008AED98E00E94632589EB92E10E94DF2483
:1098400020E0488160E08A5F0E94CE10A090DA0894
:109850008A2D6BDED82E4091030863E372E188E025
:109860000E94FD6338E0F32EBB24B39444E0942EB1
:1098700050E8852EAD1003C0E090FC0701C0E12C3C
:109880000D2D10E00031110508F097C1F801E757E0
:10989000FF4F0C94B17419812E2DAE016F2D84E50C
:1098A0000E94CE28153231F419851295169517703D
:1098B0001B5D03C0163208F01A5FEE2009F47DC16B
:1098C00047E361E0812F0E941E14853268F08C32DC
:1098D00010F0865009C085528295880F807E998548
:1098E0009F71982B998785E2898367C12E2D4A81C4
:1098F0006F2D80E60E94A9248A835FC12E2D4885A2
:109900006F2D80E60E94A924888757C18F814E2D34
:109910006F2D83FB882780F90E9424259F8180FB7F
:1099200093F909C199818F81953080F486FB88274E
:1099300080F94E2D6F2D9B2D981B892F0E94242579
:109940009B2D981B8F8190FB86F91FC086FB1127EA
:1099500010F964E272E18F2D0E94F8634E2D6F2D95
:10996000812F0E9424259F8180FB96F9E4C08F817E
:1099700081704E2D6F2D9B2D981B892F0E942425C1
:109980009B2D981B8F8190FB80F98F8316C18F814F
:1099900087FD08C08C81855E863340F410E042E18B
:1099A00052E107C011E048E152E103C012E04EE18C
:1099B00052E12E2D6F2D86E00E94D363EE2009F434
:1099C000FCC062E0812F0E942114181709F4F5C031
:1099D000823011F48C8201C01C829F8180FB97F938
:1099E000AAC08F8187FF09C004E62CE94C816F2D46
:1099F00088E40E9463248C83E0C04C818BE1840F57
:109A00008733B8F010E8140F2E2D2064412F55270E
:109A100047FD50956F2D86E60E94FB65EE2031F0E4
:109A200044E66CE9812F0E941E14182F10581C83E5
:109A3000C4C02E2D6F2D8CE00E943E28EE2009F42C
:109A4000BCC046E160EF8C810E941E148C8390E6BE
:109A5000C912B3C087303CF087508093E7088AE092
:109A60009CE30E947A198C8187FFA7C08095809320
:109A7000E7088AE09CE30E947A199FC001E0E110A8
:109A800001C000E02E2D4B816F2D8EE40E947928BD
:109A90008B8393C0E1109092E8080FE310E07724E5
:109AA000739466246A946F0C99859F71972121E0C5
:109AB00009F020E040E3410F6F2D802F0E941063DA
:109AC000EE20E9F08091D907811319C029E048E020
:109AD000662D8FEF800F0E949F6680E2C81619F0F6
:109AE0009EE2C9120CC08985972D98279F71807EB0
:109AF000892B898782E00E94315D10920208770CE1
:109B00001F5F095F153081F658C01F8112951370D1
:109B10002E2D412F6F2D8EE40E945925EE2009F441
:109B20004CC063E0812F0E94211483708295807F56
:109B30009F819F7C982B9F8340C021E08BE0A812DF
:109B400020E04F814695437066EF71E18F2D0E94B2
:109B5000F2248370880F9F81997FECCF4D814295CD
:109B60004F706E2D8F2D0E948B218295807F9D815D
:109B70009F7009C04D814F706E2D8F2D0E948B21DB
:109B80008F709D81907F982B9D8317C04E81429549
:109B90004F706E2D8F2D0E948B218295807F9E812C
:109BA0009F7009C04E814F706E2D8F2D0E948B21AA
:109BB0008F709E81907F982B9E83D39498E0F90EAE
:109BC00080E4F81257CEDF91CF911F910F91FF9053
:109BD000EF90DF90CF90BF90AF909F908F907F904D
:109BE0006F9008952F923F924F925F926F927F9263
:109BF0008F929F92AF92BF92CF92DF92EF92FF929D
:109C00000F931F93CF93DF93A82E87E791E10E94D4
:109C1000DF248091D507882301F10E94D324882373
:109C200031F01CF072E6A72E02C063E6A62E20914A
:109C3000D908211103C083E6A81661F030E08091B5
:109C4000D707992787FD90952817390721F4E2E671
:109C5000AE1201C0A12CA0920B0280915A08811172
:109C600007C04091D7076A2D89ED98E00E946325CF
:109C70006090D90880910B02803641F08F3B19F03B
:109C80008E32D1F403C01092D50716C09091D5073B
:109C9000992339F01092D5071092020810923808D3
:109CA0000BC090915A08911107C00E94C36810928E
:109CB0000B028824839401C0812C862D36DC582E1B
:109CC00080915A08811110920B028091D507882348
:109CD000E1F080910B029EE9980F9230B0F401E020
:109CE000823609F000E01091E508812F0E948F1064
:109CF000EC01111175C101117DC18881823010F014
:109D00008150888382E00E94315D77247394B12C66
:109D1000912CC52CD12C892D0E948F10EC01B514EB
:109D200088F06B2D70E06C197D096730710554F473
:109D30006F5F7F4F660F660F660F20E0472D81E053
:109D40000E94CE10FFE1F91508F4B8C02880271052
:109D5000B5C02A96492C7E018AE0E81AF108B514AC
:109D600008F49FC08B2D90E08C199D0987309105D8
:109D70000CF088C00196382E330C330C330C8091D4
:109D8000D507811112C06B1010C04092E5082092D7
:109D9000E308882031F010925B08E1E0E0935A0874
:109DA000A12C11E080915A08811110E0941459F00F
:109DB000F70127812695237000E042E751E1632DEA
:109DC00083E10E94C16320E0A701632D80E30E942C
:109DD000CE28212F8E0108501109F8014081632DF2
:109DE0008DE20E94A924F8018083FE01379740810B
:109DF000442329F020E0632D88E40E948411FE01B1
:109E0000369740814423B1F0F701878187FF03C073
:109E100020E044E60BC08BE1840F20E0873328F478
:109E2000632D80E60E943E2805C045E4632D80E650
:109E30000E941063F7018681811102C040E201C0D7
:109E400043E5F7018581882329F0433511F44AE27F
:109E500001C044E4632D89E70E949B638091D5078C
:109E60008823F9F08091E40884111BC020E046E6C5
:109E7000632D88E10E9434644092E508B092D908CD
:109E80006B2C0FC0079769F48091D507882349F0A0
:109E90008091E408841105C08091D9088F5F809378
:109EA000D908B3944394F0E24F1669F12A96FE0163
:109EB0003A978081821509F44ECF25C06B1021C0DE
:109EC0007092E3089092E5086B2D6C19660F660F8F
:109ED000660F695F29E049E180E00E949F66882063
:109EE00081F00E94FA2881110CC060E08091E508A1
:109EF0000E94AA211092D50782E09CE40E947A1960
:109F000008C0B394492C739481E1781611F0942C15
:109F100002CF80915A08882309F44CC0A0920B020A
:109F20004BE06FE382E394E10E94B52990915C08D5
:109F30008130D1F5913079F40E94FA2881110DC059
:109F40008091E5088F5F8093E50860E00E94AA2178
:109F50001092D50702C0923018F482E09CE40EC043
:109F6000943079F48091E5088093D60780910B02B4
:109F70000E94C36810920B028EE299E20E947A1945
:109F800011C0953011F48FEFEFCF923041F48091F2
:109F9000E5088F5F8093E50861E00E94AA2181E0D7
:109FA0008093D50710925A088091E5088093E408C1
:109FB00010920208BA94B092D707DF91CF911F9107
:109FC0000F91FF90EF90DF90CF90BF90AF909F9058
:109FD0008F907F906F905F904F903F902F9008955B
:109FE000113208F092CE103219F4002329F08DCEF0
:109FF000002311F01F5F01C01150812F0E948F10AC
:10A00000FC0198818FEF890F803108F07ECE20818E
:10A01000213108F07ACE291302C08BE009C0002359
:10A0200009F46FCE903108F06DCE9F5F98836ACEB1
:10A03000815029F09081288121939993F9CF109331
:10A04000E40860CE9F92AF92BF92CF92DF92EF92E0
:10A05000FF920F931F93CF93DF93D82F89E59CE056
:10A060000E94DF2447E06D2F88EC98E00E94632572
:10A07000C091C8088C2F59DAA82EDE3211F0D036E4
:10A0800059F4C8304CF4C093E9088D2F0E94C3687E
:10A0900088EA98E40E947A19E8E0BE2ECC2EDD24EE
:10A0A000C7FCD094F9E09F2EEA2CF12C9E9CE00195
:10A0B0009F9CD00D1124CC53DA4FA7014F5F5F4F07
:10A0C00006E51CE020E06B2D81E10E94E52420E004
:10A0D00048816B2D8EE10E94A01020E04A816B2DFB
:10A0E00086E30E94841120E04B816B2D8EE419D809
:10A0F0009C819770913021F0923039F441E401C095
:10A1000043E26B2D82E70E949B638C81887129F06A
:10A1100048E46B2D88E70E949B63CE14DF0431F482
:10A1200020E048E76B2D80E00E94346488E0B80EA0
:10A13000A39480E4B812B8CFDF91CF911F910F9113
:10A14000FF90EF90DF90CF90BF90AF909F900895D9
:10A150003F924F925F926F927F928F929F92AF92B7
:10A16000BF92CF92DF92EF92FF920F931F93CF9304
:10A17000DF9392E09093FB0746E067EC78E00E9463
:10A180003C21E82E4091EA084150682F87EC98E086
:10A190000E94632580915708863091F038F4813011
:10A1A00061F08530A1F489EE9DE20FC0893059F04D
:10A1B0008A3069F482E290E508C082EF9DE405C030
:10A1C00087EA9AE402C080EF96E20E947A19F09042
:10A1D000C708C091FC070091570810E00E30110528
:10A1E00010F00C94C45BF801E756FF4F0C94B17467
:10A1F0008BE595E10E94DF248DE08093EA0841E041
:10A200004F0D66E08CE39CE00E94E8210C94C45B57
:10A210008CEC93E10E94DF242AE02F1510F00E94BD
:10A22000382880E18093EA0885E08F1508F4E6C0BD
:10A23000F11003C089E08093E80801E0F11000E02C
:10A240002AE04BE452E068E08091D9070E94712C2B
:10A2500091E0F91210C0E0E6EE1204C080915502C0
:10A260000E94771461E3809155020E94211480932B
:10A2700055022C2F01C020E04091550250E04C5F68
:10A280005E4F0BE21CE060E188E50E94E52466EF8A
:10A290007BE088E10E94F86311E0D0E080917F06C6
:10A2A00082FF20C08EEF8D0F8430E0F44091FA04DD
:10A2B000D23051F4242F30E03595279535952795E8
:10A2C00045E468E18EE40CC0D43071F4242F30E012
:10A2D00094E0359527959A95E1F749E468E18AE598
:10A2E00009D902C081E001C080E090917F0694FF0F
:10A2F0000CC0D63039F420910C0641E468E186E6C2
:10A30000F9D818C0D73009F4D8E0882399F08091A3
:10A31000FA04812301E009F400E04D2F50E04F538F
:10A32000594E8D2F880F8D0F880F21E068E18E5BCD
:10A330000E949D63110FDF5FD83008F4AFCFF2E0C9
:10A34000FF121DC029E048E367E181E40E949F6697
:10A3500020E6E21619F08EE2E81211C08E2D0E945E
:10A36000C3680E94A1128093FA0485E20E94A26849
:10A3700080930C061092020882E00E94315D41E059
:10A3800093E0F91240E08091BC0560E28295817013
:10A390000E9424259091BC0580FB94F99093BC0504
:10A3A000E4E0FE1209C0C06264E68091FB040E94F2
:10A3B00021148093FB0401C0C0E24091FB0450E0F3
:10A3C0002C2F68E288E70E94FB6521E0F5E0FF1290
:10A3D00020E04091C7044295469547706AED7BE0C6
:10A3E00080E30E94F2248295880F807E9091C704BA
:10A3F0009F71982B9093C7040C94C45B2AE02F158F
:10A4000008F487C063E97BE088E00E94F86341E0DC
:10A4100086E0F81240E08091610268E086958170E4
:10A420000E9424259091610280FB91F99093610232
:10A4300091FF1BC0C091BC05C5FBCC27C0F921E032
:10A4400097E0F91220E04C2F63E87BE080E10E9466
:10A45000F22481709091BC0580FB95F99093BC0526
:10A460008C1791F00E948F190FC0E5EAF3E080810C
:10A4700087FD1082818118160CF41182359623E035
:10A48000E53FF207A0F3D6CFC091BC05C6FBCC27B1
:10A49000C0F941E088E0F81240E068E18C2F0E94AA
:10A4A000242581709091BC0580FB96F99093BC05A2
:10A4B0008C130E948F190E949610882311F041E896
:10A4C00001C040E860E280E60E949B6341E099E0C1
:10A4D000F91240E080915C0268E281700E942425BC
:10A4E00090915C0280FB90F990935C0241E0EAE07D
:10A4F000FE1240E080915C0260E3829581700E94D0
:10A50000242590915C0280FB94F990935C020C945A
:10A51000C45B6FE47BE088E00E94F86321E0FBE02D
:10A52000FF1220E040915D026DE27BE088E00E9436
:10A53000F22480935D022CE0F21204C001E0C1110C
:10A5400003C001C0C0E000E02C2F40915F0260E139
:10A5500086E60E94792880935F0241E08DE0F81240
:10A5600040E080915C0268E183FB882780F90E94CB
:10A57000242590915C0280FB93F990935C0241E06A
:10A580009EE0F91240E08091570260E2869581706A
:10A590000E9424259091570280FB91F990935702D5
:10A5A000D5E2CD2EDBE0DD2EE6011FE301E086E003
:10A5B000B82EAC2EAC18FE0144918091600280232D
:10A5C00021E009F420E068E2812F0E941063FFE09F
:10A5D000FF121DC0B092E8088091D9078A1117C0F8
:10A5E00029E048E067E28FEF810F0E949F6620E23A
:10A5F000E21619F08EE2E8120AC08091600280270C
:10A600008093600282E00E94315D10920208000F88
:10A610002196195F103769F60C94C45B8BEB96E1B9
:10A620000E94DF248AE08093EA0894E09F1528F0D6
:10A630000E943828E12C10E003C0EE24E39415E0DA
:10A64000E5E0EE9EE0011124C050DE4FD090FC0703
:10A6500061E778E088E00E94F86341E34E0D68E02E
:10A660008EE10E949B63F11202C02D2D01C020E0FB
:10A6700048815981022F68E087E40E943966F1120F
:10A6800014C08CE380933E014CE364EC80E00E94B4
:10A690001E1448815981480F511D87FD5A955983D1
:10A6A000488357FF02C01982188281E0810FF81297
:10A6B00007C063E18A810E9421148A8341E001C0BE
:10A6C00040E0E11002C021E001C021E860E18CE33C
:10A6D0000E94D41182E0810FF81205C0DD2019F02C
:10A6E0002D2D03E002C020E002E04B8168E18AE505
:10A6F0000E9479288B8321E083E0810FF81220E00B
:10A700004C8169E578E080E20E94F2248C831C5F32
:10A71000F112D12CE11003C04091BA0502C0409162
:10A72000BB05DD2011F003E001C002E02D2D68E241
:10A730008FE40E947928E11003C08093BA0502C01B
:10A740008093BB05E0E0F2E0808191819093590213
:10A750008093580282818093560283818093C6043D
:10A7600080915702948190FB80F9809357028581F4
:10A7700096819093F7048093F60487818093F80480
:10A7800080858093F9048091BC05918590FB87F9C1
:10A790008093BC05F9C78CE395E10E94DF2486E035
:10A7A0008093EA08C091FC076AED7AE088E00E9495
:10A7B000F86321E0F11020E0409161024295469556
:10A7C000477062EC7AE088E00E94F2248295880F5C
:10A7D000807E909161029F71982B90936102F1E0CD
:10A7E000FF1209C064E2809162020E9421148093EA
:10A7F00062022C2F01C020E04091620260E186E6F7
:10A800000E94A01022E0F21208C064E68091630268
:10A810000E9421148093630201C0C0E02C2F40915C
:10A82000630268E184E50E94592541E083E0F81263
:10A8300040E08091610260E282FB882780F90E94FB
:10A8400043259091610280FB92F99093610241E06F
:10A8500094E0F91240E08091610268E283FB88276E
:10A8600080F90E9443259091610280FB93F99093B7
:10A87000610241E0E5E0FE1240E08091610260E3A8
:10A88000829581700E9443259091610280FB94F92A
:10A890009093610279C784E395E10E94DF2485E00B
:10A8A0008093EA0810925601D091E60820E0F1105A
:10A8B00009C043E060E08D2F0E941414D82F8093CC
:10A8C000E60821E041E04D0F68E080E00E94A01022
:10A8D0008D2F0E94B224182F00E0282F46EB5AE05B
:10A8E00068E08AE20E94C16366E97AE088E00E943B
:10A8F000F863ED2FF0E0EE0FFF1FEC5DF74F4081A6
:10A900005181453651052CF44C395F4F24F0C2E09B
:10A9100003C0C0E001C0C1E08D2F0E940218811168
:10A9200006C0CC2329F081E0F81202C002C0C0E0CA
:10A9300080E0EE24E39400E0212F48E168E10E94EA
:10A94000112CC13011F081E0F81280E0E12C00E020
:10A95000212F48E160E30E94112CCC2319F081E003
:10A9600022E0F21280E0EE24E39401E0212F48E29D
:10A9700068E10E94112CC13019F081E092E0F912D7
:10A9800080E0E12C01E0212F48E260E30E94112CDD
:10A9900081E0E3E0FE1280E0E12C00E023E640E30A
:10A9A0006EE10E94112C81E0F4E0FF1280E0E12CC6
:10A9B00000E022E648E36EE10E94112C8091E60857
:10A9C0000E940218882311F08CE301C08CE540E45A
:10A9D00060E00E94AE6481E08093440961E08CE510
:10A9E0000E94513B8091E608E82FF0E0EE0FFF1F38
:10A9F000EC5DF74FC081D181BE010E94DD3A8C0130
:10AA000089E18C9F90018D9F300D112437FF02C08A
:10AA100021503F4F532F550F550B432F60E382E7D3
:10AA20000E94296689E1809F9001819F300D112449
:10AA300037FF02C021503F4F532F550F550B432F67
:10AA400068E084E50E942966CE01409697FF02C027
:10AA5000CE018F967C01A5E0F594E794AA95E1F7E5
:10AA6000E8016096D7FF02C0E801AF96F5E0D59502
:10AA7000C795FA95E1F7D195C195D1096C2F635E21
:10AA800047E08CE58E0D0E94AE646C2F605E47E05F
:10AA900089E58E0D0E94AC641092440975C6E09061
:10AAA0005A022E2D2F70E22ED22E81E0281741F06F
:10AAB00092E0291739F0E5E02E1731F0C4E005C027
:10AAC000C6E003C0C3E001C0C7E088E095E10E9492
:10AAD000DF24C093EA08D091FC07C091D90767E84A
:10AAE0007AE088E00E94F863F11013C080915C0264
:10AAF00067E08295869587700E9421148295880F61
:10AB0000807E90915C029F71982B90935C0221E073
:10AB100001C020E040915C024295469547704F5C31
:10AB200068E082E70E941063EE2049F08DE08E0D10
:10AB30008F70CC24C394823020F0C12C02C0CC246E
:10AB4000C394F1E0FF1202C0CC2311F000E001C079
:10AB50000D2F2E2D4BE55AE060E184E20E94C16387
:10AB6000CC2079F167E57AE080E10E94F86321E08A
:10AB7000F21202C0C13011F000E001C00D2F20918F
:10AB80005B022E5F49E35AE060E188E40E94C16302
:10AB900081E0F81202C0C23011F020E001C02D2F78
:10ABA00040915E0292E34902A0011124445D5E4F90
:10ABB00060E180E70E94FB65E1E0FE1267C082E091
:10ABC0001AC040915B02F5E0EF1201C04F7021E026
:10ABD000F21202C0C13011F020E001C02D2F552724
:10ABE00047FD509502E31AE060E18EE70E94E524FC
:10ABF00081E0F81284C08093E808809101088823DE
:10AC000009F451C0C13051F018F0C23031F12FC0F9
:10AC100066E08E2D0E942114D82E29C0CC2019F078
:10AC200044E06EEF13C095E0E9120EC080915B0224
:10AC30004FE060E08F700E941E1490915B02907F45
:10AC4000980F90935B0213C04CE760E080915B0229
:10AC50000E941E1480935B020AC0CC2041F04AE09F
:10AC60006CEF80915E020E941E1480935E028091C0
:10AC70005A02982F9F70807F2D2D2F70822B8093EA
:10AC80005A029D1581F010925B020DC0E2E0FE12A7
:10AC90000CC044E16CEE809164020E941E1480930B
:10ACA000640221E203C0CC2051F120E24091640211
:10ACB000F5E04F02A00111244F515F4F03E21AE06B
:10ACC00068E18CE40E94E5246AE17AE080E20E9477
:10ACD000F86321E083E0F81220E0409161024170C6
:10ACE00060E17AE080E20E94F2249091610280FBB0
:10ACF00090F990936102E4E0EE2E18E203C072E056
:10AD0000E72E18E195E0D912EFC064EE79E0812FCB
:10AD10000E94F863D0903C0521E0FE1020E04D2D0C
:10AD20004F716CE879E0812F0E94F22490913C05EC
:10AD3000907E980F90933C0500915B02492F552718
:10AD400047FD50952D2D30E04217530749F4402F11
:10AD500050E064E0559547956A95E1F7477001C06A
:10AD600040E088E0810F31E03E0D9F7179F0933033
:10AD700081F0953089F0973091F0993099F09B30BF
:10AD8000A1F09C30A9F46CEF78E014C060E779E0A2
:10AD900011C062E679E00EC066E579E00BC06FE2B3
:10ADA00079E008C06DE179E005C06AE079E002C0B1
:10ADB00064EF78E021E0F31220E00E94F2240F78A3
:10ADC000D02EE0E18E9FD00C1124D0925B0240E1A6
:10ADD000B42EB10E52E0C52ECE0CAD2CAA1CAA2466
:10ADE000AA1CFC1002C0CC2311F000E001C00D2F02
:10ADF0002A2D4AEE58E06B2D84E20E94C163FC10BC
:10AE000002C0C13011F020E001C02D2F40913D055E
:10AE1000552747FD50956B2D8EE70E94FB6562EE2E
:10AE200078E08B2D0E94F863FC1022C081E08093B3
:10AE3000E808C1110FC0809101088823C9F061E0C2
:10AE40008A2D0E9421149D2D9F77811190689093E7
:10AE50005B020EC0C13061F480910108882341F08B
:10AE60004FE761E880913D050E941E1480933D05E7
:10AE700028E1B22EB10E33E0A32EAE0CD0903C05EB
:10AE8000D6FACC24C0F8FA1002C0C13011F000E0AC
:10AE900001C00D2F2C2D4EED58E06B2D88E70E9440
:10AEA000C163FA101AC081E08093E808C11105C09F
:10AEB00061E08B2D0E94644A10C0C13071F4809112
:10AEC0000108882351F061E08C2D0E9421149D2DF2
:10AED0009F7B8111906490933C0584E08E0DF81265
:10AEE00053C460E280E250C0F2E0DF1212C065EDB0
:10AEF00078E0812F0E94F86321E0FE1020E040916D
:10AF00003C0566EB78E0812F0E94F22480933C059B
:10AF10003BC421E0D21238C46CE978E0812F0E9452
:10AF2000F86321E0FE1020E040913C056AE573E102
:10AF3000812F0E94F22480933C0521E081E08E0D58
:10AF4000F81220E040915A024295437066E673E1A0
:10AF500088E0810F0E94F22483708295807F909117
:10AF60005A029F7C982B90935A0282E08E0DF81221
:10AF700005C061E080E1810F0E94644A83E08E0D8C
:10AF8000F81202C460E288E1810F0E94644AFCC3A7
:10AF900088E498E00E94DF248CE08093EA0883E054
:10AFA0008093E808B090D9078F2D0E94954A982E7B
:10AFB00098E0D92EF91003C08090FC0701C0812CC5
:10AFC0004CE46D2D80E00E949B6388E0891510F4AD
:10AFD00048E301C041E3490D6D2D85E00E949B636C
:10AFE00091E0B91629F0E2E0BE1629F0712C01C0FB
:10AFF000782CA12C02C0A82C712C492D50E0EA011C
:10B00000CC0FDD1FC40FD51FCF55DB4FBB2011F078
:10B0100000E001C0082D2A812F7042EE55E16D2D10
:10B020008DE00E94C1638A818F700E948910C82EB2
:10B0300081111CC0188115327CF015526981812F55
:10B040000E94E1229C0102E8E02E0A2D412F6D2D85
:10B0500084E60E94902323C04981552747FD5095DF
:10B060002A2D6D2D83E60E94FB6519C0F1E08F1338
:10B070000DC0272D48816D2D86E30E9484112A2D55
:10B0800049816D2D8DE40E94841134C022E0821329
:10B090000DC02A2D49816D2D80E50E94A010272D1D
:10B0A00048816D2D86E30E94A01024C0488147FF8F
:10B0B00004C04095872D8062782E552747FD509516
:10B0C0004F5F5F4F04E418E0272D6D2D89E40E9447
:10B0D000E524498147FF04C040959A2D9062A92E2E
:10B0E000552747FD50954F5F5F4F2A2D6D2D8BE6FD
:10B0F0000E94FB654A8142954F7049300CF04F5FCA
:10B10000E3E0BE1611F020E001C0282D6D2D88E689
:10B110000E94841180910108882309F462C088206C
:10B1200009F45FC0F1E0BF1631F1BF1698F022E0DC
:10B13000B216D9F183E0B81254C08A816FE08295CB
:10B140008F700E9421148295807F9A819F70982B26
:10B150009A8347C08A816EE08F700E9421148F709D
:10B160009A81907F982B9A830E948910C816C9F102
:10B170001882198236C091E0C91659F0C91690F0AC
:10B18000E2E0CE1679F0F3E0CF122BC043E66EEC8E
:10B1900004C040915701642F619588810E941E145C
:10B1A00088831FC04EE260E0F8CF21E0C21671F044
:10B1B000C21648F082E0C81671F093E0C91211C0BF
:10B1C00043E66EEC0AC04DE763E807C040915701C3
:10B1D000642F619502C04EE260E089810E941E14D6
:10B1E00089839394E8E0DE0EF0E4DF12E3CECCC274
:10B1F00087E495E10E94DF2481E18093EA0883E0FF
:10B200008093E808A090D9078F2D0E94954A982E28
:10B210002FE02F15A0F0EF2DF0E0EE0FFF1FE6520C
:10B22000F84F4081518157FF02C04F5F5F4F5595E6
:10B23000479544525A4F60E08EE40E9429668091FF
:10B240000B02803819F58FE08F1540F14F2D50E03B
:10B25000FA01E919F109EE0FFF1FE652F84F2081BC
:10B260003181A11013C085E0849FF001859FF00D0E
:10B270001124EB55FC4F8281882319F031952195DB
:10B2800031093483238382E0ECD3E7D458E0E52E00
:10B2900065E0562E7AE0C72ED12C93C090E1F912CA
:10B2A000F5CF89E18093000880E80E94C3680E947E
:10B2B000D444ECCFE92DF0E05E9EE0015F9ED00D1E
:10B2C0001124CB55DC4FEE0FFF1FE652F84F808163
:10B2D00091814A812B813C81442319F0319521953C
:10B2E0003109821B930B833391050CF06EC08E3CA9
:10B2F0009F4F0CF46DC01DE266246394690C20E03E
:10B30000462D6E2D80E00E94CE10412F6E2D8BE4D5
:10B310000E949B638091610281FF5EC03DE7732EB6
:10B32000B12C44244A944E0C372C3194F91057C058
:10B33000AB1055C02091FC0780910108882309F4C7
:10B3400050C0222309F44DC010925601822E8091E4
:10B35000FB04882309F453C00B811C8101151105DE
:10B3600009F041C0C801B6010E94607482E0B816BD
:10B3700009F466C093E0B91609F486C0E1E0BE1690
:10B3800009F442C020624B815C816E2D8DE20E94E7
:10B39000FB65882059F022E048EE53E068E17CEF3D
:10B3A0008B819C810E944F139C838B83B39424E0F8
:10B3B000B212BCCF88E08E0D803409F47EC0E82E36
:10B3C000962CE0E19E1276CF6AC0411103C0EEC117
:10B3D0004111ECC11FE790CF24E6722EA1CF20E0EF
:10B3E000ABCF812CB4CF90E0801791075CF09195A2
:10B3F00081959109081719070CF0B4CF03C000E03C
:10B4000010E0B0CF8C01AECF18811456AB01410FC4
:10B41000511D17FD5A954338FFEF5F0714F443E8B9
:10B420005FEF6E2D88E40E94FB65882009F4BECF93
:10B4300049E1632D812F0E941E148C598883B6CF59
:10B4400089818C59AB01480F511D87FD5A954E37A4
:10B45000510514F04DE750E06E2D86E60E94FB6525
:10B46000012B31F029E048E3642D82E30E949F66BE
:10B47000882009F49BCF8981472D67EE8C590E9463
:10B480001E148456898392CF422F6E2D8A810E948A
:10B49000432591E0811101C090E09A8387CF21E09C
:10B4A000E0E1FE1220E080910008811181C143E3B8
:10B4B00058E06E2D82E10E94D36366C183E298E07A
:10B4C0000E94DF2489E18093EA08C090D9078F2D7C
:10B4D0000E94954AD82E88E0E82E90E1B92E8091FE
:10B4E000C704D11021C0F11010C01092E808C0911B
:10B4F000FC0760E18F710E9421148F719091C70445
:10B50000907E982B9093C70401C0C0E04091C7047F
:10B510004F7150E0485F5F4F03E118E02C2F6E2D14
:10B520008CE60E94E5242AC18F719B2C981ACD2DA0
:10B53000D0E0FD1003C082E08093E808C131D1055E
:10B540002CF4CC0FDD1FCA53DB4F04C0CC0FDD1F22
:10B55000C65DDA4F10E0FD1009C0C11207C00091AE
:10B56000FC07002321F0B2E0AB2E02C000E0A12CCA
:10B570009D1408F49EC0111118C020E04D2D6E2DB1
:10B5800080E00E94CE1048814295469546954370D2
:10B590002A2D6BE078E08E2D0E94F2248295880F90
:10B5A000880F807C98819F7331C08881113089F524
:10B5B00080905701982F907C903811F4A9E18A2E41
:10B5C000482F440F440F4595459547314CF029EEDF
:10B5D000240F44EF57E06E2D85E40E94C16305C03F
:10B5E000202F6E2D85E40E948411AA2009F4C2C088
:10B5F0006091570161958881880F880F482D859546
:10B6000085950E941E148F739881907C982B988347
:10B61000B1C0982F907C4981903491F447FD03C0CC
:10B620004F3024F401C040E0242F01C02FE02983D3
:10B6300049E556E16E2D88E70E94C1634FE015C0D1
:10B64000903831F5880F880F89358CF047FD04C09C
:10B6500049301CF049E001C040E049834F5F202F92
:10B660006E2D80E60E942E2249E060E01BC04F361E
:10B670000CF04FE64983552747FD509540585F4FE2
:10B68000202F6E2D88E70E94FB654FE660E80AC018
:10B69000552747FD5095202F6E2D88E70E94FB65AA
:10B6A0004DE763E8AA2009F465C089810E941E1451
:10B6B00060C0111122C061EF77E08E2D0E94F86307
:10B6C00020E04D2D6E2D86E10E942B66AA2069F0A8
:10B6D000409157014150888160E08F710E941E1493
:10B6E0008F719881907E982B988348814F71202F7D
:10B6F0006E2D8EE10E9484113DC08881113081F44D
:10B70000482F4295469547702A2D63EC77E08E2DA1
:10B710000E94F2248295880F807E98819F7176CF57
:10B7200082958695877090E04981069764F049304C
:10B7300008F049E049834F5F202F6E2D80E60E947C
:10B740002E2269E010C04B3F38F450E0202F6E2DC0
:10B7500086E60E94FB6506C0485F202F6E2D84E5BB
:10B760000E944B246FEFAA2029F0898190E00E946B
:10B77000261489831F5F133009F0EDCED39488E03F
:10B78000E80E90E4E912ABCEDF91CF911F910F91BB
:10B79000FF90EF90DF90CF90BF90AF909F908F90F1
:10B7A0007F906F905F904F903F9008951EE7A4CDDB
:10B7B00020E07DCE1F93CF93DF93EC011AE08881C8
:10B7C0000E94572C0E94672C89931150C1F7DF917A
:10B7D000CF911F9108959C01265F3F4FFB0144913B
:10B7E000DC014D93CD013196A217B307C1F708953F
:10B7F000EEE0F6E080E090E021913191820F931F1E
:10B8000026E0E632F207C1F7089587E7EDE0F6E0BB
:10B81000DF011D928A95E9F78BE080930D0689E19F
:10B8200080933B068AE580933C0681E08093510635
:10B8300086E180933E06EEE0F6E020E032E080E034
:10B8400093E02193319395878487938F828FB6E01D
:10B85000EC31FB07B1F76EEA78E18EE596E0BBDFED
:10B86000C7DF90933906809338060895EF920F93BF
:10B870001F9361E0680F88ECE82E02EC13E02BE4E4
:10B8800032E042E085EF98E0FCD521E0823C934035
:10B8900009F020E0822F1F910F91EF900895CF9330
:10B8A000C82F22EC33E0EBE4F2E0DF01C9011D9286
:10B8B0000197E9F763EA78E1CF018DDF8C2F90E003
:10B8C0006AE070E001960E946074605D60935002CF
:10B8D000805D8093510284E080933B0582E08093F9
:10B8E0005D020E942B6A8C2FCF91C0CF0F931F93C4
:10B8F000CF93DF93EB01042F803120F561E0680FD7
:10B9000085EF98E00FD410E0A80160E270E0CE016E
:10B910000E94D1744AE050E0BE0185EF98E085D4E2
:10B920000A9781F485EF98E0EFD3C00FD11F0097FD
:10B9300049F06AE070E00E946074805D8A93862F0F
:10B94000972FF5CFDF91CF911F910F9108958F5FC2
:10B9500093C361E0680F85EF98E0E4D382EC93E055
:10B96000EBE4F2E0DF019C011D9221503040E1F751
:10B9700042EC53E0BF0185EF98E057C4FF920F936C
:10B980001F93CF93DF93CDB7DEB768970FB6F894C8
:10B99000DEBF0FBECDBF01E0080F102F1031B0F495
:10B9A000FF24F394F10E8F2D67D381110DC0602F0A
:10B9B00085EF98E0B7D361E0610F28E532E042E01F
:10B9C000CE0140960ED506C01F2DE8CF103179F775
:10B9D00080E017C04FE050E0BE016F5F7F4F85EF02
:10B9E00098E0BDD3882349F0482FBE016F5F7F4F99
:10B9F000CE0140967DD4A895EDCFCE01409617D5C7
:10BA000081E068960FB6F894DEBF0FBECDBFDF9120
:10BA1000CF911F910F91FF900895EF920F931F9375
:10BA200061E08BE698E10E94451989E598E10E9462
:10BA30009312E6D298ECE92E07E710E02DE036E00D
:10BA400041E060E085EF98E01CD58737910521F053
:10BA50008AE498E10E94781980E01F910F91EF909D
:10BA60001ECFCF93C82F8770A1F090910009982B1B
:10BA7000909300090E9482109093FF088093FE0823
:10BA80008C2F90E024E0959587952A95E1F7809397
:10BA90000109CF910895CF93DF93D4D2811102C0D1
:10BAA00080E02EC04DD287FDFBCF60E085EF98E0AF
:10BAB00039D387E7EDE0F6E0DF011D928A95E9F7DB
:10BAC00047E750E0BF0185EF98E0AFD38EE596E001
:10BAD00071DE80910D068B3040F481E08093C701C8
:10BAE0008BE080930D0681E0BCDFC0913806D091D9
:10BAF00039067EDE21E0C817D90709F020E0822F41
:10BB0000DF91CF910895EF920F931F93CF93DF931F
:10BB100010924309C0910009CC2309F498C0909178
:10BB200001099F5C9093430981111CC00E948210FF
:10BB30002091FE083091FF08821B930B883C9105F1
:10BB400008F485C080910109882361F081508093B9
:10BB50000109882339F00E9482109093FF08809396
:10BB6000FE0875C0109201098091EB0881116FC029
:10BB7000DC2FD470C2FD02C081E001C083E080935D
:10BB8000EB08C0FF2CC082E3809343098091000939
:10BB90008E7F8093000944E1E42E07E710E02DE05A
:10BBA00036E041E061E18CEE98E06BD48737910597
:10BBB00019F461E180E02FC08091F208823051F4E5
:10BBC00080910009816030C08091F208823029F1B3
:10BBD000D1113BC089EB98E10E94781936C0C1FFB2
:10BBE00034C083E38093430980910009897F809367
:10BBF000000934E1E32E02EC13E02BE432E042E0F2
:10BC000061E18CEE98E03DD4823C9340E9F680916E
:10BC10003A0661E18F5F3ED218C080910009D111D0
:10BC200002C0826001C08660809300090E94821079
:10BC3000885C91099093FF088093FE088091910D94
:10BC4000833019F4A8951092910D1092EB08DF91B2
:10BC5000CF911F910F91EF90089580910009882353
:10BC600051F081E050DF8091910D8330B1F7A895BC
:10BC70001092910DF2CF0895EF92FF920F931F93C0
:10BC8000CF93DF93C82F803108F0BFC062DE8F3FB3
:10BC9000910509F010F48C2F02DE8BE492E08ADD2E
:10BCA0008091F304811107C080915C0286958370B6
:10BCB0008E5F8093F30480915A02982F9295969507
:10BCC00096959370933029F090933C05806C809307
:10BCD0005A0280913B05823008F062C010E0812F4B
:10BCE0000E948F10EC0189818150843018F40E94E9
:10BCF000751089831F5F103291F7C1EAD4E000E02C
:10BD000010E08A818F700E948910882389F0823028
:10BD1000C1F4C8018E559B4F7C01FC0180818823B2
:10BD200039F085302CF481500E947510F701808322
:10BD30008881882331F0853024F481500E94751069
:10BD4000888323960D5F1F4F04321105D1F688E3D7
:10BD5000E5EFF3E0AEE5B8E001900D928A95E1F7EA
:10BD6000CEE5D8E010E00EE0812F0E9475108150E2
:10BD7000089FD0011124AB50BC4FFE01802F0190D1
:10BD80000D928A95E1F71F5F2E96143069F78EE8C1
:10BD900098E10E94781982E080933B0562DE5DDFC6
:10BDA00080913B058330F8F480E090E0FC01EF5592
:10BDB000FB4F2281322F3F703C3019F4207F2A60E4
:10BDC00022832281322F3F703D3019F4207F2B6077
:10BDD000228303968432910549F783E080933B05E3
:10BDE00082E03FDE3ADF80913B05843070F4809141
:10BDF00068068093FA048BE798E10E94781984E042
:10BE000080933B0582E02DDE28DFE0E0F2E08091C8
:10BE1000560282838091C604838380915802909158
:10BE2000590291838083809157028170848380912D
:10BE3000F80487838091F90480878091F6049091BB
:10BE4000F704968385838091BC0587FB882780F95A
:10BE500081870E945E310E946431DF91CF911F91F2
:10BE60000F91FF90EF90089540E450E060E070E0A3
:10BE700082E099E00C94546741E050E062E070E0A9
:10BE800084E099E00C945467CF93DF931F92CDB771
:10BE9000DEB7698390E1899FB001112441E050E051
:10BEA000CE0101960E9454670F90DF91CF910895C3
:10BEB000CF93DF931F92CDB7DEB790E1899FB0019A
:10BEC000112441E050E0CE0101960E94D87489818E
:10BED0000F90DF91CF910895CF93DF93D82FC82F84
:10BEE0008C2FE6DF882321F08C2FE2DFC82FF8CFDC
:10BEF000609104098C2FC8DFD0930409DF91CF91A2
:10BF0000BBCFCF93C0910409CC2341F08C2FD0DF5D
:10BF100080930409B1DF60E08C2FB6DF8C2FCF91C6
:10BF20000895CF93DF9380910409C0E0D0E0882387
:10BF300019F02F96BDDFFBCFCE01DF91CF91089591
:10BF4000DF92EF92FF920F931F93CF93DF9380E8DE
:10BF5000EBE4F2E0DF011D928A95E9F7C6E0D9E053
:10BF6000F12CB4E1FB1205C08091040904E019E052
:10BF700002C08E01888190E0E12CDD24D394DF0C97
:10BF80000097E9F09C01245031092C37310530F439
:10BF9000FC01E55BFD4F2081222361F0EE2021F0C2
:10BFA00060E08E2D71DF03C0F80110825DDF80E05C
:10BFB00090E0E6CFD082E82E7BDF90E0E1CFF394F3
:10BFC0002396F5E1FF12CDCFC4E0D0E0FE01E55BA2
:10BFD000FD4F8081811107C0609104098C2F54DFCF
:10BFE000C093040949DF2196C038D10579F780E074
:10BFF000DF91CF911F910F91FF90EF90DF90089507
:10C00000CF9380E4E2E0F9E0DF01982F1D929A954A
:10C01000E9F794E0909302098093030980E180930B
:10C02000050984E0C1E0C80F6C2F2EDFCF3711F077
:10C030008C2FF8CF60E08FE727DF84E0809304093E
:10C04000CF9112CF40E450E060E070E082E099E0F0
:10C050000E94D87480910309811103C080E4809309
:10C06000030980910209843029F481E09091030949
:10C07000903409F080E0089590E0FC01EE0FFF1F7E
:10C08000E80FF91FEE5FF64F81E09481911101C036
:10C0900080E00895CF93DF9390E0EC01CC0FDD1F9B
:10C0A000C80FD91FCE5FD64F8C819D81AE8170E0C5
:10C0B000FB01EE0FFF1FE60FF71FEE5FF64F248127
:10C0C000358146812C833D834E8384839583A6836B
:10C0D000DF91CF91C9CECF9390E09C01220F331F07
:10C0E000280F391FF901EE5FF64FC481F901EA5FAD
:10C0F000F64F108211821282B7DECC2319F08C2FFA
:10C10000CF91EACECF910895FC01808190E0FC01AF
:10C11000EE0FFF1FE80FF91FE95FF64F9181808155
:10C120009F700895CF93DF93FC0160831282118288
:10C1300070E0CB01880F991F860F971FEC01CE5F2F
:10C14000D64F2C812383148215821682FC01E85F6E
:10C15000F64F808182958F70DF91CF910895AF92D5
:10C16000BF92CF92DF92EF92FF920F931F93CF93E4
:10C17000DF931F92CDB7DEB78C01FC01808190E088
:10C18000FC01EE0FFF1FE80FF91FE95FF64F8081FA
:10C190002181922F9F70F80121813281821B930BA4
:10C1A0007A018417950708F47C015B016701C114CB
:10C1B000D10421F1F8018381882301F164816F5F4B
:10C1C000648370E0F0E18F9F600D711D112441E0E8
:10C1D00050E0CE0101960E94D8748981F5018193C7
:10C1E0005F01F80184818F3028F01482838160DE42
:10C1F000F8018383F1E0CF1AD108D9CFF80181810A
:10C2000092818E0D9F1D8C199D09928381838E2DA5
:10C210008C190F90DF91CF911F910F91FF90EF90AC
:10C22000DF90CF90BF90AF9008957F928F929F92B2
:10C23000AF92BF92CF92DF92EF92FF920F931F9334
:10C24000CF93DF934C016B018A01C0E0D0E05C0129
:10C2500025E0A20EB11CC017D107D8F5F4018581E5
:10C260008F7781F0F4014581F42FFF777F2E2F2FF8
:10C2700030E0C8018C1B9D0B8217930758F4702E79
:10C280007C1A08C041E050E0B501C40168DF81308C
:10C2900049F31FC0E72CF12CC6018C0F9D1F47FFEF
:10C2A00006C0A70160E070E00E94D1740BC0A70136
:10C2B000BC01C40154DF871529F0FE01E80FF11D10
:10C2C000CF0108C0CE0DDF1DF4018581871985835C
:10C2D000C2CFCE01DF91CF911F910F91FF90EF90D0
:10C2E000DF90CF90BF90AF909F908F907F900895F8
:10C2F000AF92BF92CF92DF92EF92FF920F931F9374
:10C30000CF93DF93EC018B01D42E8B81811110C070
:10C3100089819A81892B61F4E880F12CF2DD8B838D
:10C32000F701EE0FFF1FEE0DFF1DEE5FF64F84834A
:10C33000CD2C8FE0A82ECC2009F43CC0EF80F884EF
:10C340000E948210E81AF90AF7FE02C082E004C0D7
:10C350008B81811103C081E08E832CC09C819F3032
:10C3600058F01C82A5DD811104C0CBDD682F8B81C4
:10C370008BDD8B819DDD8B838B81882361F36C81C9
:10C380009A2D961BBC2C9C1508F4B92EEB2CF12C85
:10C3900070E090E1899F600D711D11246F5F7F4FE8
:10C3A000A701C80181D50E0D1F1D8C818B0D8C83BB
:10C3B000CB18C1CF6D2D70E06C19710929813A81BC
:10C3C000260F371F3A8329838D2D8C19DF91CF914A
:10C3D0001F910F91FF90EF90DF90CF90BF90AF90A3
:10C3E0000895EF92FF920F931F93CF93DF93EC0189
:10C3F000F62EE42E890196DE6F2D70E0FB01EE0F24
:10C40000FF1FE60FF71FE95FF64F1082E29430EF4F
:10C41000E322E1820E948210800F911F98878F8310
:10C42000DF91CF911F910F91FF90EF9008951F938F
:10C43000CF93DF93EC01888190E0FC01EE0FFF1FAA
:10C44000E80FF91FE95FF64F898180839A819F7019
:10C450008181807F892B81838B81882321F028DD56
:10C46000182F81110AC010E0FFDC112311F0812F79
:10C4700033DDDF91CF911F91089560E08B8104DD62
:10C48000F3CF7F928F929F92AF92BF92CF92DF9223
:10C49000EF92FF920F931F93CF93DF931F92CDB72D
:10C4A000DEB76C0159012E2D30E09BDF198245016A
:10C4B000E12CF12C77247394F40181914F0199813F
:10C4C000811108C071104CC08081811105C0772492
:10C4D00073941BC071100AC080E09F3718F4E016F7
:10C4E000F10661F5772081F0782E01C0712C992337
:10C4F00029F19068998341E0BE016F5F7F4FC601CB
:10C50000F7DE8130D1F026C0782E9923B9F041E0D2
:10C51000BE016F5F7F4FC601EBDE8130D9F44981E8
:10C52000B701641B71096A0D7B1DC601E1DE9981AB
:10C53000891719F0981B99830DC0198289818F5F23
:10C540008983A895FFEFEF1AFF0A0E151F0508F063
:10C55000B3CF08C089818F778701081B110902C0FA
:10C56000872DBBCFC60163DFC8010F90DF91CF914C
:10C570001F910F91FF90EF90DF90CF90BF90AF9001
:10C580009F908F907F90089580E094E0E5E4F9E03B
:10C59000DF019C011D9221503040E1F70895FF9288
:10C5A0000F931F93CF93DF93FA01149131967491F7
:10C5B000795F769576957695DA011396FA0132963B
:10C5C0004491249FA00DB11D112466956695669532
:10C5D00090E0F0E86F9F800D911D112420E030E085
:10C5E00060E08B5B964F412F50E0671799F00A2F60
:10C5F000EC01C20FD31FFD01FE2EF01AF11620F43C
:10C60000F490F9923196F8CFA40FB51F6F5F2058C0
:10C610003F4FEBCFDF91CF911F910F91FF90089586
:10C62000CF93DF93382F463128F4842F880F840F5F
:10C63000880F7EC086E0830F20FD08C021FD02C068
:10C6400090E005C09091580D96FFFACF91E0687F79
:10C65000A32FB0E050E1659FA00DB11D1124AB5B8D
:10C66000B64F22FF3DC04E3211F088E0830F24ED1B
:10C67000240F2F3010F44B5211C02FEB240F2A310E
:10C6800010F441530BC02FE9240F2A3110F4465304
:10C6900005C04F3511F44AE201C040E06EE0469F0C
:10C6A000A00111244D52574E27E0FA0134913796DC
:10C6B000E491211102C0E0E030E04F5F5F4F992329
:10C6C00011F03095E095FCE0A43CBF0730F43C93BA
:10C6D000ED01C058DF4FE8831196215030F728C094
:10C6E00023FF07C0892F81958D9385E0830F31E06B
:10C6F00001C030E025E0429FF0011124E750F44EE4
:10C7000025E04491332311F0243041F05DE0A5345D
:10C71000B50718F4911140954C931196215031961C
:10C720002111EFCF6DE0A534B60710F491959C93DD
:10C73000DF91CF91089520E073CFEF92FF920F9396
:10C740001F93CF93DF93F62E122F902F9071E92E27
:10C75000FA01112379F0EE2011F0408101C04491DB
:10C76000EF012196442331F0202F6F2D59DF115016
:10C77000FE01EFCFDF91CF911F910F91FF90EF90CE
:10C7800008950F93FA0194914F5F5F4F929F400D70
:10C79000511D1124292FD1DF0F9108950F9300E02F
:10C7A000CCDF0F910895FF920F931F93CF93DF93E8
:10C7B000162F022F922F9071F92EEA01FF2011F00F
:10C7C000488102C0FE014491442361F04F3131F4AD
:10C7D000185F103438F480E02196F0CF202F612FBD
:10C7E0001FDFFACFDF91CF911F910F91FF90089536
:10C7F000AB0120E0682F80E0D6CFFB01442341F05D
:10C800009491992351F09F3109F441503196F6CF1C
:10C8100020E0AF01682F80E0C6CF089520E0C3CFAD
:10C82000FF920F931F93CF93DF93082FF62EEA0109
:10C8300014E1180F15504C2F4F704A301CF0495C12
:10C8400028E002C0405D20E06F2D812FE9DE84E00A
:10C85000D695C7958A95E1F71013ECCFDF91CF916C
:10C860001F910F91FF900895222321F09091580D70
:10C8700096FD0895480F687FE82FF0E090E1699FEA
:10C88000E00DF11D1124EB5BF64F8E1B982F9E0FD0
:10C89000941720F4908190959193F8CF08952DE00E
:10C8A0008534920760F4FC012081309144093323E0
:10C8B00019F0262B313009F02627FC01208308953A
:10C8C000262F287F6770E62FF0E0ED57F14E649138
:10C8D00090E030E1239F800D911D11248B5B964FDA
:10C8E000DECFEF92FF920F931F93CF93DF93F42E3F
:10C8F00047FF02C0840FF194962F987FC82FD0E095
:10C9000080E1989FC00DD11D1124CB5BD64F67707D
:10C91000E62FF0E0ED57F14EE490FF20B1F08DE00E
:10C92000C534D80790F4022F10E020FF08C06E2D08
:10C93000CE01B5DF15950795202F206803C015950A
:10C940000795202FFA942196E8CFDF91CF911F9180
:10C950000F91FF90EF9008952FEFC3CF1F93CF93C8
:10C96000DF93142F47FF02C0640F1195962F987F15
:10C97000C82FD0E080E1989FC00DD11D1124CB5B62
:10C98000D64F862F877099F0E82FF0E0ED57F14EE3
:10C9900064916195180F185017FF0DC0E12FFF2704
:10C9A000E7FDF095E557F14EE4916E0F04C01830A5
:10C9B0003CF018506FEFCE0172DFC058DF4FF7CF59
:10C9C000111654F4E12FFF27E7FDF095ED57F14ED6
:10C9D00064916150CE0163DFDF91CF911F91089583
:10C9E0003F924F925F926F927F928F929F92AF92FF
:10C9F000BF92CF92DF92EF92FF920F931F93CF934C
:10CA0000DF93182FB62E802F05FF04C004FF04C04B
:10CA100002E003C000E001C001E0982F9F77C92E1B
:10CA2000E7FE04C0E1946624639401C0612C57FFC3
:10CA30000AC050954095309521953F4F4F4F5F4F1D
:10CA40007724739401C0712C82FF06C098E0909304
:10CA5000450DE8E0DE2E05C096E09093450D75E0AB
:10CA6000D72E86FF28C071101D0D283E83E03807A1
:10CA70004105510514F01D0D05C024363105410551
:10CA8000510514F01D0D05C02A3031054105510531
:10CA90000CF01D0D002381F0023031F424363105F5
:10CAA000410551054CF41D0D2A3031054105510554
:10CAB0001CF41D0D01C01D198091450D810F80933F
:10CAC000450D023011F490EFC90E8824839452E092
:10CAD000A52E912CFF24E7FCF09466E0562E5B0C0B
:10CAE000E82DF0E0EE16FF060CF45DC06AE070E0A1
:10CAF000C9010E946074382EEB0140E3442E480EB9
:10CB00002C2D442D6B2D812F8BDD08112FC0C2FEE3
:10CB10001AC08FEF830D833008F4A394CE016AE02E
:10CB200070E00E946074823011F08430D9F484E3A4
:10CB3000481204C099249394910E15C099249A9494
:10CB4000910EA39410C03EEF432E410E8FEF810F44
:10CB5000C0FE04C047E06B2D01DF02C0652DB0DED2
:10CB6000142D01C0912E209709F000E09E0144276A
:10CB700037FD4095542F211531054105510581F4AC
:10CB8000002331F0023059F491E0981540F008C0CC
:10CB9000C4FE09C0611004C080EFC80E01C000E0EF
:10CBA0001D1983949DCF992059F09A944A2D6CE0D9
:10CBB0006B0D892DD1DE4A2D6DE06B0D892DCCDEFC
:10CBC000772031F02C2D4DE26B2D812F8D1928DD32
:10CBD00080E0DF91CF911F910F91FF90EF90DF9058
:10CBE000CF90BF90AF909F908F907F906F905F900D
:10CBF0004F903F900895EF920F93022F9A01442790
:10CC000037FD4095542FF5E0EF2EEADE0F91EF90BF
:10CC10000895CF93DF93D62FC22F206250E0EBDF31
:10CC2000C7FD08C02C2F46E76D2F8091450DDF9181
:10CC3000CF91F6CCDF91CF91089590913D01209155
:10CC40003C06921710F422E001C020E0242B492F6B
:10CC5000E0CF20E0D0CFEF920F93022F005F242F80
:10CC600030E040E050E0A2E0EA2EBADE0F91EF9013
:10CC70000895DF92EF92FF920F931F93CF93DF936C
:10CC8000182FE62EEA01F22E822F8470D82E22FF72
:10CC900005C01D5F57FF0FC087E103C057FF0BC0E2
:10CCA0008FE02F2D4DE26E2D912F981B892FB8DC30
:10CCB000D195C195D1092F2D20234AE36E2D812FC7
:10CCC000AFDC6CE370E0CE010E946074462FC82F89
:10CCD000D1101E5F2F2D6E2D812FBDDFDD2011F0B5
:10CCE00085E101C08FE0810F202F4C2F6E2DDF9149
:10CCF000CF911F910F91FF90EF90DF90ACCF0F93EA
:10CD00001F93CF93DF93C82FD62F142F022F422FBC
:10CD100025DE123030F0402F6D2F8FEF810F8C0FFA
:10CD20001DDE6FEF6D0F600F412F8C2F15DE412F31
:10CD30006D2F8C2FDF91CF911F910F910DCECF933F
:10CD4000C091440991E090934409D9DFC09344090C
:10CD5000CF9108950F931F93CF93DF93182FC62F72
:10CD6000D22FE42FF0E03297053608F004E60E9F4C
:10CD7000C0010F9F900D112464E670E00E94607462
:10CD8000062F2D2F6C2F812FDADF002361F0D15079
:10CD9000DC0FCF5F1F5FCD1730F4402F6C2F812F3A
:10CDA000DBDDCF5FF8CFDF91CF911F910F91089519
:10CDB000A998AB988BBBAD9AAD98AB9AA99A0895F8
:10CDC000CF93C82F81E08093420981E8F1DF8C2F57
:10CDD000EFDF10924209CF91089580913B06F0CF8A
:10CDE000CF93DF9381E080934209AA982AE02A95A5
:10CDF000F1F700C0AA9A8CED95E0E5E0EA95F1F72D
:10CE0000000001970097C9F7AC98C9ECD8E1FE0182
:10CE10008491CEDF2196F8E1C33DDF07C1F7DF91B2
:10CE2000CF91DBCF1F93CF93DF93409143094423EE
:10CE300021F08091580D86FD32C081E08093420937
:10CE400010EBC5E4D9E084E0B3DF80E1B1DF812FEE
:10CE5000AFDFA998AB9AFE019E0120583F4F808119
:10CE60008BBBAD9AAD9881818BBBAD9AAD98828119
:10CE70008BBBAD9AAD9883818BBBAD9AAD98349640
:10CE8000E217F30761F7EF01AB9AA99A1F5F183B0E
:10CE9000D1F610924209DF91CF911F9108954A5225
:10CEA00060E080E059DDC9CFBF92CF92DF92EF9270
:10CEB000FF920F931F93CF93DF937B018A01080F9B
:10CEC000191FEC01E81AF90A6701CC0EDD1EC01724
:10CED000D107C1F0B9908091EB088270E19B05C049
:10CEE0008823E1F30E94F51BF6CFDFBACEBAE09AB1
:10CEF0008DB3B81649F3BDBA8FB7F894E29AE19AA8
:10CF00008FBFE2CFDF91CF911F910F91FF90EF90F4
:10CF1000DF90CF90BF9008958091890D1092890D78
:10CF20000895FC0180818F70880F611181608F707E
:10CF30009081907F982B908381818F5F8183828104
:10CF4000882351F09F7041F4833621F0842F806252
:10CF50008093890D118212828281883069F148F4B0
:10CF6000813091F188F0823039F1843009F03FC08E
:10CF700023C08F35C1F018F48031F1F00895813667
:10CF800049F0823671F1089580818F708F3079F584
:10CF900081E62BC040664093890D109236011092B5
:10CFA00035018FE522C08181803211F4406816C0BE
:10CFB0008832E9F480E119C09181903328F090E043
:10CFC0009595879582831182828190E001972181D6
:10CFD00030E082239323892B51F440644093890DE0
:10CFE00008958181803418F088E082831182089549
:10CFF0005091630041B1282F30E02F3031056CF49F
:10D00000F901EE0FFF1FE20FF31FE45AF24F908178
:10D010009F7081E09F3051F52AC090E0FC013F975E
:10D02000E930F10518F5E955FF4F0C94B174942FD0
:10D03000947019C091B1927016C0952F10C0952FA1
:10D040009095987010C053FF11C091B102C0942FF9
:10D050009095907408C0942F907105C0942F917092
:10D0600002C0942F907281E0911101C080E0089578
:10D070008D3208F062C09FEF980F993010F4825FF4
:10D08000B7CF51EE580F5330D8F491B190959470BA
:10D090005523C9F0409180064F70415021E030E0A7
:10D0A000042E01C0220F0A94EAF730915B0D32235F
:10D0B000523041F0932B21E009F020E0922F03C081
:10D0C00090E001C0932F85528330F0F491B1969592
:10D0D000917021E09227882369F140918006429562
:10D0E0004F70415021E030E0042E01C0220F0A941D
:10D0F000EAF730915B0D3223823009F1932B81E006
:10D1000009F080E0982F16C0863019F4209182062D
:10D1100005C0873079F42091820622952F70215026
:10D1200081E090E0022E01C0880F0A94EAF7909106
:10D130005B0D982381E0911104C080E00895932F46
:10D14000F9CF0895CF93C82F93DF811107C081E0F5
:10D150008C0F8EDF882321F081E003C080E001C0C6
:10D1600082E0CF9108958F7090E08F30910551F05B
:10D17000FC01EE0FFF1FE80FF91FE45AF24F82E6A1
:10D180008283118208958F7090E08F30910549F06D
:10D19000FC01EE0FFF1FE80FF91FE45AF24F83E680
:10D1A00082830895EF92FF920F931F93CF93DF93A3
:10D1B0008091590D90915A0D019690935A0D80933C
:10D1C000590D8093580D96B3909580918A0D8823C0
:10D1D00021F0282F2877292349F4892F807609F018
:10D1E0007DC093FD77C094FF77C080E1182F166053
:10D1F000192380938A0DCCE5DDE000E011FB662762
:10D2000060F9402FCE018DDE0F5F16952396063014
:10D21000A9F780910A0281110EC0F0B2F0948091BA
:10D220006D0686FF09C08F2D837FF82E8091600EDA
:10D230008C70F82A01C0F12CCBE8DEE100E010E0B0
:10D2400076E0E72EEC1AFE0184914C2F4E0D8F21D3
:10D2500061E009F460E0C8018259924F62DE2196D4
:10D260000D5F1F4F0831110571F79091100261E0B9
:10D27000C92FC07295FF60E04EE086E89DE051DE68
:10D2800086B390E0809590958E7799278C2B19F036
:10D2900089E0809355018091600E86FD02C0817403
:10D2A00002C0817082609091630092FF88609091CB
:10D2B000630095FF8062989B84609C9B8064B79B11
:10D2C000806180935B0DDF91CF911F910F91FF9053
:10D2D000EF90089588E08ACF80E088CF80E686CFFF
:10D2E000929A1092980089E18093990080919B0016
:10D2F0008D7F80939B0086E080939D0080919B00B2
:10D3000087FF03C080919C00F9CF88E980939A0041
:10D31000089581E080938E0D80930A0280916D06BE
:10D3200086FFDECF089580916D0686FF10929A00E9
:10D3300010920A02F1C590919B0095FFFCCF80935B
:10D340009C000895E6E4FDE091898089891749F001
:10D35000DF01A90FB11D8C919F5F9F70918B90E0B1
:10D3600008958FEF9FEF08951F920F920FB60F92BF
:10D3700011242F938F939F93EF93FF9380919A00A3
:10D380008F7780939A007894E091560D81E08E0F0C
:10D390008F7090919C002091570D821731F0F0E032
:10D3A000EA5BF24F90838093560DF89480919A0037
:10D3B000806880939A00FF91EF919F918F912F91B8
:10D3C0000F900FBE0F901F90189580E491E0E5E656
:10D3D000F2E0DF019C011D9221503040E1F70895F9
:10D3E000FF920F931F93CF93DF93182FF62EC5E66E
:10D3F000D2E090E08881181738F0882329F0903225
:10D4000001F19F5F2A96F6CF9032D9F02FE130E0FC
:10D41000291B31090AE0029FA001039F500D11242E
:10D42000BE01CE010A960E94C074FE0111920A95B7
:10D43000E9F7188384E68A838F8188608F83CE0121
:10D4400002C085E692E0FC01F182DF91CF911F914D
:10D450000F91FF900895CF93DF9300D000D0CDB708
:10D46000DEB7E0915606F0E0E95AFC4FE49184E023
:10D470009E2F9370A1E0B0E0AC0FBD1FA90FB11DAE
:10D480008C93E695E695815099F79FDF61E089815D
:10D49000A7DF62E08A81A4DF63E08B81A1DF64E023
:10D4A0008C810F900F900F900F90DF91CF9198CFBC
:10D4B00080E49CE99BBD8ABD87B7806187BF1FBCA4
:10D4C0008AE08EBD08950F931F93CF93DF93109141
:10D4D0005C02129516951770882331F0A3EEBDE01B
:10D4E000833021F420E103C0ABE9BDE028E0909156
:10D4F0005B02990F910F920F60915E0224E6620227
:10D50000B0011124685A7D4F0091640248EE53E047
:10D5100004039001059F300D112428533045261B2C
:10D52000370BFD0132966D937C934091610241FF70
:10D5300003C040E055E002C040E054E0833011F405
:10D5400018EF190FCC27DD27C41BD50B1917F0F4E2
:10D55000A12FB0E0AA0FBB1FA652B84F0D90BC91EF
:10D56000A02D4A175B070CF4DA01AC17BD070CF4C9
:10D57000DE01A854B44F2A1B3B0BA61BB70BB1838B
:10D58000A083738362831F5F3496E0CF283293E2D7
:10D59000390710F428E233E231832083882331F005
:10D5A000285E334030938C0D20938B0D13821282B2
:10D5B000DF91CF911F910F9108951F920F920FB697
:10D5C0000F9211242F933F934F938F939F93EF9339
:10D5D000FF9388B391E0892788BBE0910E01F09119
:10D5E0000F018081982F9F709F3039F040912D0E50
:10D5F000949F402D1124415001C04FEF242F30E063
:10D6000037BD26BD90E024E0959587952A95E1F7F2
:10D61000009731F43196F0930F01E0930E0101C0B1
:10D620008083493C40F080915A028F70863011F41B
:10D63000C09801C0C09A8091910D81608093910D36
:10D64000FF91EF919F918F914F913F912F910F906B
:10D650000FBE0F901F9018951F920F920FB60F924A
:10D6600011242F933F938F939F93EF93FF9388B34E
:10D6700091E0892788BBE0911001F0911101808130
:10D6800028B539B580FD03C0205E3F4F02C0205F42
:10D690003F4F39BD28BD90E095958795009769F477
:10D6A000CF01019690931101809310018181811126
:10D6B00005C087B7877F87BF01C080838091910DA8
:10D6C00081608093910DFF91EF919F918F913F9198
:10D6D0002F910F900FBE0F901F901895EDE7F0E07F
:10D6E0008081857E808317981F9AAAE8B0E01C92FB
:10D6F00010928B0082E88C938081806280830895F1
:10D70000EDE7F0E080818F7D8083179AAAE8B0E092
:10D710001C9210928B008AE08C93808188618083B8
:10D7200008951F920F920FB60F9211248F939F931B
:10D73000EF93FF9380912B0E882321F01F9A109274
:10D740002B0E04C01F9881E080932B0EE0910A01FC
:10D75000F0910B01808191819093870080938600E6
:10D7600080918B0D90918C0D909385008093840017
:10D7700082819381892B11F0329608C080916102D9
:10D780008095817080932B0EE3EEFDE0F0930B010A
:10D79000E0930A018091910D81608093910DFF913A
:10D7A000EF919F918F910F900FBE0F901F90189542
:10D7B000E2E9FDE09081969596952781222311F06C
:10D7C00096959695982B908321812F5F2183808554
:10D7D000281750F0A281B3819D012F5F3F4F338303
:10D7E00022839C93108211820895FF920F931F93BE
:10D7F000CF93DF93C82F80915A028F70823069F0E7
:10D800009C2F88E0D0E0292F2078D20F990F8150EB
:10D81000D1F7D07859E0F52E03C048E0F42ED0E8D7
:10D8200010E080E190E00C2F0170901302C0805F47
:10D8300002C0BEDF80E1C695CD2B1F5FF11618F048
:10D84000D0E8902FF0CF805FDF91CF911F910F91A3
:10D85000FF90AECF882339F08091980D8F5F809331
:10D86000980D80E803C01092980D80ECA1DF8091A4
:10D87000980D8530C0F70895CF93DF93C82FE091BE
:10D88000970DE827F0E0EE0FFF1FED56F14E2591C2
:10D8900034915091960D40E0242735273093970D11
:10D8A0002093960DD8E08C2F8078D4DFCC0FD15008
:10D8B000D1F7DF91CF910895CF9380EC79DFC6E067
:10D8C00080E876DFC150E1F780ECCF9171CF8031F5
:10D8D000E0F4E82FF0E0EE0FFF1FE652F84F208152
:10D8E0003181C901880F991F820F931F97FD0396FD
:10D8F00095958795959587959C5F1816190644F41C
:10D900008E3F27E092073CF4089580E094E008956C
:10D9100081E090E008958EEF97E008956F927F92F6
:10D920008F929F92AF92BF92CF92DF92EF92FF922F
:10D930000F931F93CF93DF931F92CDB7DEB772E99A
:10D94000672E7DE0772EF3013F018BE99DE0938305
:10D950008283108211821582148281E0878382E0A3
:10D960008087F0905A02FF2DFF70FF2EF8132BC016
:10D9700080E180932D0E80918D0D86FF0DC08091EA
:10D980003C05811102C080E805C0813011F480E9B6
:10D9900001C088E980938D0D80918D0D87FF05C0B2
:10D9A00087E126DB882309F4BAC080918D0D87FDBD
:10D9B000BCC085E10E942519882309F4B6C0809176
:10D9C0008D0D8062B5C084E180932D0E86E0F81342
:10D9D00002C08FE01EC085E508DF80913C058F5FA7
:10D9E0008F7580938D0D90918F0D90FF03C080688F
:10D9F00080938D0D95FF05C080918D0D8062809381
:10DA00008D0D80918D0DF1DE80915B02EEDE8091B7
:10DA10003D05EBDE0AED17E0C12CD12CE12C912C59
:10DA200035E0A32EB12C48EF842EF801819191911D
:10DA30008F01880F991F880F991F181619061CF45B
:10DA400024E030E002C02CEF3FEF820F931FB501BE
:10DA500037D7F5E0CB01FF1202C09C5F02C08052B5
:10DA60009C4F97FD07C0811528E092072CF08FEF9F
:10DA700097E002C080E090E0AA2797FDA095092CCE
:10DA800003C0880F991FAA1F0A94DAF7C82AD92A57
:10DA9000EA2A8BE0890D89838C2DA7DECD2CDE2C24
:10DAA000EE24E981E850E983E830B0F793E0990D7E
:10DAB000892F869586958695992E889D900C1124A0
:10DAC000F7E00A3F1F0709F0B0CF26E0F21204C0CA
:10DAD00080E08BDE80E089DEF3018181A281B38169
:10DAE000882319F08FE08C9304C0FD018291806F30
:10DAF00080838BE99DE090930F0180930E010F903E
:10DB0000DF91CF911F910F91FF90EF90DF90CF9019
:10DB1000BF90AF909F908F907F906F90089580916D
:10DB20008D0D8F7780938D0D40CF80918D0D8F7DE2
:10DB300080938D0D80918D0D58DE80915B0255DEB6
:10DB40000AED17E0F12C6DE0D62EF801819191914C
:10DB50008F01D89E9001D99E300D112455E0359546
:10DB600027955A95E1F73E5F37FD07C02F3FF3E059
:10DB70003F0734F4E22E832F06C0E12C80E003C07F
:10DB8000EE24EA9483E09F2D990F990F892B2DDEC7
:10DB90008E2D2BDEF39426E0F212D7CF9DCFCF92BD
:10DBA000DF92EF92FF920F931F93CF93DF93C09179
:10DBB0005A02CF708091590685FF04C080914702B8
:10DBC0008111C4E080918E0D8111CFEF8091900D75
:10DBD0008C1709F467C0C093900D1EBC1DBC1CBC03
:10DBE00087B7837C87BF80917D008E7F80937D0087
:10DBF0008CE386BF8FE380937C008C2F90E087308E
:10DC0000910508F04FC0FC01E055FF4FAAC666DD44
:10DC10004FDC08C163DD88E59BE199BD88BD80EAE2
:10DC20009FE0909379008093780087B7886087BFE2
:10DC300080917D00816080937D001FBC82E08EBD5D
:10DC400044C04CDD88EC90E090937900809378009C
:10DC50008CE291E09DBD8CBD80EE9BEA97BD86BDB8
:10DC600087B7806287BF80917D00816080937D004F
:10DC70001FBC8AE18EBD16C0C43021F484E023DCD1
:10DC8000C09803C015DC83E01EDC80E593EC909324
:10DC900087008093860088E893E1909385008093C5
:10DCA00084002EDDC23009F4BAC038F4CC2309F464
:10DCB000B9C0C13009F0B8C008C0C33009F4B2C05F
:10DCC000C550C23008F0B0C0AAC07894F0902D0EB4
:10DCD00087B7877F87BF80917D008E7F80937D008F
:10DCE000E2E9FDE08BE99DE0909311018093100142
:10DCF0008CE99DE0938382831582148210821182C5
:10DD00001682178284E080878FEF80939B0DD4DD8D
:10DD100080915B02B1DD40918F0D80913C0540FF09
:10DD20000CC090E489029001112480915A028695DA
:10DD3000869586958670822B04C020E48202C001FD
:10DD40001124842B99DD80E097DDE0905C02E29461
:10DD5000E694A7E0EA228F2D8170D82EF0FE02C053
:10DD600098E0E90EF8E0CF2ECE0C8E2DB0DD8C01C0
:10DD7000D110185F802F80DD81E08E0DA8DDEC01D1
:10DD8000D110D85FE394E3949C2F9295907F812FDC
:10DD90008F70892B71DDCE01E4E096958795EA9529
:10DDA000E1F76ADDEC10E1CF80E066DDC091960D11
:10DDB0008091970D61DD8C2F5FDD7EDD8091930D6D
:10DDC000882319F080E0F4DCF9CFE091940DF09114
:10DDD000950D1082E8E7F0E0808191819C01285444
:10DDE000344F39BD28BD805B994B91838083C09AA5
:10DDF00088E086BF81E080937C0087B7886087BF1A
:10DE000080917D00816080937D0080913C05813010
:10DE100011F0F39401C0F12CF0922D0E05C078940E
:10DE20007DDD02C080E04FDBDF91CF911F910F912C
:10DE3000FF90EF90DF90CF9008951F920F920FB652
:10DE40000F9211242F933F934F935F936F937F9380
:10DE50008F939F93AF93BF93CF93DF93EF93FF93F2
:10DE60008CB59DB520912C0E222321F0C09A1092E2
:10DE70002C0E04C0C09821E020932C0EC0910C0100
:10DE8000D0910D01FE01219131913BBD2ABDF0934E
:10DE90000D01E0930C01E6E0F1E0282F3181381705
:10DEA00008F481833081231708F480838A819B8161
:10DEB000892BD1F48BE99DE090930D0180930C01A7
:10DEC000809161028095817080932C0E87B78F7E40
:10DED00087BF65DE80915A028F7011F0833021F484
:10DEE00087B7806187BF78948091910D816080931E
:10DEF000910DFF91EF91DF91CF91BF91AF919F91E4
:10DF00008F917F916F915F914F913F912F910F90E2
:10DF10000FBE0F901F9018958091610280958170BF
:10DF200080932C0E80932B0E811101C0C09A80919A
:10DF30005A028F70865F8093900D10928E0D2FCEB7
:10DF40001F920F920FB60F9211242F933F934F936E
:10DF50005F936F937F938F939F93AF93BF93EF9351
:10DF6000FF9380915A028F70813011F1863029F031
:10DF7000853031F080E492EA05C080E89EE302C07B
:10DF800080E99DE397BD86BD2091780030917900AE
:10DF90002F3F310538F4885893419093790080934E
:10DFA000780007C088EC90E0909379008093780027
:10DFB000F6DDFF91EF91BF91AF919F918F917F918E
:10DFC0006F915F914F913F912F910F900FBE0F90E6
:10DFD0001F9018951F920F920FB60F9211242F9336
:10DFE0003F934F935F936F937F938F939F93AF93E1
:10DFF000BF93EF93FF9380915A028F707894909122
:10E00000900D981769F0943059F480914702882355
:10E0100021F08091590685FD02C0C1DD02C084E077
:10E0200052DAFF91EF91BF91AF919F918F917F91C4
:10E030006F915F914F913F912F910F900FBE0F9075
:10E040001F9018958091830680FD05C08091650022
:10E050008B7F809365000895CF93DF93EC01F2DF0F
:10E060001C821D82188219821EA61FA6DF91CF91E5
:10E070000895F2CF21E0FC018481811101C020E0EC
:10E08000822F0895FC0121818081281B277098E050
:10E09000921B81E0933008F480E00895CF93DF93E2
:10E0A000EC018C818823F1F081508C838A819B81E3
:10E0B000890F8A838EA58823D1F18FA59FEF980FB2
:10E0C0009FA7882351F08091830680FD30C0809106
:10E0D00065008460809365002AC0B4DF80915B0690
:10E0E0008FA725C01B98AEDF8D81882319F0815042
:10E0F0008D831DC0888199818917C9F090E0FE0148
:10E10000E80FF91F26812A8326892C8326852B83F5
:10E11000268D2D8320A92EA71FA626A13FEF320F03
:10E1200036A3211104C00196877099278883DF9157
:10E13000CF910895EF92FF920F931F93CF93DF93A8
:10E14000EC01F62E142FE22E9DDF882309F451C036
:10E150008091C60181FD4DC0302F329536953695A0
:10E160003370402F4F70333009F43FEFFF2021F020
:10E1700080915A06865FF80E809150068873803130
:10E1800029F48BEA189F112D112402C0883111F453
:10E19000169509C0883211F4110F05C0803319F4A7
:10E1A000812F880F180F288104FF0DC0FA821C836D
:10E1B000ED8205FB882780F98EA71FA63B83298364
:10E1C0004423B9F001C04F5FE981F0E0CF0101962F
:10E1D00087709927281769F0EC0FFD1FF682168BC0
:10E1E000E68E05FB002700F900AB415046A33687B9
:10E1F0008983DF91CF911F910F91FF90EF90089548
:10E200000F931F93CF93DF93EC01062F642F809120
:10E2100050068695869586958770388129813213B8
:10E22000EFC010E00332110508F0EAC0F801E9542C
:10E23000FF4F97C300E326C000E321E0C0C002EA1D
:10E2400022E04AE064E6DAC00AE222E045E06FE557
:10E25000CE0170DF01E22AE045E06FE5CE016ADF22
:10E260000AE222E045E06FE5C9C002EC23E04AE0A3
:10E2700060E5CE015FDF02E423E04AE06CE3CE011B
:10E2800059DF00E221E065C001E221E045E066E4FB
:10E29000CE0150DF22E04FE062E3CE014BDF22E00F
:10E2A0004FE062C002E221E045E06EE6CE0142DFCF
:10E2B00003E221E045E097C000E025E045E062E3AD
:10E2C000CE0138DF25E045E06AE5CE0133DF02E02C
:10E2D00024E043E06EE692C003E22AE045E060E518
:10E2E000CE0128DF01E224E145E060E5CE0122DF36
:10E2F00003E22AE045E038C002E625E044E16AE0B6
:10E300007DC002E22AE044E062E3CE0113DF01E2D5
:10E3100024E148E066E4CE010DDF02E22AE048E0B5
:10E3200062E3CE0107DF01E224E144E04DC00AE2EE
:10E330002AE002C002E222E345E04BC001E203C052
:10E3400002E201C003E22AE044E160E057C002E1DA
:10E3500022E04AE039C002E423E044E16CE3CE016C
:10E36000E9DE02EE23E044E160E548C000E321E09D
:10E3700048E22AC0813009F443C000E121E04AE0CC
:10E380006BE43CC08130E1F100E121E04AE061E46E
:10E3900035C000E121E046E031C000E3D9CF813053
:10E3A00079F100E1D5CF00E112C003E303C002E33D
:10E3B00001C001E323E04FE00CC001E329E144E1A7
:10E3C00003C000E321E04EE166E418C001E321E070
:10E3D0004AE068E713C002E321E04AE06AE70EC0C2
:10E3E00003E321E04AE06CE709C000E520E04AE0F1
:10E3F00062E804C000ED20E04AE062E3CE019ADE6C
:10E40000DF91CF911F910F91089546E4682F88EC1A
:10E4100091E0F6CE462F682F88EC91E0F1CE9091F6
:10E420005C0691FF03C0862F0C947B14EECFCF9235
:10E43000DF92EF92FF920F931F93CF93DF93EC0144
:10E44000062F142F47FF03C0842F0E947B14D7FF91
:10E4500006C0D195C195D1098AE10E947B140023A1
:10E4600069F0023019F464E670E002C06AE070E01E
:10E47000CE0126D2262FC22FD72FF82E64E670E0C9
:10E48000CE011ED29B01FB01EC016115710591F1DA
:10E490006A307105C4F06AE070E0C90111D26B0105
:10E4A0007C01653171051CF48EE68C0D05C08CE88D
:10E4B0008C0D0E9477148EE60E947B14F701309732
:10E4C00069F001E001C000E084E68E0F0E947B1439
:10E4D000011104C0209741F18C2F0AC0209721F12F
:10E4E000CE016AE070E0ECD19E01281B390BC90116
:10E4F000845713C084570E9477140023A9F0023078
:10E5000079F46AE070E08F2D90E0DAD1C82F86E0D0
:10E51000860F0E947B148CE88C0F0E94771404C035
:10E5200086E08F0D0E947B1411161CF4812F0E942F
:10E530007B14DF91CF911F910F91FF90EF90DF90AF
:10E54000CF90089586B380958E7708958FEF8ABB1C
:10E550001BBA91E897BB9EE798BB9EE394BB91ECF6
:10E5600095BB11BA82BB98E092B997EF93B910921C
:10E5700061001092620094E1909364009BEF90938D
:10E58000650080938D0DD4B714BE80E487B985E80B
:10E5900086B987E083BF8CE981BF82E085BD83E4D3
:10E5A00087BF1FBC8AE08EBD10928B0082E88093EB
:10E5B0008A0080E280937D00789489E395E49093CB
:10E5C0004C0180934B010E944B5D882319F00E94FF
:10E5D000F06606C00E94055C0E94F0660E940D5D18
:10E5E00091E080B38095837C813419F49093C601C7
:10E5F000F8CF823849F4F89466E072E088E00E942F
:10E60000F8630E941267FFCFD0903A068D2D0E94CA
:10E610003C5E98DF982F9670963031F48091C60159
:10E6200082608093C60125C0C0E081FD05C086954B
:10E63000CF5FC630D1F71DC08C2F0E94A75C882306
:10E64000C1F0C0933A068C2F0E943C5E81E00E948C
:10E65000315D0E94C46224E04EEF51E060E086E14B
:10E660000E94D36388E10E9433330E9412670E94A4
:10E670005C120E94D41080916D0686FD0E94706924
:10E6800081E0809339010E944C1A109239018091E7
:10E690006906895F0E947D14D3FD76C08091530680
:10E6A00084FF05C08091500682FD47C03DC0809127
:10E6B0005C06882319F06CE187E0B1DE0E9428191E
:10E6C0000E94C46220E046E753E060E080E00E94E0
:10E6D000CF628091590684FD08C000E12AE04EE532
:10E6E00056E068E380E00E949D630E9412670E94EA
:10E6F0005C120E944D160E941E168C010E94821010
:10E70000EC01C057DE4F0E9412670E9428190E9438
:10E710004D160E941E167C0115DF8111C3CFE01635
:10E72000F10609F45CC0BECF0E94915F883C910560
:10E7300020F48FEE91E00E9478190E944D1680918E
:10E740002101909122016EE070E0A6D060933D011E
:10E750000E948F190E94AA1990915006987B21F46B
:10E760008FED91E00E9478198091C701882331F0E4
:10E7700084EB91E00E9478191092C7010E945C120C
:10E78000809155020E9477149091050192609093B8
:10E7900005011092EA0660E08AED97E00E94AC471E
:10E7A000BBDB8DE028E130E00FB6F894A89521BDE1
:10E7B0000FBE81BD2AE43AE230934E0120934D0111
:10E7C00080913A06D81629F081E00E94315D0E94BE
:10E7D0002D5E81E0809348020E94F51BFDCF0E94D0
:10E7E0008210C817D90709F08ECF5CCF88EC91E072
:10E7F00040CC05D0332312F48A1B9B0B10C0A29F80
:10E80000B001B39FC001A39F700D811D1124911D04
:10E81000B29F700D811D1124911D0895F0DFB7FF87
:10E820000895821B930B0895EADFA59F900DB49F76
:10E83000900DA49F800D911D11240895B7FFF4CF72
:10E84000F3DF821B930B0895DB018F939F93ECDF23
:10E85000BF91AF91A29F800D911DA39F900DB29F7C
:10E86000900D11240895991B79E004C0991F961703
:10E8700008F0961B881F7A95C9F78095089587FB45
:10E88000082E062687FD819567FD6195ECDF0EF465
:10E89000919507FC81950895AA1BBB1B51E107C008
:10E8A000AA1FBB1FA617B70710F0A61BB70B881F20
:10E8B000991F5A95A9F780959095BC01CD010895AF
:10E8C00097FB072E16F4009406D077FD08D0E4DFFE
:10E8D00007FC05D03EF4909581959F4F0895709563
:10E8E00061957F4F0895A1E21A2EAA1BBB1BFD0163
:10E8F0000DC0AA1FBB1FEE1FFF1FA217B307E4071F
:10E90000F50720F0A21BB30BE40BF50B661F771F76
:10E91000881F991F1A9469F7609570958095909556
:10E920009B01AC01BD01CF010895052E97FB16F4A4
:10E9300000940FD057FD05D0D6DF07FC02D046F477
:10E9400008C050954095309521953F4F4F4F5F4FF0
:10E95000089590958095709561957F4F8F4F9F4F4B
:10E960000895EE0FFF1F0590F491E02D0994FB012F
:10E97000DC0102C001900D9241505040D8F708953B
:10E980006817790768F4FB01DC01E40FF51FA40F99
:10E99000B51F02C002900E9241505040D8F7089522
:10E9A000E6CFDC0101C06D9341505040E0F708957F
:10E9B000DC01CB01FC01E199FECF06C0FFBBEEBB41
:10E9C000E09A31960DB20D9241505040B8F708953B
:04E9D000F894FFCFE9
:10E9D400F00064000A02FF000000E30D9B0D9B0D94
:02E9E4009B0D89
:00000001FF
